:020000040800F2
:100000000000022039A6000839A500083DA5000817
:1000100051A5000853A5000855A5000800000000E0
:1000200000000000000000000000000057A50008CC
:1000300059A50008000000005BA500085DA50008A8
:1000400089A6000889A6000889A6000889A60008D4
:1000500089A6000889A6000889A6000889A60008C4
:1000600089A6000889A6000889A6000889A60008B4
:1000700089A6000889A6000889A6000889A60008A4
:1000800089A6000889A6000889A6000800000000CB
:1000900000000000000000000000000089A6000829
:1000A00089A6000889A6000889A6000889A6000874
:1000B00061A500086DA5000889A6000889A60008AA
:1000C00089A6000889A6000889A6000889A6000854
:1000D00089A6000889A6000889A60008000000007B
:1000E00089A6000889A6000889A60008000000006B
:1000F00000000000000000000000000089A60008C9
:100100000000000089A6000889A6000889A600084A
:1001100000000000000000000000000000000000DF
:1001200089A6000889A6000889A6000889A60008F3
:1001300089A6000800000000000000000000000088
:1001400000000000000000000000000079A5000889
:1001500089A6000889A6000889A6000889A60008C3
:1001600089A6000889A60008000000000000000021
:10017000000000000000000000000000000000007F
:100180000000000089A60008000000000000000038
:0801900089A6000889A60008F9
:1001C0000348044B834202D0034B03B118477047E6
:1001D000C4090020C40900200000000005480649A9
:1001E0000B1AD90F01EBA301491002D0034B03B145
:1001F00018477047C4090020C4090020000000000F
:1002000010B5064C237843B9FFF7DAFF044B13B15E
:100210000448AFF300800123237010BDC4090020FF
:10022000000000009004010808B5044B1BB104490C
:100230000448AFF30080BDE80840CFE700000000AD
:10024000C80900209004010853B94AB9002908BF21
:1002500000281CBF4FF0FF314FF0FF3001F0DEB837
:10026000ADF1080C6DE904CE00F006F8DDF804E00D
:10027000DDE9022304B070472DE9F047089E0D46E2
:1002800004468846002B4DD18A42944668D9B2FA7A
:1002900082F252B101FA02F3C2F1200120FA01F117
:1002A0000CFA02FC41EA030894404FEA1C45210C79
:1002B000B8FBF5FE1FFA8CF705FB1E8341EA0343EA
:1002C0000EFB07F199420BD91CEB03030EF1FF3033
:1002D00080F01E81994240F21B81AEF1020E634410
:1002E0005B1AA4B2B3FBF5F005FB103344EA0344F8
:1002F00000FB07F7A7420AD91CEB040400F1FF3307
:1003000080F00881A74240F2058164440238E41B72
:1003100040EA0E4000211EB1D4400023C6E900434C
:10032000BDE8F0878B4208D9002E00F0EE80002156
:10033000C6E900050846BDE8F087B3FA83F1002955
:100340004AD1AB4202D3824200F2F980841A65EBB3
:10035000030301209846002EE2D0C6E90048DFE7FB
:1003600002B9FFDEB2FA82F2002A40F09180A1EBDE
:100370000C054FEA1C471FFA8CFE0121B5FBF7F371
:1003800007FB1350250C45EA00450EFB03F0A8427D
:1003900008D91CEB050503F1FF3802D2A84200F290
:1003A000CB8043462D1AA4B2B5FBF7F007FB1055DE
:1003B00044EA05440EFB00FEA64508D91CEB0404E4
:1003C00000F1FF3502D2A64500F2BB802846A4EB1F
:1003D0000E0440EA03409EE7C1F120078B4022FA59
:1003E00007FC4CEA030C20FA07F405FA01F31C435E
:1003F000FD404FEA1C4900FA01F3B5FBF9F8200C67
:100400001FFA8CFE09FB185540EA054508FB0EF063
:10041000A84202FA01F20BD91CEB050508F1FF3ADC
:1004200080F08880A84240F28580A8F102086544E7
:100430002D1AA4B2B5FBF9F009FB105544EA0545A5
:1004400000FB0EFEAE4508D91CEB050500F1FF349C
:100450006CD2AE456AD90238654440EA0840A0FB38
:100460000294A5EB0E05A542C846A64656D353D026
:100470005EB1B3EB080265EB0E0505FA07F722FA49
:1004800001F3CD401F43C6E900750021BDE8F087A8
:10049000C2F1200320FA03F10CFA02FC25FA03F35F
:1004A00095400D434FEA1C471FFA8CFEB3FBF7F152
:1004B00007FB11302B0C43EA004301FB0EF098427E
:1004C00004FA02F408D91CEB030301F1FF382FD220
:1004D00098422DD9023963441B1AADB2B3FBF7F031
:1004E00007FB103345EA034500FB0EF3AB4208D986
:1004F0001CEB050500F1FF3816D2AB4214D90238C7
:100500006544ED1A40EA014138E73146304607E7D5
:100510008646E5E61846FAE64B45A9D2B9EB02084D
:1005200064EB0C0E0138A3E74046EAE7204694E767
:100530004146D1E7D0467BE7023B654432E70846B7
:1005400009E76444023842E703685A004CBF43F0AD
:10055000004323F000431844704700BF2DE9F843DF
:1005600029B34F1E044615463E464FF0000808EBDF
:10057000060101EBD171491004EBC1094846FFF7B0
:10058000E3FF0346C80008308F42204409D0AB4245
:1005900009D8FFF7D9FF0138A8420AD201F10108B2
:1005A000E5E7AB4205D9884501D04E1EDFE74FF0A5
:1005B00000094846BDE8F883012807D0022807D083
:1005C000044B00280CBF18460020704702487047B3
:1005D00002487047910C0008950C0008990C00081F
:1005E00030B5234B83B004468D1E3BB301A928468A
:1005F000AFF30080E8B101992A46FFF7AFFF01464B
:10060000B8B1FFF7A1FF4B68A064012B2CD0002BE1
:1006100001F1040024DBFFF797FF0023C4E9130373
:100620000368002B11DBFFF78FFF2061002003B070
:1006300030BD00230920236103B030BD0D4B0E49AE
:10064000C91AC91018460191D6E7C3F30360FFF732
:10065000B3FF0028206114BF0020092003B030BD83
:100660000123C4E91303DBE7002323610520DEE750
:100670000000000028180108881C01080368DA0738
:1006800010B5044606D49B0700F1480009D500F0D8
:100690005BFC2368590709D51A070ED5DB0613D56D
:1006A00010BD00F049FC23685907F5D404F1D000CF
:1006B00000F052FC23681A07F0D404F5A87000F08B
:1006C00053FC2368DB06EBD404F5E870BDE810406A
:1006D00000F08EBC092070470346006800B1184442
:1006E000704700BF704700BF70B504460E46316CBE
:1006F0002046FFF775FF054688B9326C62612369B1
:1007000032462146012098470828F0D0072806D114
:100710002846316CFFF7E6FF301D00F001FC00F0C9
:100720007FFE00BF2DE9F0470D1DD0F80C80D0F8FA
:100730001890074614460FCDADF5727D0DF10C0CE7
:10074000ACE80F000FCDACE80F000FCDACE80F0008
:1007500095E80F0002AE4FF0000E8CE80F00C6F8CF
:1007600000E020E0336C7B614FF4F07231467AA8F0
:1007700001F0AEF93B697AAA394650469847889B02
:1007800073642146CDE9006905463B463A4601209F
:10079000C0470446E0B94FF4F0727AA9304601F040
:1007A00097F9082D1AD1316C3846FFF719FF093433
:1007B0005FFA84FA05460028D4D0B36B73643A46D6
:1007C000CDE900693B464AF010010120C04700B165
:1007D000092528460DF5727DBDE8F087072DF7D174
:1007E0002046316CFFF77EFF03A800F099FB00BFA5
:1007F000406C7047F0B5CB6B0B6401F1040C0E46F6
:100800000546BCE80F00F9B001AC0FC4BCE80F000E
:100810000FC4BCE80F000FC49CE80F004FF0FF3777
:1008200084E80F00009706E02B696A46294698473E
:100830000828044608D110992846FFF7D1FE002861
:10084000F2D0092079B0F0BD6846FFF717FF062CFB
:10085000F7D131462846FFF747FF00BFC160D96B8B
:1008600082611964002219465CE700BF70B5C66852
:1008700043690B64AEB903690A4604460D46014656
:1008800002209847072805D008280FD1294620467E
:10089000FFF72AFF3046296CFFF724FF281D00F0E0
:1008A0003FFB0122FFF73EFF00F0BAFD00F0B8FD6C
:1008B000C2681AB1CA6B0A64002233E79AE700BF24
:1008C000704700BF836801460BB10120184770478D
:1008D000012912D009D873B90F2A0CD800EB820273
:1008E00018465368009A136070470339012994BF72
:1008F000012002207047022070470846704700BF61
:1009000000B585B00A46002303A900911946FFF7F8
:10091000DFFF039805B05DF804FB00BF012912D08A
:1009200009D873B90F2A0CD800EB8200009A12681C
:100930004260184670470339012994BF0120022004
:100940007047022070470846704700BF10B584B05A
:10095000002303AC039200940A461946FFF7DEFF1A
:1009600004B010BD70B5D36B136402F1040C0546DE
:100970000C46BCE80F00ADF50E7D0DF15C0EAEE847
:100980000F00BCE80F00AEE80F00BCE80F00AEE8B7
:100990000F009CE80F004FF0FF368EE80F00169610
:1009A00010E0FFF7D3FF214616A8A847034616AA72
:1009B0006946082083B9049B9847052806460CD051
:1009C000092809D026996846FFF70AFE03466A46B9
:1009D0000C2116A8002BE4D0092616A8FFF74EFE1E
:1009E00030460DF50E7D70BD2DE9F04FCC6C89B011
:1009F0001E4654F8043B06940D46174600F00308C3
:100A0000002E79D01A0C1B0405938DF81D200223AB
:100A1000D2B204EB82048DF81C302B6DB8F1020FBA
:100A200008BFAC6B13F001030CD005A9384600F0E9
:100A300079FB18B9082009B0BDE8F08F092009B08A
:100A4000BDE8F08FD4F800A0BAF1000FEDD001930B
:100A500000F008030293022E4AD0B4F800A0B4F8C4
:100A600002900434AB6C29F0010B0F2138469B44F3
:100A7000FFF746FF834539D82AF001039B4483459D
:100A800094BF002001204FEA490303F002030AF05B
:100A9000010A43EA0A03012B49D0022B32D0002B72
:100AA000CCD1B8F1000F02D0002840F0CD80043442
:100AB000D4F800A0BAF1000FCDD105A9384600F056
:100AC00031FB0028BAD1019B002BB3D00F2138464F
:100AD000FFF716FF0E2102463846FFF737FF38466C
:100AE0006A4A0F21FFF732FF0720A8E70020CAE774
:100AF000D4F804900834B5E71B0205930323ADF83E
:100B00001C308AE7236823F0004BB8F1000F45D171
:100B100028B1029A002A5CD0BBF1000F74D0002BE0
:100B200000DA04340BF1010B04EB8B04C0E7B8F1DD
:100B3000000F19D1B0B163682268991C4FEAD272D4
:100B40003FF47CAF05F158010133049100F090802F
:100B5000201DFFF7C1FD04AB014628460EF000F84A
:100B600000285BD10834A3E70D213846D5F8209042
:100B7000FFF7C6FE8145F5D1AB6A9C42F2D1204613
:100B8000FFF7E2FC0F2102463846FFF7DFFE38464A
:100B90002A460021FFF7DAFE072050E70D213846EC
:100BA000D5F82090FFF7ACFE814501D02368B6E769
:100BB000AB6A9C42FAD104230022C5E90B23E31857
:100BC000C5F828B06B632368002B59DB0123019320
:100BD000A8E705F15803CDF80C8004F1040AB046EB
:100BE00091461E460EE050460496FFF775FD002222
:100BF000014604AB284609F101090AF1040A0DF087
:100C0000AFFFE0B9D945EED10D213846FFF778FEA8
:100C1000049BAC62C5E90803062010E781460D215C
:100C20003846FFF76DFEB9F1020F286225D12B4639
:100C3000049A43F82C2F6B62AC620620FFE646460E
:100C40002368DDF80C806AE72046FFF77DFC04345A
:100C50000246AC63284614460DF0DCFF00283FF442
:100C6000EDAE384622460F21FFF770FE0720E6E67C
:100C70000D213846FFF744FE2862049B6B62DBE7D8
:100C80000BF1010004EB80007AE700BFBD00010812
:100C90000023A9E60123A7E60223A5E62DE9F043F8
:100CA0000646C3B015461C46042900F2BF80DFE8A3
:100CB00001F09E57BD2D0300002C40F0B780102A94
:100CC00000F2B4800368D80600F1F98020AF3846FE
:100CD00000F098F9B46B394600234FF0010C0CFA80
:100CE00003F22A42204603F1010303D050F8042BFB
:100CF0000A600446042B01F10401F0D13846B463C4
:100D000000F076F9002043B0BDE8F083032C40F0FA
:100D10008D8094B204EB1243102B4FEA124500F27F
:100D2000858003681F0700F1D28020AF384600F0AD
:100D30003DF9B26B07EBC50154B10B46D01A01EB7C
:100D4000C401E4001D5843F8045B8B42FAD12244ED
:100D50003846B26300F008F9002043B0BDE8F083E4
:100D6000012C4FEA124895B25CD0052C5ED108EBFD
:100D70000509B9F1200F59D8B8F10F0F79D9A94653
:100D8000002D40F08A80B36B6DB320AF4FF00009A7
:100D900007EBC807043F03EBC50553F8041B47F8EE
:100DA000041FAB42F9D1B9F1000F0FD06F46414695
:100DB000102938BF102107EBC101843903EBC905A5
:100DC00053F8040B41F8040FAB42F9D1012C00F0A9
:100DD0008680B8F10F0FB56347D9B9F1000F02D083
:100DE000684600F0B9F8002043B0BDE8F083ECB9E4
:100DF000806B23461FFA82FC0124371D04FA03F29C
:100E000012EA0C0F014604D051F8042B47F82320B6
:100E100008460133102BF1D115F40055E3D1B0632E
:100E2000284604E008EB0503102B03D9022043B049
:100E3000BDE8F083B8F10F0FF8D83368DA0706D5AC
:100E4000304623F0030340F8483B00F079F820AF28
:100E5000384600F075F8B36B002D97D11D46043568
:100E6000B563384600F068F8BDE720A800F06CF8DC
:100E7000B3E7B9F1100F40D9A9F110093368D907C8
:100E800008D523F00103304643F0020340F8483B05
:100E900000F05EF8B9F1000F32D033685A0720D461
:100EA000B8F10F0F25D96F463846C8F1100500F08C
:100EB00057F8002DB36B7FF77AAF20AF68E723F0C8
:100EC0001003336006F5E87000F09CF8FEE623F0AE
:100ED0000803036000F5A87000F068F825E720AF6C
:100EE000BDE7304623F0040340F8D03B00F038F86B
:100EF000D6E720A800F02CF8D5E74FF00009BDE7B1
:100F0000B8F10F0F3FF63FAF20AF384600F020F8A2
:100F1000B36B002D7FF43AAF384600F015F862E766
:100F200000F1340191E838009C46A6464CF8045D77
:100F300090E8FF0FE54600BD90EC210B704700BF25
:100F400080EC210B704700BF90EC200B704700BF76
:100F500080EC200B704700BFD0EC200B704700BF27
:100F6000C0EC200B704700BFF0EC0201F0EC021166
:100F7000F0EC0221F0EC0231F0EC0241F0EC025115
:100F8000F0EC0261F0EC0271F0EC0281F0EC029105
:100F9000F0EC02A1F0EC02B1F0EC02C1F0EC02D1F5
:100FA000F0EC02E1F0EC02F1704700BFE0EC02016E
:100FB000E0EC0211E0EC0221E0EC0231E0EC024155
:100FC000E0EC0251E0EC0261E0EC0271E0EC028145
:100FD000E0EC0291E0EC02A1E0EC02B1E0EC02C135
:100FE000E0EC02D1E0EC02E1E0EC02F1704700BF7E
:100FF000B0FC0181B0FC0191B0FC01A1B0FC01B1D9
:10100000704700BFA0FC0181A0FC0191A0FC01A1E0
:10101000A0FC01B1704700BFEC4600B52DE90050BF
:101020002DE9FF1F4FF000032DE90C0001A9FFF788
:10103000E1FBDDF840E012B0704700BFEC4600B5C0
:101040002DE900502DE9FF1F4FF000032DE90C00A2
:1010500001A9FFF70BFCDDF840E012B0704700BFBC
:10106000EC4600B52DE900502DE9FF1F4FF00003BD
:101070002DE90C0001A9FFF71BFCDDF840E012B0E0
:10108000704700BFEC4600B52DE900502DE9FF1F69
:101090004FF000032DE90C0001ABFFF7DFFBDDF89B
:1010A00040E012B0704700BFEC4600B52DE900509B
:1010B0002DE9FF1F4FF000032DE90C0001AAFFF7F7
:1010C00051FCDDF840E012B0704700BF027A0346E1
:1010D0007AB9427AA2B14168013A10B44272086802
:1010E00003220C1D1A7202025C60000E10BC1A6012
:1010F00070470068013A1A7202021A60000E7047C7
:10110000B020704700B585B0002303AA00921946AD
:101110000C22FFF7DDFB039805B05DF804FB00BF70
:10112000F0E700BF2DE9F043054685B00E464FF0CD
:1011300000083046FFF7CAFFB028044600F0BA8026
:10114000070620D500F0F003802B4DD0902B36D031
:10115000A02B60D0B02B74D0C02B00F08B8000F09F
:10116000F803D02B0BD100F007020132052342F423
:10117000002201212846FFF791FD0028D9D009203F
:1011800005B0BDE8F0838300DBB21F1D0DF10C0933
:1011900000231946CDF800900D222846FFF798FB52
:1011A000039BCDF8009060064CBFDF1BFF180023A7
:1011B0000D22194628460397FFF7B0FBB9E700F068
:1011C0000D030D2BDBD003AF002300F00F021946F7
:1011D00000972846FFF77CFB002300970D22194655
:1011E0002846FFF79BFBA4E73046FFF76FFF24027A
:1011F0002043B0F5004FC2D004010023A2B219462B
:101200002846FFF74BFD0028B9D114F4004F18BF52
:101210004FF001088DE7C24302F007034FF47F62ED
:101220001A41010702F47F624FF0000348BF42F405
:10123000804219462846FFF731FD00283FF479AF78
:101240009DE7B1283BD0B22800F09380B32841D06D
:1012500000F0FC03B42B92D000F00702013201230E
:1012600042F4002219462846FFF718FD00283FF4F3
:1012700060AF84E7C6284AD0C72854D000F0F803EE
:10128000C02B63D0C82868D0C9287FF478AF304617
:10129000FFF71CFF020300F00F0002F47022013080
:1012A0000243012105232846FFF7F8FC00283FF4FC
:1012B00040AF64E7B8F1000F18D0002060E7304677
:1012C000FFF704FF024600283FF459AF10F0F00387
:1012D000C8D054E73046FFF7F9FE020300F00F03D1
:1012E000013302F470221A430123BBE703AC4346E7
:1012F0000E22414600942846FFF7EAFA009443463E
:101300000F2241462846FFF709FB404638E73046A2
:10131000FFF7DCFE020300F00F03013302F470223A
:101320001A4303239EE73046FFF7D0FE024600280B
:101330003FF425AF10F0F0037FF421AF04212846DD
:10134000FFF7ACFC00283FF4F4AE18E700F00F0202
:101350000132032342F4202284E73046FFF7B6FE31
:1013600000F0F00200F00F031032013343EA0232C2
:1013700097E700230DF10C090D221946CDF80090D6
:101380002846FFF7A5FA3046FFF7A0FE02064FF009
:1013900002040CD5039B00F07F00A040184403908A
:1013A0003046FFF793FE030604F10704F2D4039BD3
:1013B000CDF8009000F07F02A24003F501731A44BB
:1013C0000023039219460D222846FFF7A7FAB0E63C
:1013D00010B5C26C536884B04FF0030C08321C0285
:1013E00008461B0E01A9019402928DF80CC08DF8DD
:1013F0000D30FFF797FE04B010BD00BF08B5FFF732
:101400008FFE806C08BD00BF08B5FFF789FEC06C79
:10141000C379023300EB830008BD00BF704700BFF3
:1014200008B5062000F06EFD012009F0B5F800BFF8
:10143000002301461A46184602F07CBA014B186890
:10144000704700BF0000002038B5084B084D5B1BFB
:101450009C1007D0043B1D44013C55F804399847C3
:10146000002CF9D1BDE838400FF018B8981C0108DD
:10147000941C010870B50D4E0D4D761BB61006D0AC
:10148000002455F8043B01349847A642F9D1094E8F
:10149000094D761B0EF0FCFFB61006D0002455F85F
:1014A000043B01349847A642F9D170BD881C01085D
:1014B000881C0108941C0108881C0108024B014685
:1014C000186800F00BB800BF00000020024B014676
:1014D000186803F0B7BA00BF000000202DE9F04FF4
:1014E00001F10B06162E83B0044624D8102900F211
:1014F000BA8000F055FC102618220220B74F3A445B
:10150000A2F1080153688B4200F0BA805A68D9688A
:1015100022F003021A449D68E9608D60516841F031
:1015200001012046516003F1080500F03BFC28460C
:1015300003B0BDE8F08F36F0070600F19480B142A9
:1015400000F2918000F02CFCB6F5FC7FC0F0968193
:10155000730A00F08F80042B00F26B81B30903F152
:10156000390003F1380CC3009C4F3B44A3F108053C
:101570005B689D4206D10CE0002980F22B81DB687C
:101580009D4206D05A6822F00302911B0F29F3DD19
:1015900060463D69DFF848C265457CD06A6822F044
:1015A0000302931B0F2B00F37781002BC7E904CCB8
:1015B00080F26881B2F5007F80F01681D3087968E7
:1015C00001334FEA521E012202FA0EF20A4357F883
:1015D00033E0C5F808E007EBC3010839E9607A6039
:1015E00047F83350CEF80C508310012199409142B6
:1015F00057D8114206D120F003004900114200F1F2
:101600000400FAD007EBC0094D468646D5F80C8099
:10161000454508D119E1002B80F22081D8F80C80D3
:10162000454500F01281D8F8042022F00302931BF4
:101630000F2BF0DD2046D8E9025408EB060146F0F6
:101640000106C8F80460EC60A56043F00104C7E936
:101650000411C1E902CC4C6048F8023000F0A2FB52
:1016600008F1080502E00C2323600025284603B09A
:10167000BDE8F08F4FF4007340204FF03F0C73E74C
:10168000D3689A4208BF02307FF440AF3D69DFF86B
:1016900050C1654582D17A688310012199409142F9
:1016A000A7D9BD686B6823F00308464503D8A8EBAB
:1016B00006030F2B7EDCDFF82C91D7F80824D9F82D
:1016C00000300132334405EB080A00F02F8103F5A6
:1016D00080530F3323F47F6B2BF00F0B59462046BA
:1016E00000F062FB411C024600F0EF80824500F2F0
:1016F000EA80D9F804105944C9F804100B4600F0E8
:101700004B81D7F8081401311BBFA2EB0A0A5344DE
:10171000C7F80824C9F8043012F0070300F012815A
:10172000C3F108010A44C3F5805193440831A1EB89
:101730000B01C1F30B0A514620460192009300F0C1
:1017400033FB421CDDE9003200F04B81831A03EBCE
:101750000A0BD9F80400BA604BF001030AEB000150
:10176000BD425360C9F8041000F02281B8F10F0F98
:1017700040F220816B68A8F10C0020F0070003F014
:10178000010303436B604FF0050C2B180F28C3E9CE
:1017900001CC00F22D8153681546D9F82C208A42DD
:1017A000D9F8302038BFC9F82C108A4238BFC9F8A0
:1017B00030108CE0AA1943F0010346F001066E6078
:1017C0002046BA60536000F0EDFA0835284603B0B1
:1017D000BDE8F08FD9681A449DE600BF30040020B0
:1017E00038040020E0090020B2F5206F4FEA5223B0
:1017F00063D3142B00F2B88003F15C01C9005B33A2
:1018000007EB010E7958AEF1080E8E4500F091807D
:101810004B6823F00303934202D989688E45F7D1C0
:10182000D1F80CE07A68C5E9021ECEF80850CD6008
:10183000DAE6142B59D9542B00F29E80330B03F1B6
:101840006F0003F16E0CC3008EE60EF1010E1EF068
:10185000030F05F108057FF4D9AE51E04244454637
:101860005368D8F80C1043F00103536055F8083F53
:101870002046D9608B6000F095FAF7E6F00806F193
:1018800008023BE62A442046536843F001035360B4
:10189000083500F087FAE9E6A919204646F0010666
:1018A00043F001046E60C7E90411C1E902CC4C6049
:1018B000AB5000F077FA0835D8E6930903F1390107
:1018C000C90038339CE7BD4260D0BD686B6823F027
:1018D000030B5E45ABEB060302D80F2B3FF76AAF55
:1018E000204600F05FFA0025C0E603F15C0003F13A
:1018F0005B0CC30038E659F808394B4540F0968038
:1019000010F0030F00F1FF30F5D17B6823EA0103EB
:101910007B60490099423FF6C4AE19B9C1E649005F
:101920000EF1040E1942FAD070466BE603F1100B6B
:10193000D4E69A104FF001087B6808FA02F21A43C5
:101940007A6070E702EB0B014942C1F30B0A514682
:1019500020460193009200F027FA431CDDE90023A2
:101960007FF4F4AE9A46F4E6542B26D8130B03F119
:101970006F01C9006E3343E7B3F5AA7F26D8F30B96
:1019800003F1780003F1770CC300EDE5D9F80430DA
:101990005B44C9F80430B4E6CAF30B0000287FF4B6
:1019A000B0AEBD6808EB0B0343F001036B60F4E6D7
:1019B0001546F2E60123536092E7B3F5AA7F21D8DA
:1019C000D30B03F17801C900773319E740F2545281
:1019D000934221D8B30C03F17D0003F17C0CC300CA
:1019E000C2E5083B9B44ABEB020B4FF0000AB0E6AC
:1019F00005F10801204603F025F8BD68D9F8041068
:101A00006B68CAE640F254518B420BD8930C03F139
:101A10007D01C9007C33F3E64FF47E737F204FF0E5
:101A20007E0CA1E54FF47E717E23E9E67B6870E7CA
:101A300001F0FF01102A2BDB10F0070F08D010F87F
:101A4000013B013A8B422DD010F0070F42B3F6D183
:101A5000F0B441EA012141EA014122F007047FF09C
:101A600000070023F0E80256083C85EA010586EAF3
:101A7000010685FA47F5A3FA87F586FA47F6A5FA2F
:101A800087F68EB9EED1F0BC01F0FF0102F007023B
:101A900032B110F8013B013A83EA010313B1F8D1E6
:101AA0000020704701387047002D06BF35460338C7
:101AB000073815F0010F07D1013015F4807F02BF00
:101AC000013015F4C03F0130F0BC0138704700BF51
:101AD000844641EA000313F003036DD1403A41D339
:101AE00051F8043B40F8043B51F8043B40F8043BF8
:101AF00051F8043B40F8043B51F8043B40F8043BE8
:101B000051F8043B40F8043B51F8043B40F8043BD7
:101B100051F8043B40F8043B51F8043B40F8043BC7
:101B200051F8043B40F8043B51F8043B40F8043BB7
:101B300051F8043B40F8043B51F8043B40F8043BA7
:101B400051F8043B40F8043B51F8043B40F8043B97
:101B500051F8043B40F8043B51F8043B40F8043B87
:101B6000403ABDD2303211D351F8043B40F8043B27
:101B700051F8043B40F8043B51F8043B40F8043B67
:101B800051F8043B40F8043B103AEDD20C3205D337
:101B900051F8043B40F8043B043AF9D2043208D02F
:101BA000D2071CBF11F8013B00F8013B01D30B88A1
:101BB00003806046704700BF082A13D38B078DD07F
:101BC00010F003038AD0C3F10403D21ADB071CBF51
:101BD00011F8013B00F8013B80D331F8023B20F8BB
:101BE000023B7BE7043AD9D3013A11F8013B00F8F4
:101BF000013BF9D20B7803704B7843708B7883707C
:101C00006046704788420DD98B1883420AD900EB91
:101C1000020CBAB1624613F801CD02F801CD994227
:101C2000F9D170470F2A0ED8034602F1FF3C4AB1A2
:101C30000CF1010C013B8C4411F8012B03F8012F2E
:101C40006145F9D1704740EA01039B0750D1A2F1E9
:101C5000100370B501F1200C23F00F0501F1100EF7
:101C600000F11004AC441B095EF8105C44F8105CF1
:101C70005EF80C5C44F80C5C5EF8085C44F8085CA8
:101C80005EF8045C44F8045C0EF1100EE64504F1C5
:101C90001004E9D1013312F00C0F01EB031102F033
:101CA0000F0400EB031327D0043C24F003064FEA93
:101CB000940C1E441C1F8E465EF8045B44F8045FBF
:101CC000B442F9D10CF1010402F0030203EB8403E6
:101CD00001EB840102F1FF3C4AB10CF1010C013B24
:101CE0008C4411F8012B03F8012F6145F9D170BD27
:101CF00002F1FF3C03469BE72246EBE7830730B542
:101D000048D0541E002A3FD0CAB2034601E0013C2D
:101D10003AD303F8012B9D07F9D1032C2DD9CDB26D
:101D200045EA05250F2C45EA054536D9A4F11002F0
:101D300022F00F0C03F1200EE6444FEA121C03F1CF
:101D4000100242E9045542E9025510327245F8D1B9
:101D50000CF1010214F00C0F03EB021204F00F0C53
:101D600013D0ACF1040323F003030433134442F80B
:101D7000045B9342FBD10CF003042CB1CAB21C44A7
:101D800003F8012B9C42FBD130BD64461346002C66
:101D9000F4D1F9E703461446BFE71A46A446E0E744
:101DA000704700BF704700BF38B5074D002204469A
:101DB00008462A6008F01EFC431C00D038BD2B6882
:101DC000002BFBD0236038BD140A002038B5D0F8B2
:101DD000DC420CB1002038BD80210546FFF77EFBB8
:101DE0000246C5F8DC0230B1031F7C3243F8044FD1
:101DF0009342FBD1EEE74FF0FF3038BD1F29F8B515
:101E0000054609D8D0F8DC620C4617464EB156F8A4
:101E1000240046F82470F8BD162303604FF0FF300D
:101E2000F8BD8021FFF75AFB0646C5F8DC0240B139
:101E3000031F00F17C05002143F8041F9D42FBD1E4
:101E4000E5E74FF0FF30F8BD1F2938B5054621D82A
:101E5000D0F8DC220C466AB152F8213053B1012B84
:101E600016D0591C10D00025204642F8245098471F
:101E7000284638BD284600F003F922460146284688
:101E8000BDE8384000F0E6B816230360012038BDF5
:101E9000002038BD162303604FF0FF3038BD00BF6F
:101EA0001F292CD8D0F8DC2238B50C46054682B163
:101EB00052F8243002EB84024BB1591C1AD0012B8A
:101EC00016D00025204615609847284638BD0120C9
:101ED00038BD8021FFF702FB0246C5F8DC0258B18D
:101EE000031F00217C3043F8041F9842FBD1DFE739
:101EF000032038BD022038BD4FF0FF3038BD4FF011
:101F0000FF30704738B5154B1F281D6820D8D5F80D
:101F1000DC22044662B152F820304BB1012B15D0BF
:101F2000591C0FD0002542F820509847284638BD4C
:101F3000284600F0A5F8224601462846BDE838406C
:101F400000F088B816232B60012038BD002038BD72
:101F500016232B604FF0FF3038BD00BF000000207B
:101F6000134B1F2870B51E6809D80D46D6F8DC1231
:101F7000044649B151F8240041F8245070BD16239D
:101F800033604FF0FF3070BD80213046FFF7A6FA76
:101F90000146C6F8DC0240B1031F00F17C0C0022B0
:101FA00043F8042F6345FBD1E4E74FF0FF3070BDE9
:101FB0000000002038B50C4B1D68D5F8DC420CB190
:101FC000002038BD80212846FFF788FAC5F8DC02DA
:101FD00038B1031F00F17C0243F8044F9342FBD158
:101FE000EEE74FF0FF3038BD0000002038B5184B49
:101FF0001F281D6828D8D5F8DC22044682B152F883
:10200000243002EB84024BB1591C1BD0012B17D09A
:102010000025204615609847284638BD012038BD68
:1020200080212846FFF75AFA0246C5F8DC0258B16B
:10203000031F00217C3043F8041F8342FBD1DEE7FD
:10204000032038BD022038BD4FF0FF3038BD00BF3F
:102050000000002070B50C46084D034600262046BF
:1020600011461C462E6008F08FFA431C00D070BD4C
:102070002B68002BFBD0236070BD00BF140A00202A
:1020800008F080BA0CB410B59CB01EAB6FF00044E1
:10209000CDE906140291084953F8042B059102A9D1
:1020A0000193049400F01AFA029B00221A701CB0EB
:1020B000BDE8104002B070470802FFFF0EB410B533
:1020C0009DB06FF000411FABCDE9060104910949B5
:1020D00053F8042B0290084C0868019302A9059458
:1020E00000F0FCF9029B00221A701DB0BDE8104000
:1020F00003B07047000000200802FFFF000000004E
:10210000A2EB0300704700BF02780B78012A28BFBA
:102110009A42F5D16DE9044540EA0104CDE9026730
:102120006FF0000C4FEA447212B380EA010414F01D
:10213000070F6AD100F0070420F0070004F0030540
:1021400021F007014FEAC505F0E8042314F0040F5D
:10215000F1E804670CFA05F462EA040266EA040690
:102160000AD063EA0403624667EA0407664603E0AE
:10217000F0E80423F1E8046782FA4CF582EA0604E9
:10218000A4FA8CF46CBB83FA4CF583EA0705A5FA34
:102190008CF595B950E9022351E9026782FA4CF5B2
:1021A00082EA0604A4FA8CF483FA4CF583EA070564
:1021B000A5FA8CF52543DBD09CB92DBAB5FA85F488
:1021C00024F0070427FA04F1DDE9026723FA04F397
:1021D00003F0FF0001F0FF01FDE80445A0EB010062
:1021E000704724BAB4FA84F424F0070426FA04F100
:1021F000DDE9026722FA04F202F0FF0001F0FF01BC
:10220000FDE80445A0EB0100704714F0030F3CD13A
:1022100010F0030428D150F8082B51F8083B82FA3B
:102220004CF582EA0305A5FA8CF55DB950F8042C4B
:1022300051F8043C82FA4CF582EA0305A5FA8CF5C4
:10224000002DE8D02DBAB5FA85F424F0070423FA5E
:1022500004F122FA04F202F0FF0001F0FF01FDE8B0
:102260000445A0EB010070474FEAC40420F00300CE
:1022700050F8082B21F0030151F8083B0CFA04F444
:1022800062EA040263EA0403C9E710F003041AD007
:10229000A1EB040120F00300E40750F8042B06D062
:1022A0000FD28B785FFAA2F4E41A06D12BB1CB7867
:1022B0005FFAB2F4E41A00D11BB920465DF8104B66
:1022C000704701F1040150F8042BCC0721F0030101
:1022D00051F8043B48D824D222F07F4482FA4CF5CE
:1022E00094EA1325A5FA8CF50AD165B951F8043B97
:1022F00084EA0204B4EB036F0ED150F8042BEBE731
:102300004FEA132355E035F07F454DD10878FDE8BD
:102310000445C0F1000070474FEA126203F0FF036A
:1023200047E002EA1C4482FA4CF594EA1345A5FA08
:102330008CF50AD165B951F8043B84EA0204B4EB88
:10234000034F0CD150F8042BEBE74FEA134330E076
:1023500015EA1C4528D10B884FEA124229E04FEAC2
:10236000124203EA1C4324E002F0FF0482FA4CF517
:1023700094EA1365A5FA8CF50AD165B951F8043BC6
:1023800084EA0204B4EB032F09D150F8042BEBE7E5
:102390004FEA13630DE015F0FF0F05D10B684FEA0C
:1023A000122223F07F4304E04FF00000FDE80445D3
:1023B000704712BA1BBA82FA4CF482EA0304A4FAF8
:1023C0008CF5B5FA85F402FA04F203FA04F34FEA45
:1023D0001260FDE80445A0EB1360704700000000A8
:1023E00000000000000000000000000000000000ED
:1023F00000000000000000000000000000000000DD
:1024000090F800F06DE9024520F007016FF0000C34
:1024100010F0070491F820F040F049804FF00004DC
:102420006FF00700D1E9002391F840F000F10800B7
:1024300082FA4CF2A4FA8CF283FA4CF3A2FA8CF3EF
:102440004BBBD1E9022382FA4CF200F10800A4FA56
:102450008CF283FA4CF3A2FA8CF3E3B9D1E90423AA
:1024600082FA4CF200F10800A4FA8CF283FA4CF3E1
:10247000A2FA8CF37BB9D1E9062301F1200182FA9B
:102480004CF200F10800A4FA8CF283FA4CF3A2FAA1
:102490008CF3002BC6D0002A04BF04301A4612BAAF
:1024A000B2FA82F2FDE8024500EBD2007047D1E9B2
:1024B000002304F00305C4F100004FEAC50514F041
:1024C000040F91F840F00CFA05F562EA05021CBF12
:1024D00063EA050362464FF00004A9E72DE9F04FD7
:1024E000BFB0884691460D930C9002F0B3FB036891
:1024F00014931846FFF784FFB8F80C3013901806B1
:1025000004D5D8F81030002B00F0CA860023CDE99E
:1025100022330F9312931593099300240023CDE9DE
:1025200010342EAA2192924699F80030002B00F028
:1025300080814C4604E014F8013F002B00F0C58078
:10254000252BF8D1B4EB090540F0C3802378002B8C
:1025500000F06F8100234FF0FF3265788DF867300F
:1025600004F10109184608920A939B4609F10109F2
:10257000A5F12002582A00F2D380DFE812F05302BE
:10258000D100D1004E02D100D100D100D100D10044
:10259000D10001024902D1000C021102D100440213
:1025A0005900590059005900590059005900590063
:1025B0005900D100D100D100D100D100D100D1000B
:1025C000D100D100D1002B026401D1006401D100FF
:1025D000D100D100D1005B02D100D1007800D10040
:1025E000D100D100D100D1006800D100D1006E022D
:1025F000D100D100D100D100D100D100D100D10053
:10260000D100D1006002C4016401640164018F0241
:10261000C401D100D1000303D100ED027A00D2023F
:10262000CD02D100AB02D1006A00D100D1009402EA
:10263000A5F13002002119F8015B01EB810102EBE9
:102640004101A5F13002092AF5D90A9190E74BF032
:10265000100B1BF0200100F048810D9B073323F085
:102660000703596853F8080B0D9301230EE04BF054
:10267000100B1BF0200100F02B810D9B073323F082
:102680000703596853F8080B0D93002300248DF8B5
:102690006740089A561C00F084822BF0800606964C
:1026A00050EA010640F07B82002A40F00383002BB1
:1026B00040F024851BF001030B9300F0908530233C
:1026C0008DF8B7300DF1B70690E2B4EB090500F0D4
:1026D000B080239B2B442393229B0133072BCAE911
:1026E0000095229305DC0AF1080A099B2B44099303
:1026F0002CE70C9821AA414602F0EAFF18B90DF127
:10270000B80AF2E7B846B8F80C3013F0400F099B4E
:1027100018BF4FF0FF33099309983FB0BDE8F08F21
:10272000002B40F0C587002D00F0838000238DF83A
:10273000673001238DF8905007930B9324AE00234C
:10274000CDF818B008930E93069B13F0020302D045
:10275000079A02320792069A12F0840B05D10A9A60
:102760000799571A002F00F39883239C9DF8672040
:102770008AB1229A0DF1670101320134CAF80010C2
:10278000072A4FF0010123942292CAF8041000F3A3
:10279000CD830AF1080A83B1229B1AAA01330234BD
:1027A000CAF80020072B4FF0020223942293CAF8A4
:1027B000042000F3C9830AF1080ABBF1800F00F07E
:1027C0009582089B0B9AA3EB020BBBF1000F00F361
:1027D000CF82069BDF0500F112820B9BCAF8043002
:1027E0001C44229BCAF800600133072B23942293D8
:1027F00000F347830AF1080A069B5B0705D50A9B8D
:10280000079A9D1A002D00F3AB83DDE90932079981
:102810008A42ACBF9B185B180993002C40F0E282FF
:102820000023229399F800300DF1B80A002B7FF4B1
:1028300080AE239B002B3FF466AF0C9821AA414643
:1028400002F046FF5FE7002B40F0D4870D9B073373
:1028500023F00702F2E80234CDE91034DDE9103448
:1028600024F000440D921E4618462146B54B4FF009
:10287000FF3206F097F9002840F0B884B14B30469B
:1028800021464FF0FF3206F06FF9002840F0AE8489
:10289000DDE910010022002306F05CF9002840F079
:1028A000E0869DF86740A84E2BF080030693A74B67
:1028B0000022472DC8BF1E460323CDE907320B93E4
:1028C0000E92002C3FF440AF079B013307933BE788
:1028D0001BF0100348D11BF0400145D00D9A52F86F
:1028E000040B0D92194680B2D0E61BF0100341D1C3
:1028F0001BF040013ED00D9A52F8040B0D92194680
:1029000080B20123C2E6002B40F07C871BF0200F31
:102910000D9B68D0073323F007031A465B6852F813
:10292000080B0D921946002BC0F23084089B01332E
:1029300000F06B852BF08003069350EA01039DF8AD
:10294000674000F0D783DDF818B00A2871F1000362
:1029500080F0FC84303001238DF8B700CDF818B03A
:102960000B930DF1B70641E10D9B53F8040B0D934A
:102970000B468BE60D9B53F8040B0D93012385E664
:102980000D9A52F8041B0A91002980F223840A99B7
:102990000D9249420A9199F800504BF0040BE5E57D
:1029A000494611F8015B2A2D00F0A387A5F13002FA
:1029B000092A894698BF002100F2208719F8015B97
:1029C00001EB810102EB4101A5F13002092AF5D9A1
:1029D0000891CDE5002B40F019874BF0100B1BF050
:1029E000200F0D9B96D153F8040B0D931BF0100F85
:1029F00040F0C7831BF0400F00F0C38340F3C031A9
:102A00000B4600B28FE799F800504BF0800BADE514
:102A100099F8005001232B20A8E599F800504BF0BD
:102A2000010BA3E599F8005000287FF49FAD012326
:102A300020209BE599F800504BF0080B96E50D9B84
:102A400000228DF8672053F8042B0D9301238DF895
:102A5000902007930B9324AE71E6002B40F0DA86AA
:102A60003B4B12931BF0200125D00D9B073323F025
:102A70000703596853F8080B0D931BF0010F0BD097
:102A800050EA010308D030238DF868308DF8695082
:102A90004BF0020B0223F9E50223F7E599F8005009
:102AA0004BF0400B62E5002B40F0A086294B1293BF
:102AB0001BF02001D9D11BF0100340F05D831BF007
:102AC000400100F059830D9A52F8040B0D921946FB
:102AD00080B2D2E70D9C089B54F8046B00278DF858
:102AE0006770002E00F0C8845A1C00F0E9831A4673
:102AF00039463046FEF79CFF002800F05F86831BB6
:102B00000B9323EAE3730D9408979DF86740CDF883
:102B100018B007930E97D4E699F800504BF0200BAD
:102B200024E50D9B53F8040B0D93302378258DF885
:102B30006830084B12934BF0020B8DF8695000215E
:102B40000223A3E5FFFFEF7FC0110108C4110108B4
:102B5000E4110108D0110108002B40F05F861BF042
:102B6000200F40F087831BF0100F40F0E1831BF033
:102B7000400F00F0DD830D9B099953F8042B0D9352
:102B80001180D1E499F800506C2D03BF99F80150E1
:102B90004BF0200B09F101094BF0100BE6E4DDF8D6
:102BA00018B0012B3FF4D1AE022B00F08B802EAE7B
:102BB00000F00703C00840EA4170C908303350EA0A
:102BC0000107324606F8013DF2D11BF0010F00F07B
:102BD0008780302B00F084803023023A06F8013CD5
:102BE0002EAB9B1ACDF818B00B931646089B0B9A88
:102BF0009342B8BF1346079300230E9361E6652DF9
:102C000040F3F980DDE910010022002305F098FF70
:102C1000002800F0DE81229BC14ACAF8002001335F
:102C200001340122072B23942293CAF8042000F3D5
:102C3000FC830AF1080A1B9B0F9A934203DB069B55
:102C4000D8077FF5D9AD139B149A1C44CAE9002319
:102C5000229B23940133072B229300F300840AF173
:102C6000080A0F9B5D1E002D7FF7C6AD102D229B1D
:102C7000AC4F40F3CE83DDF830B0102605E00AF10A
:102C8000080A103D102D40F3C48301331034072B84
:102C9000CAE90076CDE92234F1DD21AA4146584641
:102CA00002F016FD00287FF42EADDDE922340DF18F
:102CB000B80AE6E7012B00F04C85022BDDF818B0CE
:102CC0007FF475AF129A2EAE00F00F030009D35CAB
:102CD00006F8013D40EA0170090950EA0103F3D109
:102CE0002EAB9B1BCDF818B00B937FE70A9B079A7E
:102CF000A3EB020BBBF1000F7FF763ADBBF1100F2D
:102D0000229A884F26DD214610230C9C06E0ABF169
:102D1000100BBBF1100F0AF1080A1ADD0132103155
:102D2000072ACAE90073CDE92221F0DD21AA414634
:102D300020460DF1B80A02F0CBFC00287FF4E3AC8A
:102D4000ABF1100BBBF1100FDDE922214FF01003A6
:102D5000E4DC0C4601325C44072ACDE92224CAF89F
:102D60000070CAF804B000F36D830AF1080A28E580
:102D7000BBF1100F229A6B4F26DD214610230C9CCD
:102D800006E0ABF1100BBBF1100F0AF1080A1ADDD7
:102D900001321031072ACAE90073CDE92221F0DDA2
:102DA00021AA4146204602F093FC00287FF4ABACF8
:102DB000ABF1100BBBF1100FDDE922210DF1B80AC8
:102DC0004FF01003E4DC0C4601325C44072ACDE9E5
:102DD0002224CAF80070CAF804B000F3C0810AF1D6
:102DE000080AF6E40C9821AA414602F071FC00287A
:102DF0003FF416AD87E40F9B012B40F35D81229DCC
:102E0000CAF80060013501340123072D239422956F
:102E1000CAF8043000F3C4810AF1080A139B149A1B
:102E200001351C44072DCAE90023CDE9225400F3E3
:102E3000C4810AF1080ADDE910010022002305F02F
:102E40007FFE002840F05F810F9B0135013B01367A
:102E50001C44072DCAF800602295CAF80430239458
:102E600000F33B810AF1080A159BCAF804300135CA
:102E70001C44072D1DABCDE92254CAF800307FF762
:102E8000B9AC0C9821AA414602F022FC00287FF43C
:102E90003AAC239C0DF1B80AAEE4102FDDE92221F3
:102EA0002FDDCDE916354B460C9DB14610243E462C
:102EB00008464746984604E0103E102E0AF1080ADC
:102EC00017DD0132184B1030072ACAE90034CDE96A
:102ED0002220F1DD21AA394628460DF1B80A02F078
:102EE000F7FB00287FF40EAC103E102EDDE9222007
:102EF000E7DCDDE9163501464046B84637464E4622
:102F0000814601327C18072A0749CAF80470CDE9C6
:102F10002224CAF8001000F335820AF1080A25E4D9
:102F200000120108BC040108AC0401080C981693B7
:102F300021AA414602F0CCFB00287FF4E4AB239C9D
:102F4000169B0DF1B80A26E40C9821AA414602F01E
:102F5000BFFB00287FF4D7AB239C0DF1B80A2CE40B
:102F6000102D229B1FDD0C9F102604E0103D102D1C
:102F70000AF1080A17DD01339A4A1034072BCAE90F
:102F80000026CDE92234F1DD21AA414638460DF173
:102F9000B80A02F09DFB00287FF4B5AB103D102D60
:102FA000DDE92234E7DC01338E4ACAF804502C44B0
:102FB000072BCDE92234CAF800207FF726AC0C9805
:102FC00021AA414602F084FB00287FF49CAB239C9D
:102FD0001BE41B99002940F3E481DDE90E379F4291
:102FE000A8BF1F46002F0BDD229B01333C44072B5B
:102FF000CAE900672394229300F3C2830AF1080A06
:103000000E9D002FA8BFED1B002D00F369811B9DB5
:103010000F9B9D4280F23881139B149A1C44CAE98D
:103020000023229B23940133072B229300F31E835A
:103030000AF1080A0F9B0E9A5D1B9F1AAF42A8BFA8
:103040002F46002F0EDD229BCAF804700133164470
:103050003C44072BCAF800602394229300F39F831B
:103060000AF1080A002FA8BFED1B002D7FF7C4ABA3
:10307000102D229B5C4F40F3CC81DDF830B0102640
:1030800005E00AF1080A103D102D40F3C28101331A
:103090001034072BCAE90076CDE92234F1DD21AAEC
:1030A0004146584602F014FB00287FF42CABDDE9C2
:1030B00022340DF1B80AE6E7069BDA073FF59FAE2A
:1030C000229DCAF80060013501340123072D2394A5
:1030D0002295CAF804307FF7C5AE0C9821AA414664
:1030E00002F0F6FA00287FF40EABDDE922540DF170
:1030F000B80AB9E6089B002B40F02B830023089305
:103100000B932EAE72E50F9B5E1E002E7FF7ACAECA
:10311000102E354F40F3F081CDF820904FF0100B7A
:10312000C146DDF8308005E00AF1080A103E102E95
:1031300040F3DF8101351034072DCAE9007BCDE96A
:103140002254F1DD21AA4946404602F0C1FA002886
:1031500040F06883DDE922540DF1B80AE6E70C98E7
:1031600021AA414602F0B4FA00287FF4CCAA239C9D
:103170000DF1B80AFFF72DBB0D9B53F8040B0D930F
:103180007BE4C1170B46002BBFF6D0AB40424FF09B
:103190002D0461EB41018DF867400123FFF779BAF7
:1031A0000C9821AA414602F093FA00287FF4ABAABA
:1031B000DDE922540DF1B80A30E60C9821AA414607
:1031C00002F086FA00287FF49EAADDE922540DF170
:1031D000B80A30E699F800500D92FFF7C7B92EAE45
:1031E00004E500BFAC040108BC040108DDE91001DE
:1031F00002460B4605F0D6FC002840F03C83089BB5
:10320000013325F020030B9300F0C682472B00F01A
:103210009780DDE910124BF48073171E0693C0F2FD
:103220003F82109B079300231693662D00F0708158
:10323000462D00F06D810B9B079A0C98452B1FA91A
:1032400008BF089B04911CA903911BA90CBF5C1C1F
:10325000089C029102213B460194009100F042FC3F
:10326000672D064640F082821BF0010F00F0988126
:10327000344464E10D9B099853F8041B0D93C21765
:10328000C1E90002FFF750B9069BD9073FF5C4AE6C
:10329000DDE90E239F1A5D1BAF42A8BF2F46E1E672
:1032A0000C984021FEF71AF9C8F80000C8F8100081
:1032B000002800F02D834023C8F81430FFF726B90A
:1032C00030460D940897CDF818B0FFF799F820EA2A
:1032D000E0739DF867400B9007930E97FFF7F1BAE4
:1032E000102D229BAB4F40F3AF813A4608964746DC
:1032F0000C9E4FF0100B904605E00AF1080A103DB5
:10330000102D40F39D8101331034072BCAE9008B47
:10331000CDE92234F1DD21AA3946304602F0D8F950
:1033200000287FF4EFA9DDE922340DF1B80AE6E7C1
:103330000D9B099953F8042B11600D93FFF7F4B816
:10334000089B002B08BF0123089362E72EAE069569
:103350000A22002307460D46FCF776FF303206F8B6
:10336000012D0023384629460A22FCF76DFF0A2F5B
:1033700075F10003ECD22EAB9B1B069D0B93CDF891
:1033800018B033E40C98169321AA414602F0A0F934
:1033900000287FF4B8A9239C169B0DF1B80AFFF70B
:1033A000E5B9229B7C4ACAF800200133013401228E
:1033B000072B23942293CAF8042000F364810AF1B6
:1033C000080A002961D1069B0F9A03F001031343F9
:1033D0003FF412AA139B14991A19CAE90013229BED
:1033E00023920133072B229300F366810AF1080A26
:1033F0000F99CAF8006001338C18072BCDE92234ED
:10340000CAF804107FF7F6A93BE59DF86740FFF77F
:103410009CBA01332C44072BCAF80070CAF8045038
:10342000CDE922347FF7E6A92BE50C9821AA414685
:1034300002F04EF900287FF466A9239C0DF1B80A2A
:10344000FFF7F9BB0C9821AA414602F041F9002888
:103450007FF459A9239C0DF1B80AFFF7B2B90C9873
:1034600021AA414602F034F900287FF44CA9239C9C
:103470000DF1B80AFFF7F5BB062B28BF0623474E10
:103480000B930D940793FFF75AB9139B14981A19CD
:10349000CAE90003229B23920133072B229300F3F6
:1034A0000B810AF1080A0029A2DA4D421031394F86
:1034B00080F2BB81DDF830B0102405E00AF1080A83
:1034C000103D102D40F3B18101331032072BCAE9B2
:1034D0000074CDE92232F1DD21AA4146584602F0BE
:1034E000F7F800287FF40FA9DDE922320DF1B80AC0
:1034F000E6E7C846DDF82090CAF80070013534448C
:10350000072DCDE92254CAF804607FF7ABACE4E59F
:103510001FA904911CA903911BA9089C02910321D6
:103520003B460194079A0C98009100F0DBFA06469E
:1035300004193378302B00F090811B9B1C440798B2
:1035400039460022002305F0FBFA002840F0AE8047
:103550001F9BA34206D230215A1C1F9219701F9B39
:103560009C42F9D89B1B0F930B9B472B1FD0662DBA
:1035700040F0D6811B9B0E93002B0BF0010B40F308
:10358000EC8008995BEA010240F098810E9B07935A
:103590000B9321E0BC04010800120108F811010896
:1035A0001F9B9B1B0F930B9B472B40F0B9811B9BD1
:1035B0000E93D91C1BDB089A934218DCDDE90E320E
:1035C0009342C0F207811BF0010F40F06E8123EAA5
:1035D000E37207920B936725169B002B00F0CA80BD
:1035E0002D238DF8673000230893FFF76DB9023D56
:1035F0000E9A8DF87450531E002B1B93B6BFC2F168
:1036000001032B222D22092B8DF875206EDC30331F
:103610008DF8773030238DF87630042315930F9A88
:10362000159B012A13440B9340F336810B9B139A8D
:1036300013440B9323EAE373079300230E93CBE722
:103640004246089EB846174601332C44072BCDE965
:103650002234CAF80070CAF804503BDC0AF1080AA8
:10366000D5E42D248DF86740FFF71DB90C9821AAE9
:10367000414602F02DF800287FF445A81B9D239CAD
:103680000DF1B80AD6E40C9821AA414602F020F8C0
:1036900000287FF438A81B99239C0DF1B80A90E606
:1036A0002D23079102F100471693BEE5234659E703
:1036B0008DF86700FFF737B80C9821AA414602F051
:1036C00007F800287FF41FA8DDE922321B990DF1CD
:1036D000B80AE8E60C9821AA414601F0F9FF002853
:1036E0007FF411A8239C0DF1B80A90E40DF1830436
:1036F0008D4F2246104687FB0321DA17C2EBA10249
:1037000002EB8201A3EB4101303100F8011C1946A4
:103710006329134600F1FF32ECDC3033D9B2831E4B
:103720009C4202F8011C40F2F08013460DF1760233
:1037300001E013F8011B02F8011B9C42F9D10DF1C5
:1037400085030DF176021B1A13441DAA9B1A1593CB
:1037500065E7DDF818B0FFF7FDB8089A5BEA0203E9
:1037600040F0B480012307930B9335E7472D3FF4D6
:103770007BAD7DE5169B9DF867400893FFF7A1B8E8
:103780000C9821AA414601F0A3FF00287EF4BBAFAC
:10379000239C0DF1B80A33E40623089339E50C980D
:1037A00021AA414601F094FF00287EF4ACAF1B9D96
:1037B0000F9B239C5D1B0DF1B80A53E4089B0D94ED
:1037C000CDF818B09DF8674007930B9308900E90C2
:1037D000FFF777B8139A0F9B13440E9A0B93002AA6
:1037E0007CDD23EAE37307936725F5E68DF8670030
:1037F000FFF75CB98DF86700FFF728B80022089240
:10380000FEF7B6BE8DF86700FFF780B88DF8670049
:10381000FFF7E3B88DF86700FFF722B98DF867006E
:10382000FFF79DB9C846FEF76EBF01332A44072B48
:10383000CDE92232CAF80070CAF804507FF7D6AD3D
:103840000C9821AA414601F043FF00287EF45BAFAB
:10385000DDE922320DF1B80ACAE50798394600229F
:10386000002305F06DF900287FF467AE089BC3F1D3
:1038700001031B9362E6119B2C4E002BB8BF2D2435
:103880002BF080030693A8BF9DF86740284BB8BF74
:103890008DF86740FFF70CB81BF001020E927FF421
:1038A000C5AE23EAE373079396E60E9B139A13447F
:1038B0000B9323EAE373079367258DE6139A13446A
:1038C000194421EAE1730B91079385E6139B0133B9
:1038D0001A4422EAE2730B9207937DE60E9B0B9A41
:1038E000C3F101031A4422EAE2730B92079367259E
:1038F00072E60D9A99F80150894652F8041B0D9210
:1039000041EAE1710891FEF731BE0223159386E684
:103910000C9A0C2313604FF0FF330993FEF7FCBEA3
:103920001B9B0E9364E600BF67666666C8110108BC
:10393000CC11010870B4184C2568D5F848411CB367
:1039400065681F2D25DC38B9AB1C0135656044F86E
:103950002310002070BC704704EB850C0228CCF8C3
:103960008820D4F888614FF0010202FA05F246EA95
:103970000206C4F88861CCF80831E5D1D4F88C315E
:103980001343C4F88C31DFE705F5A674C5F8484148
:10399000D6E74FF0FF30DDE7A804010838B5074D42
:1039A0000022044608462A6006F018FE431C00D098
:1039B00038BD2B68002BFBD0236038BD140A0020D3
:1039C0002DE9F04F03690C69A34283B0C0F28680F1
:1039D000013C01F11405A30000F11408009355F80F
:1039E000243058F8242001338A469A4208EB840197
:1039F000814605EB84070191B2FBF3F638D300232F
:103A0000AE4640469B465EF8041B02681FFA81FCE6
:103A100006FB0C33090C4FEA134C06FB01CC99B2A0
:103A2000ABEB01011FFA8CF311FA82F1C3EB1242E6
:103A300002EB214289B241EA0241774540F8041B7A
:103A40004FEA1C434FEA224BDDD2009B58F803306B
:103A500073B9019B043B984504D307E0984504F1F2
:103A6000FF3403D253F80429002AF7D0C9F81040D4
:103A70005146484601F0D2FB00282BDB0136404678
:103A8000002355F8041BD0F800C08AB29A1A0B0C18
:103A900012FA8CF2C3EB1C4303EB224392B242EACC
:103AA0000342AF4240F8042B4FEA2343E9D258F8CF
:103AB000242008EB84036AB9043B984504D307E04B
:103AC000984504F1FF3403D253F80429002AF7D0B3
:103AD000C9F81040304603B0BDE8F08F002003B0B5
:103AE000BDE8F08F2DE9F04F016C99B090469946F2
:103AF000CDE90489259D044641B1426C4A60012309
:103B000093408B6001F0D4F800232364B9F1000ADC
:103B1000B4BF012300232B60754BBCBF2AF0004AC1
:103B2000CDF814A033EA0A0300F0AA80DDE90423EB
:103B30001046194600220023CDE90A0105F000F8DD
:103B4000074670B1249A01231360269B002B00F0D6
:103B5000E28268481860431E0393039819B0BDE8D9
:103B6000F08F16AB019317AB00932046DDE90A23D3
:103B700001F0A4FC5FEA1A56054640F09780DDE9A3
:103B800016763E4406F23240202840F3B383C0F15B
:103B900040000AFA00FA06F2124028FA00F04AEA57
:103BA000000004F0EBFC0123013EA1F1F8710F933A
:103BB000514B002204F0A4FB47A3D3E9002304F0F7
:103BC00057FD47A3D3E9002304F09CFB8046304611
:103BD000894604F0E3FC44A3D3E9002304F048FD44
:103BE00002460B464046494604F08CFB8046894617
:103BF00004F0EEFF0022834600234046494604F0CD
:103C0000A9FF002840F07A82BBF1160F00F269820A
:103C10003A4B03EBCB03D3E90023DDE90A0104F0BF
:103C200099FF002870D00023BE1B0E93731E0BF16A
:103C3000FF3B069300F15C8200230993BBF1000F68
:103C400069DA099BCDF81CB0A3EB0B030993CBF108
:103C500000030D93229B092B4FF0000B64D8052B1A
:103C600040F34683043B22930026229B023B032B16
:103C700000F26686DFE813F05A0457044E0431045C
:103C8000249A42F20F73CAF3130A13605AEA080324
:103C90001AD1269B002B00F06286194B0393083340
:103CA000269A0398136019B0BDE8F08FDDE90A1277
:103CB000C2F31303084643F07F510F97A6F2FF3675
:103CC000169F41F4401173E7269B002B40F0E883D8
:103CD0000C4B039341E700BF61436F63A787D23F5B
:103CE000B3C8608B288AC63FFB799F501344D33FEB
:103CF0000000F07F011201080000F83FE005010814
:103D00000812010804120108BE1B731E069300F17D
:103D100085840E900990069B5B44CDE9063B002309
:103D20000D93229B092B9AD90023CDE9223301263A
:103D30004FF0FF330C960893089B129300216164A7
:103D4000204600F08FFF0390002800F00186039BBF
:103D50002364089B0E2B00F21381002E00F01081CB
:103D60000799002940F35C84AE4B01F00F0203EB8E
:103D7000C2034FEA2118C905D3E9006740F1148452
:103D8000A94BDDE90A01D3E9082304F09BFDCDE945
:103D9000100108F00F084FF0030AB8F1000F13D01C
:103DA000DFF8849218F0010F09D030463946D9E97E
:103DB000002304F05DFC0AF1010A06460F465FEAA3
:103DC000680809F10809EDD1DDE9100132463B46EA
:103DD00004F078FD804689460E9B43B1934B002248
:103DE0004046494604F0B6FE002840F03085504673
:103DF00004F0D4FB42464B4604F03AFC8C4B0022C4
:103E000004F080FAA1F15073CDE910011193089BE1
:103E1000002B00F09780079B1493089B13930C9B37
:103E2000002B00F0A584139A7E4B8249039E03EB7E
:103E3000C20353E90223002004F044FDDDE910230E
:103E400004F05EFACDE910014946404604F0C0FE98
:103E5000074604F0A3FB02460B464046494604F0E1
:103E60004FFA3037DDE9102306F8017B804689469A
:103E700004F070FE002840F02985CDF854B00027EA
:103E8000DDE910AB1095139D13942AE00137AF4282
:103E900080F22C85684B50465946002204F0E8FB1E
:103EA000654B002282468B464046494604F0E0FBC3
:103EB0008946804604F08CFE044604F06FFB0246FF
:103EC0000B464046494604F01BFA303406F8014BD5
:103ED00052465B468046894604F03CFE002840F08E
:103EE000F38442464B465149002004F009FA5246F9
:103EF0005B4604F02FFE0028C8D0DDE91343109D77
:103F0000039A079302E0964200F0C884B24616F87E
:103F1000013D392BF7D00133DBB23370079B0133FE
:103F20000793C8E1504604F039FB42464B4604F083
:103F30009FFB3F4B002204F0E5F9A1F15073CDE95E
:103F4000100111933D4B40464946002204F0D8F938
:103F5000DDE910894B46424606460F4604F018FE3E
:103F60008146002840F0AA84DDE91001024601F1F3
:103F700000433046394604F0EDFD002840F045830B
:103F8000179B002BC0F28C80079A0E2A00F38880C2
:103F9000244B03EBC203D3E900AB239B002B1BDABA
:103FA000089B002B18DC40F02E83244B0022504647
:103FB000594604F05DFB02460B46DDE90A0104F0B8
:103FC000D3FDDDF820904E46002800F0C782239BE9
:103FD000DDF80C80DF43C9E2DDE90A7852465B4632
:103FE0003846414604F06EFC04F0F2FD814609902B
:103FF00004F0D4FA52465B4604F03AFB039E0B46AB
:1040000002464146384604F07BF909F1300306F8D0
:10401000013B089B012B00F05C830694012704956B
:104020001C462AE0E0050108D00601080000F03F28
:1040300000001C400000E03F00002440000014404D
:1040400052465B464046494604F03CFC04F0C0FD45
:10405000054604F0A3FA52465B4604F009FB01371B
:104060000B4602464946404604F04AF905F1300342
:10407000A74206F8013B00F02983AC4B002204F074
:10408000F7FA002200238046894604F059FD0028F3
:10409000D6D0049D069C079B01330793B2460AE1E4
:1040A0000C9A002A3DD0229A012A40F39C82089B58
:1040B00003F1FF380D9B4345C0F26D82A3EB080866
:1040C000089B002BC0F23C83069A1A440692099A78
:1040D00017461A4409920121204600F0EBFE0646DD
:1040E00023E00123BE1B0E93731E06937FF5A4AD40
:1040F000C6F101030993002306939FE5584604F097
:104100004DFA42464B4604F01BFD00287FF47CAD7F
:104110000BF1FF3B78E5864B0393039819B0BDE89C
:10412000F08FDDF83480099F0C9E002F0CDD06997E
:1041300000290B4608DD099AB942A8BF3B46D21AAE
:10414000FF1ACB1A099206930D9BDBB10C9B002B37
:1041500000F05D82B8F1000F0FDD31464246204687
:1041600000F084FF2A4601460646204600F0D0FEB5
:1041700029460546204600F09BFD0D9BB3EB080247
:1041800040F0D8820121204600F094FEBBF1000FE0
:10419000814600F3B480229B012B40F386814FF0CF
:1041A000000A0120BBF1000F40F0B580069A1044D0
:1041B00010F01F0000F09380C0F12003042B40F3A7
:1041C000D283099BC0F11C000344024409930744B5
:1041D0000692099B002B05DD29461A46204600F071
:1041E000A5FF0546069B002B05DD49461A462046DD
:1041F00000F09CFF81460E9B002B40F03681089B0F
:10420000002B40F31D810C9B002B40F0A080079BEE
:1042100001330793DDF80C80DDF820A0012707E0CB
:10422000294600230A22204600F04CFD01370546AE
:1042300049462846FFF7C4FB574500F1300308F80C
:10424000013BEDDB089A002AC8BF9346039AD8BF0A
:104250004FF0010B93440027294601222046049386
:1042600000F064FF4946054600F0D8FF002840F3FF
:10427000A8811BF8013C039A0BF1FF3B04E05A456F
:1042800000F0AA811BF8013D392B0BF1010AF6D091
:1042900001338BF800304946204600F009FD56B145
:1042A0002FB1B74203D03946204600F001FD314618
:1042B000204600F0FDFC2946204600F0F9FC0023D2
:1042C0008AF80030249B079A1A60269B002B3FF443
:1042D00044AC0398C3F800A019B0BDE8F08F1C20CF
:1042E000099B03440993069B03440744069370E724
:1042F0000126BAE4C0F1200008FA00F051E40146BA
:104300005A46204600F0B2FE229B012B814640F324
:10431000B3814FF0000AD9F8103009EB8303186914
:1043200000F07AFDC0F1200040E700BF000024400B
:1043300000120108314600230A22204600F0C2FC88
:10434000129B002B064640F3E782CDE90783002F3E
:1043500000F31A81BAF1000F40F0D581B046049BFA
:10436000039F089903F001027B1E1944229B0C92C3
:10437000134309910A9349462846FFF721FB31462A
:104380008346284600F04AFF424649468246204678
:1043900000F064FFC26801460BF13003002A42D1ED
:1043A00006902846089300F039FF069904902046AD
:1043B00000F07EFC049A089B1AB90A99002900F0C3
:1043C0009B82BAF1000FC0F2638122994AEA010A86
:1043D0000C9951EA0A0100F05B81002A00F3B481D4
:1043E000099A3B7007F1010A9742D34600F0B28167
:1043F000294600230A22204600F064FC4645054673
:1044000031464FF000034FF00A02204612D000F070
:1044100059FC4146064600230A22204600F052FC81
:1044200057468046A7E72046049300F041FC049BD2
:104430000122C6E700F046FC5746064680469AE74A
:10444000229B022B79DC0C9B002B80D1079B4946D9
:10445000013328460793FFF7B3FADDF80CB000F1FB
:1044600030030BF8013B0027F6E64946284600F0EA
:10447000D5FE0028BFF6C3AE294600230A222046F7
:1044800000F020FC079B03F1FF380C9B0546002B36
:104490007FF450AF129B002B40F335820893B9E6AE
:1044A000AF4B03930333FFF7FBBBDDE90412002995
:1044B0007FF475AEC2F31303002B7FF470AEA94BEB
:1044C0001340002B00F0FE81099B01330993069BEA
:1044D000013306934FF0010A63E601230C93239BFB
:1044E000079A134412930133012B1F460893B8BF58
:1044F00001270021172F61647FF722AC01220423DA
:104500005B0003F11400B842114602F10102F7D931
:10451000616415E401230C93239B002B4CDD129363
:1045200008931F46E5E700230C93D8E700230C937C
:10453000F2E7129BCDF81C800893089B002B7FF4B8
:1045400046AD49460522204600F0BCFB01468146A7
:10455000284600F063FE00287FF739AD0398079FD7
:104560003123804600F8013B01370390494620463D
:1045700000F09EFB7B1CDDF80CA00793CDF80C80AF
:10458000002E7FF494AE96E631463A46204600F07F
:10459000CDFD0646DEE60D9BCDF83480A8EB030387
:1045A0009B444FF000088BE5DDE90A234FF0020A37
:1045B000CDE91023FFF7F1BB012323930893FFF705
:1045C000BBBB03D1049BDB073FF553AEDA461BF8B8
:1045D000013D302BFAD05EE6079B039A0133079327
:1045E0003123137057E60F9A002A00F0268103F258
:1045F0003343069ADDF834801A440692099A174626
:104600001A44099267E54FF000094E46DFE4294657
:104610000D9A204600F02AFD0546B3E50E9067E5A9
:1046200000F00F81079A504B564206F00F0203EB41
:10463000C203D3E90023DDE90A0104F019F83611B9
:104640008046894600F07181484F00234FF0020AEE
:10465000F20706D5D7E9002304F00AF80AF1010AA7
:104660000123761007F10807F2D1002B3FF4B4AB19
:1046700080468946FFF7B0BB049B002B7FF449AE10
:10468000DDE90412C2F31303002B3FF418AF40E638
:10469000002A12DD294601222046049300F046FD3F
:1046A0004946054600F0BAFD0028049B40F31881F6
:1046B000392B00F0F9800BF13103BA460AF8013BBF
:1046C000079B0133374607934646E4E50995069C68
:1046D000049D02460B4603F015FE52465B4680469B
:1046E000894604F055FA60B952465B464046494651
:1046F00004F026FA00283FF4CEAC099BD9077FF5D9
:10470000CAAC039A02E47168204600F0ABFA07468F
:10471000002800F00E81336902339A0006F10C0183
:104720000C30FDF7D5F939460122204600F0FEFC99
:10473000804614E62946204600F098FC054621E50F
:10474000DDE908239F1AC6E4392B00F0AD80BA4694
:104750000133B3E7079A01323746079246467BE5B5
:10476000041201080000F07FE0050108D0060108EE
:10477000DDF84CA0844901EBCA01DDE9102351E9C1
:10478000020103F075FFCDE910014946404604F0EF
:104790001FFA064603F002FF0B4602464946404612
:1047A00003F0AEFD039F53463036012B07F8016B33
:1047B0008046894600F0AE80139E039B1E44734BD7
:1047C00000224046494603F053FF8946804604F0E4
:1047D000FFF9824603F0E2FE0AF1300A02460B4678
:1047E0004046494603F08CFD07F801ABB7428046CE
:1047F0008946E4D1664B0022DDE9100103F082FD19
:1048000042464B4604F0A6F9002864D1DDE91023A6
:104810005F49002003F074FD42464B4604F0B8F9AE
:1048200000283FF4ADABB246013E1AF8013C302BF4
:10483000F9D0149B013307933DE5169BC3F1360372
:10484000D7E6DDE90A894FF0020AFFF7C5BA089BEF
:10485000002B3FF467AB129B002B7FF791AB079ABD
:10486000013ACDE913324046484B0022494603F055
:10487000FFFE804689460AF1010003F08FFE4246A2
:104880004B4603F0F5FE434B002203F03BFDA1F144
:104890005073CDE910011193FFF7C1BA079B0133A3
:1048A00007933123FFF739BB079BBB4601330793BF
:1048B000392337460BF8013B4646DCE44FF000094C
:1048C0004E464BE69A466CE4109D139C149B0133B4
:1048D0000793B246EFE4149B039A0793FFF716BBC6
:1048E0007FF4EBAEDA077FF5E8AEE1E6DDF854B031
:1048F000109D139CFFF744BB392BD5D0BAF1000FA4
:104900003FF7D9AED9E6229B022B3FF712AECDF886
:104910001C809BE53E466DE7229B022B3FF709AECC
:10492000129BCDF81C80089311E54FF0020AFFF7A7
:1049300053BA194B19483A4640F2EA2101F072FC89
:10494000002666643146204600F08CF9039078B961
:10495000114B124800224FF4D57101F063FC104B4B
:104960000393FFF7FAB83FF434ACC0F13C00B7E46E
:10497000039B236401224FF0FF33239612930C9282
:104980000893FFF7FDBA00BFE005010800002440CE
:104990000000E03F00001C4014120108281201082A
:1049A00008120108F8B5244F0C460646FDF7F8F941
:1049B000BA685568C4F57E630F3325F003052B44B0
:1049C00023F47F6323F00F03A3F58054B4F5805FD5
:1049D00007DB00213046FDF7E7F9BB682B4498421E
:1049E00004D03046FDF7DEF90020F8BD61423046C4
:1049F000FDF7DAF901300DD0104ABB682D1B45F0E8
:104A000001055D60136830461B1B1360FDF7CAF992
:104A10000120F8BD00213046FDF7C6F9BA68831AB7
:104A20000F2BDEDD43F001035360054B03491B6888
:104A3000C01A0860D5E700BF30040020E409002058
:104A400038080020002961D0F8B50C460646FDF76D
:104A5000A7F954F8042C7B4FA4F1080522F00101BA
:104A600005EB010CB868DCF80430604523F0030363
:104A700000F08B80D207CCF8043032D454F8082CE4
:104A8000AD1A1144AA6807F1080082426AD00CEB03
:104A90000304D4F804E0EC68D4601EF0010FA260B7
:104AA00000F0978041F001036B60CCF80010B1F585
:104AB000007F35D27A68CB08480901210133814053
:104AC0001143796007EBC30257F83310083AC5E980
:104AD000021247F83350CD603046BDE8F840FDF78C
:104AE00061B90CEB03025268D00710D4194407F1E6
:104AF0000800DCF80830834273D0DCF80C20DA6060
:104B0000936041F001036B606950D0E7704741F05A
:104B10000103B1F5007F44F8043CCCF80010C9D380
:104B2000B1F5206F4FEA512348D28B0903F13900C8
:104B300003F13802C300F818FB580838984259D0DE
:104B40005A6822F003028A4202D99B689842F7D140
:104B5000D868C5E902308560DD603046BDE8F840C0
:104B6000FDF720B90CEB03025268D20763D40B4463
:104B7000DCE90212CA60916043F001026A603046CB
:104B8000EB50BDE8F840FDF70DB90B44D10707D451
:104B900054F8082CAD1A1344D5E90212CA6091608A
:104BA00043F001026A60284ABD6012689A4293D8B5
:104BB000264B30461968FFF7F5FE8DE7142B0AD90E
:104BC000542B1FD80B0B03F16F0003F16E02C300CF
:104BD000B1E719448DE703F15C0003F15B02C30008
:104BE000A9E741F00103C7E90455C5E902006B607C
:104BF000695071E779689210012404FA02F20A43BD
:104C00007A60A6E7B3F5AA7F06D8CB0B03F178004C
:104C100003F17702C3008EE740F25452934206D864
:104C20008B0C03F17D0003F17C02C30083E74FF49A
:104C30007E737E227FE741F001036B60CCF80010A9
:104C40004AE700BF300400203C080020E0090020B3
:104C5000F030704700487047300900200048704726
:104C600030090020C36C70B505460C464BB153F8B3
:104C7000240080B1026843F824200023C0E90333F4
:104C800070BD2122042101F0F3FA0346E8640028F4
:104C9000EDD1002070BD012101FA04F6721D9200D1
:104CA000284601F0E5FA0028F3D0C0E90146E4E720
:104CB00031B1C36C4A6853F82200086043F82210EF
:104CC000704700BF2DE9F0410D6907460E461C46AE
:104CD00001F1140E0020DEF800108BB202FB03433A
:104CE0004FEA134C090C02FB01CC01309BB203EBE1
:104CF0000C4385424EF8043B4FEA1C44EBDC3CB1CC
:104D0000B368AB4207DD06EB850301355C613561B5
:104D10003046BDE8F081716838460131FFF7A2FFE7
:104D20008046A8B13269023206F10C0192000C30C3
:104D3000FCF7CEFEFB6C726853F82210316043F82A
:104D40002260464606EB850301355C613561DFE78D
:104D5000024B03484246B52101F064FA14120108DF
:104D60005C1201082DE9F8430C4628491E461746F7
:104D700003F1080281FB0231092E4FEAE273054676
:104D8000C3EB610339DD4FF0010C00214FEA4C0CFD
:104D9000634501F10101F9DC2846FFF763FF014695
:104DA00068B3089B4361092F4FF00103036112DCD4
:104DB0000A340927BE420BDDF61B264414F8013BDA
:104DC0000A22303B2846FFF77DFFA6420146F5D177
:104DD0000846BDE8F88304F10909C8463C4418F8C0
:104DE000013B0A22303B2846FFF76CFFA0450146F5
:104DF000F5D1A7F108044C44DCE70021CCE70A46D2
:104E0000034B0448CE2101F00DFA00BF398EE33880
:104E1000141201085C120108020C12040346CAB9FC
:104E20000304102013F07F4F04BF1B02083013F05F
:104E3000704F04BF1B01043013F0404F04BF9B00B0
:104E40000230002B05DB13F0804F00F1010008BF9A
:104E5000202070470020E5E70368024613F00700B2
:104E600007D0D9071DD498071FD55B081360012010
:104E7000704799B209B91B0C1020D9B209B9083092
:104E80001B0A190704BF1B090430990704BF9B08BC
:104E90000230D90703D45B0800F1010003D013608E
:104EA000704700207047202070479B081360022045
:104EB000704700BF38B5C36C04460D464BB1586807
:104EC000B0B102685A6000220123C0E90435C26013
:104ED00038BD2122042101F0CBF90346E06400280B
:104EE000EDD1094B094800224FF4A07101F09AF965
:104EF0001C220121204601F0BBF90028F1D001223B
:104F00000223C0E90123DEE7141201085C12010844
:104F10002DE9F04F0E691569AE4285B088461446FA
:104F200005DB2A46234635460C4616469846A368B6
:104F30006168AF19BB42B8BF0131FFF793FE019022
:104F4000002800F08780019B03F1140909EB870A10
:104F5000D14505D24B46002243F8042B9A45FBD895
:104F600008F1140808EB860B04F11403D8451A461F
:104F700003EB85055FD22B1B153B23F003030433A2
:104F80001534A54238BF0423CDE902A7AC461F461D
:104F9000924605E0000C29D1C34509F1040948D91E
:104FA00058F8040B85B2002DF4D056464C46002329
:104FB00056F8040B216882B21FFA81FE05FB02EE4F
:104FC000000C0A0C734405FB002202EB13429BB257
:104FD00043EA0243B44544F8043B4FEA1243E7D89E
:104FE00049F8073058F8040C000CD5D0D9F8003037
:104FF000544619464D4600222688090C00FB06112E
:105000000A449BB243EA024345F8043B54F8046B5C
:105010002968360C8BB200FB063303EB1243A44520
:105020004FEA1342E8D8C34549F8073009F10409AB
:10503000B6D8DDE902A7002F02DC05E0013F03D06E
:105040005AF8043D002BF9D0019B18461F6105B0AA
:10505000BDE8F08F034B0448019A40F25D1101F066
:10506000E1F800BF141201085C12010812F00303FA
:105070002DE9F0411446064632D10D46A41020D049
:10508000D6F84880B8F1000F33D0E3074FF000079F
:1050900007D4641015D0D8F80000A8B18046E30703
:1050A000F7D5424629463046FFF732FFB5B1696869
:1050B000F36C641053F821202A6043F82150054610
:1050C000E9D12846BDE8F081424641463046FFF727
:1050D0001FFFC8F8000007608046E0E70546D8E7F4
:1050E000013B0F4A52F823200023FFF7EBFD054652
:1050F000C4E701213046FFF7B5FD804640B10123EA
:1051000040F27122C0E904320023B0640360BCE7BE
:10511000044B054842464FF4A07101F083F800BFEC
:10512000D0050108141201085C1201082DE9F047AE
:105130000C4690462669A368496806EB6216751C02
:105140009D4207464FEA621904DD5B009D4201F172
:105150000101FADC3846FFF785FD8446002851D06E
:10516000B9F1000F00F114000EDD09F105024FEA5C
:10517000820E03460CEB8202002143F8041B93428B
:10518000FBD1AEF114031844216904F1140318F0A3
:105190001F0803EB81012DD0C8F1200986464FF08E
:1051A000000A1A6802FA08F242EA0A024EF8042BD0
:1051B00053F8042B994222FA09FAF2D80B1B153B3B
:1051C00023F00303043304F11502914238BF042392
:1051D000BAF1000F18BF2E4640F803A0FB6C6268BE
:1051E000CCF8106053F822102160604643F822404A
:1051F000BDE8F087043853F8042B40F8042F994297
:10520000F9D8EBE7034B0448624640F2D91101F0AC
:1052100009F800BF141201085C1201080B698446EA
:105220000069C01A15D10CF1140C14310CEB830277
:1052300010B401EB830301E0944508D252F8044D09
:1052400053F8041D8C42F7D004D24FF0FF3010BC4D
:1052500070477047012010BC704700BF2DE9F84F20
:105260000F691369FF1A002F0E4690467AD101F19B
:105270001405143202EB830205EB830301E09D4227
:1052800073D253F8041D52F8044DA142F7D064D3F1
:105290007168FFF7E7FC8146002872D03569D8F8BD
:1052A0001020C76008F1140E06F1140009F1140A69
:1052B00006F1100C0EEB820200EB8507564600212A
:1052C0005EF8044B5CF804BFA3B211FA8BF1CB1A61
:1052D000210CC1EB1B4101EB23419BB243EA01438B
:1052E000724546F8043B4FEA2141E9D8A2EB080495
:1052F000153C08F11508424524F0030606F10406A2
:1053000038BF0426304424F0030238BF002287420D
:105310005244B24416D95646044654F8043B11FA96
:1053200083F10A1402EB134289B241EA0243A74215
:1053300046F8043B4FEA2241EFD87A1E101A20F0BB
:105340000302524423B952F8043D013D002BFAD028
:10535000C9F810504846BDE8F88F33460127464645
:10536000984695E7F9DB002792E70021FFF77AFCE2
:10537000814668B101220023C9E904234846BDE8FB
:10538000F88F074B07484A464FF4107100F04AFF68
:10539000034B04484A4640F2322100F043FF00BF6D
:1053A000141201085C1201080F4B0B40A3F150735B
:1053B000002B02DD0020194670475B42B3F1A07F4D
:1053C0004FEA235205DA4FF40023002043FA02F19A
:1053D0007047143A1E2ADABF4FF0004323FA02F254
:1053E00001220021104670470000F07F2DE9F843AC
:1053F000066900F1140808EB8606A6F1040956F8C0
:10540000047C3846FFF708FDC0F120030A280B6032
:1054100036DDC8451ED2B0F10B0356F8082C26D055
:10542000C3F1200C22FA0CF19F400F43A6F10801B2
:1054300047F07F55884545F440153AD202FA03F00B
:1054400056F80C3C23FA0CF303431C46204629462D
:10545000BDE8F883B0F10B0308D007FA03F343F07B
:105460007F55002345F440151C46EFE71A4647F0E8
:105470007F5545F44015144620462946BDE8F8837B
:10548000C0F10B0327FA03F2C84542F07F553CBF39
:1054900056F8082CDA4000F1150328BF002207FA5D
:1054A00003F345F4401543EA020420462946BDE8CB
:1054B000F88302FA03F31C46C8E700BF70B5012168
:1054C00082B016461D46FFF7CDFB044600284BD0A0
:1054D0002B46C5F30A55C3F313030DB143F48013F0
:1054E000002E019322D068460096FFF7B5FC0028F5
:1054F00036D0019B0099C0F1200203FA02F20A4360
:10550000C34001936261002B14BF02210121A361FA
:105510002161ADB1069AA5F2334303441360079BA2
:10552000C0F135001860204602B070BD01A8FFF739
:1055300093FC019B0121C4E904132030002DE9D123
:1055400004EB8102A0F232431069069A1360FFF760
:1055500063FC079BC0EB41112046196002B070BD8F
:10556000DDE900236261CEE7034B0448224640F2A6
:105570000A3100F057FE00BF141201085C12010846
:105580002DE9F04383B00F4669468046FFF72EFFB2
:1055900004460D46384601A9FFF728FFD8F8103019
:1055A0003A690F469A1ADDE90013CB1A03EB42134E
:1055B000002B06460BDD05EB03594D4632463B46B4
:1055C0002046294603F07EF903B0BDE8F083C3EB23
:1055D000033307EB03510F46F0E700BF172870B500
:1055E00006460ADD0849094D0020002422462B46C4
:1055F00003F03EF8013EF9D170BD054B03EBC00648
:10560000D6E9040170BD00BF0000F03F0000244057
:10561000D00501080139491101F1010C116902F1AC
:10562000140303EB81018B4200EB8C0C16D210B5F6
:10563000A0F1040E53F8044B4EF8044F9942F9D8E8
:105640008B1A153B23F0030304331844844504D913
:10565000002340F8043B8445FBD810BD844505D9A0
:10566000002340F8043B8445FBD87047704700BFD7
:1056700003694A11934200F1140009DA00EB830335
:1056800002E053F8042DC2B98342FAD800207047D3
:1056900010DD11F01F010DD010B450F8224000EBC6
:1056A000820324FA01F202FA01F18C420BD00120AC
:1056B00010BC704700EB8203E6E70120704753F807
:1056C000042D002AF3D18342F9D8002010BC704782
:1056D0002DE9F04F936883B09146002B6DD0176889
:1056E0008D6880460C460868083743E0A38913F4A8
:1056F000906F2ED0D4E90415A0EB010A05EB450507
:1057000005EBD5750AEB06006D100130A8422A465C
:1057100084BF05462A465B0536D511464046FBF751
:10572000DDFE00283AD0524621690190FCF7D0F9FD
:10573000A289019B22F4906242F08002A281A5EB33
:105740000A0203EB0A006561A2602361206035460E
:10575000B24659465246FCF755FAD9F80830A168C6
:1057600020684D1B50449E1BA5602060C9F808604E
:105770001EB3083757E902B6002EFAD0B542AA4642
:10578000B4D93546B246E4E7404600F029FE034668
:105790000028D4D121694046FFF754F90C23C8F8FA
:1057A0000030A389002243F040034FF0FF30A38173
:1057B000C9E9012203B0BDE8F08F0020C9F8040058
:1057C00003B0BDE8F08F00BF2DE9F04FABB0174636
:1057D00006938B891A068846834603D50B69002BEE
:1057E00000F0A5841AAB0D930023CDE90E33099385
:1057F0000DF1680903935E463B78002B00F036817B
:105800003C4604E014F8013F002B00F05781252BA3
:10581000F8D1E51B40F054812378002B00F026815D
:1058200000214FF0000263788DF82F20671C084696
:105830004FF0FF3B05918A460137A3F12002582A19
:1058400000F25881DFE812F0AB0256015601A702C0
:105850005601560156015601560156019D02990204
:1058600056013601800256017C0259005900590048
:105870005900590059005900590059005601560164
:105880005601560156015601560156015601560160
:105890006202560156015601560156015601560143
:1058A0005601560156012301560156015601560173
:1058B000560168005601560116025601560156015E
:1058C000560156015601560156015601560107026E
:1058D00085015601560156015E02850156015601A9
:1058E000540256013E0225012D02E2015601C1017A
:1058F00056016A0056015601E601A3F13002002468
:1059000017F8013B04EB840402EB4404A3F13002DA
:10591000092AF5D9059490E74AF0100A1AF02001F7
:1059200000F00981069B073323F00703596853F8F9
:10593000080B069301234FF000028DF82F20002260
:105940000792BBF1FF3F00F033822AF080020292FF
:1059500050EA010240F02A82BBF1000F40F00E84B1
:10596000002B40F08A831AF00103049300F0878330
:1059700030238DF867300DF16704049A079B5A4570
:10598000B8BF5A46019213B1134601330193029BEB
:1059900013F00203079302D0019B02330193029B91
:1059A00013F08403089305D1059B019A9D1A002DDD
:1059B00000F3CB82DDE90E219DF82F0080B101328A
:1059C0000DF12F000131C9F80000072A4FF0010046
:1059D000CDE90E21C9F8040000F3F18209F10809AC
:1059E000079B7BB101320CAB0231C9F80030072AAA
:1059F0004FF00203CDE90E21C9F8043000F3EC8228
:105A000009F10809089B802B00F00882049BABEB8E
:105A10000305002D00F34582049BC9F800400132C4
:105A20001944072ACDE90E21C9F8043000F3788221
:105A300009F10809029B5B0705D5059B019A9C1A91
:105A4000002C00F3D682039B059A01988242ACBFDA
:105A50009B181B180393002940F06E8200230E93BD
:105A60003B780DF16809002B7FF4CAAE0F9B002B29
:105A700040F0A083B8F80C3013F0400F039B18BF20
:105A80004FF0FF33039303982BB0BDE8F08F4AF03B
:105A9000100A1AF0200141D0069B073323F00703B8
:105AA000596853F8080B0693002344E7059A5242BD
:105AB000CDE905233B784AF0040ABDE6E51BD5D0C5
:105AC0000F9B2B440F930E9B0133072BC9E90075E5
:105AD0000E9305DC09F10809039B2B4403939BE615
:105AE0000DAA41463046FFF7F3FD0028C2D10DF163
:105AF0006809F1E7002940F06383002BB6D08DF8E8
:105B000040304FF000038DF82F30012301930493B0
:105B100010ACCDF808A04FF0000B38E71AF01003D6
:105B200047D11AF0400144D0069A52F8040B06926D
:105B3000194680B2FFE61AF0100340D11AF0400176
:105B40003DD0069A52F8040B0692194680B2012302
:105B5000F1E6002940F04B831AF0200F069B00F07D
:105B6000DF80073323F007031A465B6852F8080BFF
:105B700006921946002BC0F28E82BBF1FF3F00F067
:105B8000F9829DF82F30079350EA01032AF0800A2A
:105B900000F06D820A2871F1000380F092823030AB
:105BA00001238DF86700CDF808A004930DF1670478
:105BB000E3E6069B53F8040B06930B46BBE6069BF5
:105BC00053F8040B06930123B5E6069D55F8044BE4
:105BD0004FF000038DF82F30002C00F0E282BBF173
:105BE000FF3F00F097825A4600212046FBF720FF36
:105BF000002800F0E882031B04939DF82F300695DF
:105C0000CDF808A007934FF0000BB6E63B784AF0BA
:105C1000200A11E6002940F0ED82A74A09921AF005
:105C200020012FD0069A073222F00702516852F85D
:105C3000080B06921AF0010F0BD050EA010208D0AF
:105C40008DF8313030238DF830304AF0020A0223CB
:105C500071E602236FE6069B4FF000028DF82F20BD
:105C600053F8042B069301238DF8402001930493ED
:105C700010AC4EE7002940F0B182904A09921AF028
:105C80002001CFD11AF0100240F0FB811AF0400140
:105C900000F0F781069C54F8040B0694114680B27C
:105CA000C8E7069B53F8040B069330238DF8303079
:105CB00078238DF83130804B09934AF0020A002195
:105CC000022338E6002940F08C821AF0200F40F0C1
:105CD00017821AF0100F40F038821AF0400F00F0CF
:105CE0003482069B039953F8042B0693118083E5B5
:105CF0003B786C2B03BF7B784AF0200A01374AF0CF
:105D0000100A99E53B784AF0400A95E5002940F0F1
:105D10006B824AF0100A1AF0200F069B7FF421AF25
:105D200053F8040B06931AF0100F40F0AF811AF0ED
:105D3000400F00F0AB8140F3C0310B4600B219E7D1
:105D40003B784AF0800A77E53C4614F8013B2A2B61
:105D500000F05382A3F13002092A27464FF0000BCE
:105D60003FF66BAD17F8013B0BEB8B0B02EB4B0BCC
:105D7000A3F13002092AF5D95FE53B7801212B20F8
:105D80005AE5069B53F8042B0592002AFFF68EAEC7
:105D900006933B7850E53B784AF0010A4CE53B78A6
:105DA00000287FF449AD0121202045E5DDF808A059
:105DB000012B3FF4EFAE022B1AAC12D1099A00F07E
:105DC0000F030009D35C04F8013D40EA01700909A2
:105DD00050EA0103F3D11AAB1B1BCDF808A00493C2
:105DE000CBE500F00703C00840EA4170C908303332
:105DF00050EA0105224604F8013DF2D11AF0010FE4
:105E0000E9D0302BE7D03023023A04F8013C1AAB3A
:105E10009B1ACDF808A004931446AEE5059B0198A3
:105E20001D1A002D7FF7F2AD102DDFF894A025DDAF
:105E300050461023A246044604E0103D102D09F1FF
:105E4000080918DD01321031072AC9E90043CDE9FC
:105E50000E21F2DD0DAA414630460DF16809FFF72B
:105E600037FC00287FF406AE103D102DDDE90E2131
:105E70004FF01003E6DC234654469A46013229448B
:105E8000072ACDE90E21C9F800A0C9F8045000F393
:105E90007B81049BABEB0305002D09F108097FF71B
:105EA000BBAD102DDFF818A02CDD0B4651464FF08E
:105EB000100BA2460C460AE0D0110108E4110108BB
:105EC00008070108103D102D09F1080916DD0132FF
:105ED0001033072AC9E9004BCDE90E23F2DD0DAAE4
:105EE00041463046FFF7F4FB00287FF4C3AD103D78
:105EF000102DDDE90E230DF16809E8DC1946234673
:105F000054469A4601322944072ACDE90E21C9F8A0
:105F100000A0C9F8045000F3C78009F108097BE527
:105F20000DAA41463046FFF7D3FB00287FF4A2AD0F
:105F30000F990DF168097DE50DAA41463046FFF73E
:105F4000C7FB00283FF48AAD94E5102DDDE90E2152
:105F5000DFF8C8A225DD50461023A246044604E01F
:105F6000103D102D09F1080918DD01321031072A02
:105F7000C9E90043CDE90E21F2DD0DAA41463046C4
:105F80000DF16809FFF7A4FB00287FF473AD103D05
:105F9000102DDDE90E214FF01003E6DC23465446B8
:105FA0009A4601322944072ACDE90E21C9F800A0FA
:105FB000C9F8045000F3D18009F10809FCE40DAAE6
:105FC00041463046FFF784FB00287FF453ADDDE9FE
:105FD0000E210DF1680903E50DAA41463046FFF791
:105FE00077FB00287FF446ADDDE90E210DF168094D
:105FF00008E5102C0E9BDFF824A225DD0A46514649
:106000001025B2460E4604E0103C102C09F1080998
:1060100016DD01331032072BC9E90065CDE90E32D8
:10602000F2DD0DAA41465046FFF752FB00287FF4EF
:1060300021AD103C102CDDE90E320DF16809E8DCD1
:10604000114632465646924601332144072BC9E990
:1060500000A4CDE90E317FF7F6AC0DAA41463046DB
:10606000FFF736FB00287FF405AD0F99EBE4BBF199
:10607000000F7FF494ADCDF808A0CDF810B01AACA5
:106080007BE4069A52F8040B0692D3E5C1170B463F
:10609000002BBFF672AD2D2340428DF82F300793B1
:1060A00061EB410101234CE40DAA41463046FFF764
:1060B0000FFB00287FF4DEACDDE90E210DF168094D
:1060C000AAE41AACCDF804A00A22002382460D46A9
:1060D000FAF7BAF8303204F8012D00235046294669
:1060E0000A22FAF7B1F8BAF10A0F75F10003EBD200
:1060F0001AABDDF804A0CDF808A01B1B04933CE408
:10610000069B039853F8041B0693C217C1E90002CB
:10611000FFF772BB20460695CDF808A0FCF770F992
:106120009DF82F30049007934FF0000B25E4402199
:10613000FBF7D4F9C8F80000C8F81000002866D0B2
:106140004023C8F81430FFF74DBB069B039953F862
:10615000042B11600693FFF74FBB0DAA4146304652
:10616000FFF7B6FA00287FF485ACDDE90E210DF1CA
:10617000680921E49DF82F3007930BE5012BDDF82A
:1061800008A07FF418AE0AE50DAA41463046FFF795
:106190009FFA00287FF46EACDDE90E210DF168094D
:1061A00034E45B46062B28BF06231D4C049306955A
:1061B0000193AEE40DAA41463046FFF789FA59E44F
:1061C0008DF82F0099E49DF82F30CDF810B006958A
:1061D000CDF808A083460793FFF7CFBB8DF82F00BB
:1061E0004BE58DF82F0070E58DF82F0091E58DF8C7
:1061F0002F00B1E48DF82F000FE5069A7B78274633
:1062000052F8044B069244EAE47BFFF715BB0C23DB
:10621000CBF800304FF0FF33039334E4F806010865
:10622000F811010800B50B4C25681446EE681A46B3
:1062300085B003460D464CB107490095CDE90114E0
:106240003046064900F052F8FBF7EAF804490C46DC
:10625000F3E700BF0000002090120108A01201081F
:10626000F00F010808B513460022FFF7DBFF00BF5F
:1062700010B502FB01F1FBF731F9044668B150F8A3
:10628000042C22F00302043A242A18D8132A06D830
:1062900002460023C2E900339360204610BD00236C
:1062A0001B2AC0E900330FD9242AC0E9023311BFE9
:1062B00000F11002036100F118024361E9E70021D7
:1062C000FBF71CFD204610BD00F10802E1E700BF0E
:1062D0000CB400B583B004AB53F8042B019300F069
:1062E000B1FA03B05DF804EB02B070470EB410B51C
:1062F00083B005AB064C53F8042B0193014620688C
:1063000000F0A0FA03B0BDE8104003B0704700BF32
:106310000000002042B110B50B4910461446FBF7AF
:10632000F3FE18B9094810BD0848704707492046D0
:10633000FBF7EAFE0028F5D005492046FBF7E4FE0E
:106340000028EFD0002010BDD4120108D01201089F
:10635000F00F0108014B93F8280170474008002016
:1063600041B110B50C4620460A49FBF7CDFE18B9DD
:10637000094810BD0848704707492046FBF7C4FE8E
:106380000028F5D005492046FBF7BEFE0028EFD0D7
:10639000002010BDD4120108D0120108F00F01082E
:1063A00010B4034CD4F8E440A44610BC604700BFCE
:1063B0004008002082B049B15AB16BB113780B602C
:1063C0001278101E18BF012002B0704701A9002AE0
:1063D000F3D1104602B070476FF00100F4E700BF40
:1063E0002DE9F84F1746002900F0988007F10B05BA
:1063F00080460C46FBF7D4FC162D5DD810252A46A6
:10640000AF425ED854F8041C21F003069642A4F172
:10641000080962DABC4BD3F808C009EB06008445D2
:1064200000F09780D0F804C02CF0010303445B68AF
:10643000DB0768D42CF0030C06EB0C03934247DA1D
:10644000CB0710D454F8083CA9EB030ADAF804305F
:1064500023F003018C44B444944580F211817318F5
:10646000934280F2E88039464046FBF737F807460A
:10647000E0B154F8043C23F001034B44A0F10802BE
:10648000934200F0D280321F242A00F2F580132AB2
:1064900000F2AC80034622461168196051685960C9
:1064A00092689A6021464046FEF7CCFA4046FBF7D8
:1064B00079FC3846BDE8F88F25F00705002D2A46FF
:1064C0009EDA0C23C8F8003000273846BDE8F88F64
:1064D0001E46D0E90223D3609A60731B0F2B22D88B
:1064E000D9F8043003F0010333434E44C9F80430B3
:1064F000736843F00103736040462746FBF752FC84
:106500003846BDE8F88FC907ADD454F8083CA9EB6C
:10651000030ADAF8041021F00301A0E7BDE8F84F00
:106520001146FAF7DBBFD9F8041001F00101294345
:10653000C9F8041009EB05014E4443F001034B6018
:10654000736843F00103083173604046FEF77AFA3E
:10655000D2E7DCF8040020F0030B06EB0B0C05F18E
:10656000100084454DDAC9073FF57DAF54F8081C8B
:10657000A9EB010ADAF8041021F003018B44B344BB
:1065800058453FF76CAF5746DAF80C1057F8080F2C
:10659000321F242AC160886000F2DB80132A40F297
:1065A000D6802168CAF808106168CAF80C101B2A46
:1065B00000F2DF8008340AF110022168116061687E
:1065C0005160A16891600AEB0501ABEB050242F056
:1065D000010299604A60DAF8043003F001031D43B8
:1065E0004046CAF80450FBF7DDFB6EE72368036002
:1065F000636843601B2A68D804F1080200F10803AD
:106600004AE709EB05029A60ACEB050343F001038E
:10661000536054F8043C03F001031D43404644F822
:10662000045CFBF7BFFB27464FE750F8043C23F020
:1066300003031E4451E75746DAF80C1057F8080FC9
:10664000321F242AC16088604CD8132A48D9216897
:10665000CAF808106168CAF80C101B2A56D808340A
:106660000AF110021E462368136063685360A36832
:106670009360D1463C4630E72146FBF7C3FA11E769
:10668000D0E902135746CB60996057F8081FDAF833
:106690000C30CB60321F242A99602DD8132A29D9B7
:1066A0002368CAF808306368CAF80C301B2A42D83D
:1066B00008340AF1100322681A6062685A60A268FE
:1066C0009A606646D1463C4607E7A3688360E36864
:1066D000C360242A26D004F1100200F11003DBE687
:1066E0003A46BFE7214638461E46D146FBF78AFAAE
:1066F0003C46F2E63B46DEE7214638466646D14652
:10670000FBF780FA3C46E8E630040020A168CAF8AE
:106710001010E168CAF81410242A20D010340AF1AD
:1067200018029FE7236903616169416104F118025E
:1067300000F11803B0E6A368CAF81030E368CAF89D
:106740001430242A21D010340AF11803B3E73A4652
:1067500033E721463846FBF755FA164B33E72269F3
:10676000CAF818206269CAF81C2018340AF12002FD
:1067700078E7A168CAF81010E168CAF81410242A52
:106780000DD010340AF1180217E72369CAF818303F
:106790006369CAF81C3018340AF120038BE72269B8
:1067A000CAF818206269CAF81C2018340AF12002BD
:1067B00003E700BF300400202DE9F84F4B6E9C0426
:1067C00090462DD59368126843B38B46064602F176
:1067D000080959E9025A5FEA9A0715D0043D0024D6
:1067E00001E0A7420ED055F8041F5A46304601F08A
:1067F00033F9431C04F10104F3D10023C8E9013348
:10680000BDE8F88FD8F808302AF0030AA3EB0A0392
:10681000C8F8083009F10809002BDAD10020ECE7AC
:1068200001F04CF90023C8E90133BDE8F88F00BF3F
:1068300010B494680CB110BCBEE72046546010BC84
:10684000704700BF2DE9F04FABB01C468846174695
:106850000693834618B1836B002B00F02582B8F9AC
:106860000C1088048AB20AD4D8F8643041F400527B
:1068700023F40053A8F80C20C8F8643092B2130730
:1068800040F1A480D8F81030002B00F09F8002F077
:106890001A020A2A00F0A8801AAB0D930023CDE952
:1068A0000E3309930DF1680905933B78002B00F036
:1068B0000D813C4604E014F8013F002B00F0E88015
:1068C000252BF8D1E51B40F0E5802378002B00F064
:1068D000FD804FF0000200218DF82F206378049195
:1068E0004FF0FF32671C084602928A460137A3F137
:1068F0002002582A00F2F780DFE812F03302F50098
:10690000F5002F02F500F500F500F500F500F500A3
:10691000E5012B02F500F001F401F5002702590012
:10692000590059005900590059005900590059009F
:10693000F500F500F500F500F500F500F500F500AF
:10694000F500F5000E02F500F500F500F500F50084
:10695000F500F500F500F500F5009400F500F500F0
:10696000F500F500F5008400F500F5004802F5009B
:10697000F500F500F500F500F500F500F500F5006F
:10698000F5003A02A701F500F500F5008902A7011C
:10699000F500F5007F02F50069029600C902C50204
:1069A000F500A402F5008600F500F5008D02A3F1C4
:1069B0003002002417F8013B04EB840402EB44048A
:1069C000A3F13002092AF5D9049490E741465846CC
:1069D00000F0AAFD002840F03985B8F80C2002F03C
:1069E0001A020A2A7FF458AFB8F90E30002BFFF6CE
:1069F00053AF23463A46414658462BB0BDE8F04FC8
:106A000000F044BD4AF0100A1AF0200100F00F8196
:106A1000069B073323F00703596853F8080B0693C6
:106A200001230EE04AF0100A1AF0200100F0F28073
:106A3000069B073323F00703596853F8080B0693A6
:106A400000234FF000028DF82F2000220792029AB7
:106A5000541C00F02F822AF08004019450EA0104B3
:106A600040F02682002A40F09584002B40F00E84EE
:106A70001AF00103039340F03E841AACDDE902638F
:106A80009E42B8BF1E46079B002B3ED001363CE01D
:106A9000E51B1BD00E9B0F9A01332A44072BC9E933
:106AA00000750F920E9305DC09F10809059B2B4434
:106AB00005930AE7002A00F0D1830DAA4146584603
:106AC000FFF77AFE30B90DF16809EFE70F9B002B55
:106AD00040F08584B8F80C305B0600F1B784059867
:106AE0002BB0BDE8F08F002940F07584002BEDD06D
:106AF0008DF8403001264FF000038DF82F300396BB
:106B000010AC0023CDF804A00293019B13F0020304
:106B10000793019B18BF023613F08403089304D136
:106B2000049B9D1B002D00F3DB82DDE90E1001F1BB
:106B3000010C9DF82F3093B101300DF12F0301218D
:106B4000BCF1070FCDE90EC0C9F80030C9F8041038
:106B500000F3A682614609F108090CF1010C079BBC
:106B6000EBB10CAB0230C9F80030BCF1070F4FF0AD
:106B70000203CDE90EC0C9F8043040F3AB8200280F
:106B800000F066830DAA41465846FFF715FE00281F
:106B9000A0D1DDE90E100DF1680901F1010C089B8F
:106BA000802B00F0C881DDE902329D1A002D00F330
:106BB0001C82039BC9F800401844BCF1070FCDE9C3
:106BC0000EC0C9F8043040F3B381002800F0D2822F
:106BD0000DAA41465846FFF7EFFD00287FF47AAF33
:106BE0000F980DF16809019B5A0704D5049B9C1B63
:106BF000002C00F3C982DDE90423B242ACBF9B182C
:106C00009B190593002840F0368200230E930DF166
:106C100068094AE61AF0100349D11AF0400146D03B
:106C2000069A52F8040B0692194680B209E71AF048
:106C3000100342D11AF040013FD0069A52F8040BDB
:106C40000692194680B20123FBE6002940F0E58355
:106C50001AF0200F069B68D0073323F007031A466B
:106C60005B6852F8080B06921946002BC0F20483A9
:106C7000029B013300F08A839DF82F30079350EA7E
:106C800001032AF0800A00F054830A2871F10003FE
:106C900080F01283303001238DF86700CDF804A016
:106CA00003930DF16704E9E600F062FED7E5069B69
:106CB00053F8040B06930B46C3E6069B53F8040BEC
:106CC00006930123BDE6069B53F8042B0492002A89
:106CD00080F20D83049A0693524204923B784AF064
:106CE000040A03E63C4614F8013B2A2B00F0B38368
:106CF000A3F13002092A274698BF002400F29383AB
:106D000017F8013B04EB840402EB4404A3F13002C6
:106D1000092AF5D90294EAE5002940F088834AF06F
:106D2000100A1AF0200F069B96D153F8040B069315
:106D30001AF0100F40F09B821AF0400F00F097827B
:106D400040F3C0310B4600B28FE73B784AF0800A2F
:106D5000CCE53B7801212B20C8E53B784AF0010ABD
:106D6000C4E53B7800287FF4C1AD01212020BDE5BA
:106D7000069B4FF000028DF82F20012653F8042BBC
:106D80008DF840200693039610ACBAE6002940F037
:106D90005183BD4A09921AF0200144D0069A073265
:106DA00022F00702516852F8080B06921AF0010F00
:106DB0000BD050EA010208D08DF8313030238DF825
:106DC00030304AF0020A02233BE6022339E600296A
:106DD00040F026831AF0200F40F09A821AF0100F2C
:106DE00040F0CC821AF0400F00F0C882069B059953
:106DF00053F8042B0693118057E53B786C2B03BFA7
:106E00007B784AF0200A01374AF0100A6EE53B7899
:106E10004AF0400A6AE5002940F0FC829B4A099248
:106E20001AF02001BAD11AF0100240F01B821AF0B9
:106E3000400100F01782069C54F8040B069411469A
:106E400080B2B3E7069D55F8044B4FF000038DF870
:106E50002F30002C00F0A482029B5E1C00F0728296
:106E60001A4600212046FAF7E3FD002800F0C2820E
:106E7000031B03939DF82F30079300230695CDF84D
:106E800004A00293FAE53B784AF0200A2EE5069B1F
:106E900053F8040B069330238DF8303078238DF8A7
:106EA00031307A4B09934AF0020A00210223C8E5E7
:106EB000DDF804A0012B3FF4E8AE022B1AAC12D18E
:106EC000099A00F00F030009D35C04F8013D40EA81
:106ED0000170090950EA0103F3D11AAB1B1BCDF86D
:106EE00004A00393CAE500F00703C00840EA41701C
:106EF000C908303350EA0105224604F8013DF2D1B9
:106F00001AF0010FE9D0302BE7D03023023A04F811
:106F1000013C1AAB9B1ACDF804A003931446ADE5CF
:106F200003981A9401231B900F900E930DF168099A
:106F300009F1080957E6049B9D1B002D7FF733AE2E
:106F4000102D40F37F82DFF848A152461023A2465D
:106F5000144607E001F1020E09F108091146103D3F
:106F6000102D1DDD4A1C1030072AC9E90043CDE968
:106F70000E20EFDD0DAA002800F08C804146584617
:106F80000DF16809FFF718FC00287FF4A3ADDDE9D7
:106F90000E10103D102D01F1010E4FF01003E1DC39
:106FA000234654469A462844BEF1070FCDE90EE029
:106FB000C9F800A0C9F8045040F3A481002800F0EB
:106FC000F8810DAA41465846FFF7F6FB00287FF4EA
:106FD00081ADDDE90232DDE90E109D1A002D01F1CF
:106FE000010C0DF168097FF7E4AD102DDFF8A0A0CA
:106FF0002BDD52461023A246144607E001F1020C95
:1070000009F108091146103D102D1BDD4A1C1030F6
:10701000072AC9E90043CDE90E20EFDD0DAA41465C
:1070200018B358460DF16809FFF7C6FB00287FF436
:1070300051ADDDE90E10103D102D01F1010C4FF0A6
:107040001003E3DC234654469A462844BCF1070F5C
:10705000CDE90EC0C9F800A0C9F8045000F3E380E0
:1070600009F108090CF1010CA3E54FF0010C0146F0
:107070000DF16809C7E70DAA41465846FFF79CFB8A
:1070800000283FF4C2AD25E5E4110108D011010844
:10709000280701084FF0010E01460DF168095EE76F
:1070A000002800F0D2800DAA41465846FFF784FB25
:1070B00000287FF40FADDDE90E100DF1680901F134
:1070C000010C4CE502200CAB1B901A934FF0010C05
:1070D0000DF16809614609F1080901F1010C5EE54D
:1070E000102D40F39181DFF804A3DDE90EC0524674
:1070F0001023A2466146144607E001F1020C09F193
:1071000008091146103D102D1BDD4A1C1030072ABE
:10711000C9E90043CDE90E20EFDD0DAA20B34146B9
:1071200058460DF16809FFF747FB00287FF4D2AC01
:10713000DDE90E10103D102D01F1010C4FF0100390
:10714000E3DC2346614654469A4628440729CDE9A4
:107150000E10C9F800A0C9F8045000F39C8009F192
:10716000080901F1010CE4E401464FF0010C0DF1B6
:107170006809C7E7019B0E9059074CD5049B9C1BDF
:10718000002C48DD0DF16809102C40F35681DFF822
:107190005CA20E9A53461025B2461E4606E0911C8C
:1071A00009F108091A46103C102C19DD531C103047
:1071B000072BC9E90065CDE90E30F0DD0DAA28B333
:1071C00041465846FFF7F8FA00287FF483ACDDE922
:1071D0000E20103C102C02F101010DF16809E5DCD4
:1071E000334656469A4620440729C9E900A4CDE90A
:1071F0000E107FF700AD70B10DAA41465846FFF75B
:10720000DBFA00287FF466AC0F98F4E40121024613
:107210000DF16809C7E7DDE90423B242ACBF9B1852
:107220009B190593F1E400283FF47AAE0DAA41467C
:107230005846FFF7C1FA00287FF44CAC0E9B0F981C
:1072400003F1010C0DF16809B3E4079B002B69D130
:107250004FF0010C01460DF16809A0E40E920DF10A
:10726000680923E4069A52F8040B06929EE5C117BA
:107270000B46002BBFF6FCAC2D2340428DF82F307F
:10728000079361EB41010123FFF7E1BB029B0393ED
:107290001AACFFF7F3BB002862D00DAA414658464E
:1072A000FFF78AFA00287FF415ACDDE90E100DF126
:1072B000680901F1010C3CE41AAC0A2200230646DD
:1072C0000D46F8F7C1FF303204F8012D0023304697
:1072D00029460A22F8F7B8FF0A2E75F10003ECD20E
:1072E0001AAB1B1BCDF804A00393FFF7C7BB069393
:1072F0003B78FFF7FBBA30238DF867300DF1670458
:10730000FFF7BCBB09F108090EF1010C71464AE414
:10731000DDE9050353F8041B0693C217C1E9000217
:10732000FFF7C3BA02200CAB1B901A930DF168094A
:10733000D1E6029B002B7FF4ADACCDF804A0039303
:10734000FFF79BBB20460695CDF804A0FBF758F845
:107350009DF82F300793002303900293FFF78EBB15
:107360009DF82F3063B301239C461B930DF12F032F
:107370001A930DF168096046FFF7ECBB069B05996F
:1073800053F8042B11600693FFF78FBA9DF82F3046
:1073900007937AE4012BDDF804A07FF48EAD79E445
:1073A000029E134C0695062E28BF06260396FFF76D
:1073B000A8BB4FF0010C01460DF16809FFF7F3BBC4
:1073C000079B002B7FF47EAE01464FF0010C0DF1C0
:1073D0006809FFF7E8BB8DF82F00FFF787BB0DAA00
:1073E00041465846FFF7E8F9FFF774BB1807010854
:1073F000F8110108029B03939DF82F300695CDE903
:1074000001A00793FFF73ABB0E990F98DFF85CA035
:1074100001319AE68DF82F0000E58DF82F0017E472
:107420008DF82F00D6E400220292FFF760BA8DF8A3
:107430002F0074E48DF82F00ABE40E99DFF82CA038
:107440000131D0E6DFF828A0E646ACE54FF0FF3387
:107450000593FFF744BB069A7B78274652F8044B06
:10746000069244EAE4740294FFF740BA1807010850
:107470002807010810B4044C84461346206810BC49
:107480000A466146FFF7DEB90000002070B50C46E1
:107490008989ADF58D6D21F00201ADF80C10616E9A
:1074A0001991E189ADF80E10E1690791616A0991BE
:1074B0001AA9009104914FF4806102910591002175
:1074C000069169460646FFF7BDF9051E07DB6946CA
:1074D000304600F023F9002818BF4FF0FF35BDF803
:1074E0000C305B0603D5A38943F04003A3812846F3
:1074F0000DF58D6D70BD00BF10B4034CD4F8E040A5
:10750000A44610BC604700BF4008002049B1FF2AD4
:1075100002D80A70012070478A2303604FF0FF30C1
:1075200070470846704700BF38B5334B1B680546A7
:107530000C460BB19A6B12B3B4F90C3018079AB21F
:1075400025D5216900292DD012F0010007D0002097
:10755000A06060694042A06139B1002038BD950744
:1075600058BF6069A0600029F7D1120658BF0846CD
:10757000F4D543F04003A3814FF0FF3038BD1846E7
:1075800000F0F6F9B4F90C3018079AB2D9D4D10644
:107590002AD5520714D4216943F00803A3819AB273
:1075A0000029D1D102F42070B0F5007FCCD0214663
:1075B000284600F03BFCB4F90C3021699AB2C3E7CD
:1075C000216B51B104F14002914204D02846FDF7ED
:1075D00039FAB4F90C300022226321690022C4E98F
:1075E000001223F02403D7E7092243F040032A6066
:1075F0004FF0FF30A38138BD00000020B1F90C200E
:10760000F8B50C461107074642D4636842F400629D
:10761000002BA28159DDA56A002D54D000233E68BD
:107620003B6093B212F4805253D1E1690123384692
:10763000A847421C63D0A389A56A5B0705D5636888
:10764000C01A236B0BB1E36BC01AE1690246002339
:107650003846A847411C3ED13B68002B3BD01D2B30
:1076600001D0162B52D1A3892269226023F4006332
:1076700000216160A381216B3E6021B304F14003CE
:10768000994202D03846FDF7DDF900202063F8BDAD
:107690002669C6B193B2256826609A070CBF636954
:1076A0000023AD1BA3600CE0D4F824C0E1692B4695
:1076B00032463846E047B0F1000CA5EB0C056644B5
:1076C00016DD002DF0DC0020F8BDE36B002BA2DC02
:1076D000F9E7206DB1E7B4F90C302269226023F498
:1076E0000063A3810022DB046260C4D52065C2E789
:1076F000A38943F040034FF0FF30A381F8BD3B68FE
:10770000002B98D01D2B06D0162B04D0A38943F054
:107710004003A381F8BD3E60D5E700BF38B50D46F4
:10772000044608B1836B1BB1B5F90C0030B938BD04
:1077300000F01EF9B5F90C000028F8D029462046C3
:10774000BDE83840FFF75ABF38B5B8B10F4B1D68D8
:1077500004460DB1AB6B4BB1B4F90C0000B938BDA8
:1077600021462846BDE83840FFF748BF284600F0CC
:10777000FFF8B4F90C000028F1D0F1E7044B0549FB
:107780001868BDE8384000F02DBB00BF00000020A5
:10779000A80401081D77000800207047014900F087
:1077A00021BB00BFE1810008002070472DE9F84FA0
:1077B0002D4A4668C26300240323C0E9B843074644
:1077C00000F53B720423C0F8E8222146C6E90243D3
:1077D0000822C6E90044C6E904447466B46106F1AF
:1077E0005C00FAF78BFADFF884B0BD68DFF880A0A0
:1077F000DFF88090DFF88080204BC6F824A0C6E92F
:10780000076BC6F82890C6F82C800822EB60C5E903
:107810000044C5E904446C66AC60AC61214605F1E6
:107820005C00FAF76BFAC5E9075BC5E909A9C5F879
:107830002C80FD68124BEB60C5E90044C5E90444A7
:107840006C66AC60AC612146082205F15C00FAF779
:1078500055FA0123C5E9075BC5E90A98C5F824A0D4
:10786000BB63BDE8F88F00BF9D7700086D7F0008FF
:10787000957F0008D57F0008F57F0008090001000A
:107880001200020070B568224D1E02FB05F50E467F
:1078900005F17401F9F722FE044640B100210C30D5
:1078A000C4E90016A06005F16802FAF727FA20463D
:1078B00070BD00BF274B2DE9F0411E68B36B074632
:1078C0005BB306F538764FF00408D6E90134013B86
:1078D00004D51EE05A1C04F168041AD0B4F90C5007
:1078E000013B002DF6D11C4B6566C4E90055C4E987
:1078F0000253C4E90455A5610822294604F15C003D
:10790000FAF7FCF9C4E90C55C4E911552046BDE865
:10791000F08135682DB12E46D7E73046FFF746FF98
:10792000CFE74FF4D6713846F9F7D8FD044668B171
:107930000560C0F804800C302946A06025464FF44D
:10794000D072FAF7DBF934602E46BEE70C233060C4
:107950003B60DBE7A80401080100FFFF024B03497D
:10796000186800F03FBA00BFA8040108E1810008D0
:10797000836B03B1704719E7704700BF704700BFC2
:10798000704700BF704700BF024B0349186800F002
:1079900009BA00BF0000002099770008024B034994
:1079A000186800F0FFB900BF00000020A9770008A8
:1079B0002DE9F04383B0074688461446FEF7CAFC1B
:1079C000012803D108F1FF33FE2B37D9424604F1D9
:1079D0005C0301A9384600F075FB421C064633D013
:1079E00038B39DF804C00DF10509002509E02368AE
:1079F0005A1C226083F800C00135B54219D219F82B
:107A000001CBA368013B002BA360F0DAD4F818E0A7
:107A1000734561462246384602DBBCF10A0FE6D1C7
:107A200000F0ECFA431CE7D10646304603B0BDE84F
:107A3000F0834646304603B0BDE8F0835FFA88FC29
:107A40008DF804C00646CEE7A389304643F04003D4
:107A5000A38103B0BDE8F083B2F90C3013F4005FEA
:107A60000AD110B4546E43F4005344F400545466E5
:107A7000938110BCFFF79CBFFFF79ABF0E4B70B508
:107A80001E6805460C460EB1B36B8BB1B4F90C30D1
:107A90009A0406D4626E43F4005342F40052A38168
:107AA0006266224629463046BDE87040FFF780BF37
:107AB0003046FFF75DFFE9E7000000209368002BE8
:107AC00000F081802DE9F04FB1F90C300C46190718
:107AD000804683B0174698B223D523690BB310F0C4
:107AE00002033D682BD04FF0000ADFF8B4B25646CF
:107AF0005E453346524628BF5B464046002E4FD077
:107B0000E169D4F824C0E047002852DDBB681B1AA5
:107B10008244361ABB60002BEAD1002003B0BDE8D6
:107B2000F08F21464046FFF7FFFC002840F03481EB
:107B3000B4F90C303D6898B210F00203D3D110F0C4
:107B4000010942D14E463EB38205D4F808B040F157
:107B50008180B3455A4600F2B18010F4906F40F036
:107B6000BE80206801924946FAF74CF8A368216864
:107B7000019AA3EB0B030A44B246A36022600026DD
:107B8000B868A0EB0A00D144B8600028C5D0B4F9A9
:107B90000C0080B2002ED7D1D5E900960835D2E787
:107BA000D5E900A60835A3E721464046FFF7B6FD14
:107BB00080B3B4F90C3043F040034FF0FF30A381A1
:107BC00003B0BDE8F08F002070471E46AA469946D4
:107BD00018461D4656B388B34A46D4E904132068B4
:107BE000B24228BF3246884205D9A16803EB010B97
:107BF0005A4500F3A780934264DCE169D4F824C0BD
:107C00002A464046E047B0F1000BD2DDB9EB0B0944
:107C1000CAD00120BB68A3EB0B035D44A6EB0B06A7
:107C2000BB60002B3FF479AF002ED4D10AF10803DA
:107C300053E902569A460833002EF9D032460A21FB
:107C40002846F9F7F5FE002800F09D800130A0EBF2
:107C50000509C1E720682369984217D86369B342D0
:107C600014D86FF00042B24228BF3246E16992FB5D
:107C7000F3F2D4F824C002FB03F340464A46E0473F
:107C8000B0F1000A95DDA6EB0A0679E7B345DA46BE
:107C900028BFB24652464946F9F7B4FFA3682268A6
:107CA000A3EB0A035244A3602260002BEBD12146D0
:107CB0004046FFF733FD0028E5D07AE72068B34659
:107CC00032464FE729460192F9F79CFF019AA368D3
:107CD0009B1AA360236813442360934696E72368A6
:107CE0002169A3EB010B636903EB430A0AEBDA7A20
:107CF0000BF101034FEA6A0A33445345524684BFED
:107D00009A46524643052CD511464046F9F7E6FB04
:107D100000283BD05A4621690190F9F7D9FEA28983
:107D2000019B22F4906242F08002A28103EB0B00DF
:107D30002361AAEB0B03C4F814A0A3602060B34630
:107D400032460FE729465A46F9F75CFF23685B4441
:107D5000236021464046FFF7E1FC00283FF456AF80
:107D600027E74046FEF73CFB03460028DED12169A9
:107D70004046FCF767FEB4F90C300C2223F0800378
:107D8000C8F8002017E7721C914626E70C22B4F9C8
:107D90000C30C8F800200EE74FF0FF30BEE600BF01
:107DA00000FCFF7F2DE9F041884600F5387700267A
:107DB000D7E90154013D0FD4A389012B05F1FF350B
:107DC00006D9B4F90E300133204601D0C04706432E
:107DD0006B1C04F16804EFD13F68002FE8D13046F6
:107DE000BDE8F0812DE9F8430746884600F538766E
:107DF0004FF00009D6E90154013D11D4A389012BAC
:107E000005F1FF3508D9B4F90E300133214603D00E
:107E10003846C04749EA00096B1C04F16804EDD1FB
:107E20003668002EE6D14846BDE8F8832DE9F041DA
:107E30008B890C46990796B008D504F143030122BB
:107E4000C4E90432236016B0BDE8F081B4F90E1025
:107E50000029064627DB6A4600F0FAF9002821DBF4
:107E6000019D05F47045A5F50055B5FA85F54FF46B
:107E700080686D094FF4006741463046F9F72EFBE4
:107E8000B4F90C30F0B1204AF26343F08003C4F837
:107E90001480A3812060206135BB3B43A38116B0D1
:107EA000BDE8F081A38913F0800519D04FF0400898
:107EB00041463046F9F712FB0025B4F90C302F4645
:107EC0000028E0D19A05BED423F0030304F1430255
:107ED00043F002030121C4E90421A3812260B2E737
:107EE0004FF480682F46C7E7B4F90E10304600F013
:107EF000C5F910B9B4F90C30CFE7A38923F0030317
:107F000043F001031BB2C8E79D77000870B50C462B
:107F1000B1F90E10002996B015461E4614DB6A46CC
:107F200000F096F900280FDB019A02F47042A2F5E6
:107F30000052B2FA82F24FF4806352094FF40060AB
:107F400032602B6016B070BDB4F90C10002311F034
:107F50008000336004D0402218462A6016B070BDFD
:107F60004FF480632B6016B070BD00BF10B50C4697
:107F7000B1F90E1000F0AAF9002803DB236D0344C9
:107F8000236510BDA38923F48053A38110BD00BFD6
:107F9000002070472DE9F0410C46B1F90C101F4646
:107FA000CB05054616460BD421F48051A1813B46F2
:107FB000B4F90E1032462846BDE8F04100F0C8B8CA
:107FC000B4F90E100223002200F06AF9B4F90C1083
:107FD000EAE700BF10B50C46B1F90E1000F060F9E9
:107FE000A389421C0EBF23F4805343F480532065C1
:107FF000A38110BDB1F90E10FBF7D0BCF8B50D464A
:108000001446064610B1836B002B43D0B4F90C2004
:10801000A369A360170790B21BD52369CBB1EDB25A
:1080200081042F4622D522686169D31A994229DD3D
:108030000133A1680139A160511C2160157062698A
:108040009A422AD0A389DB0701D50A2D25D03846CC
:10805000F8BD21463046FFF767FA20BBB4F90C2083
:10806000236990B2EDB281042F46DCD442F4005271
:10807000A281626E616922F4005262662268D31A9C
:108080009942D5DC21463046FFF748FB58B92268B3
:108090000123CEE7FFF76CFCB8E721463046FFF737
:1080A0003DFB0028D3D04FF0FF37D0E710B4044C8D
:1080B00003460A46206810BC1946FFF79FBF00BF61
:1080C0000000002070B5054684B01C4639B10B4E47
:1080D000D6F8E060B047431C09D004B070BD0A4632
:1080E0000649D1F8E06001A9B047431CF5D1002250
:1080F0008A2322602B6004B070BD00BF40080020BE
:1081000070B5114B84B01D6814460B46014650B142
:108110000E481A46D0F8E06023462846B047431C74
:108120000BD004B070BD094A2346D2F8E06001A923
:1081300002462846B047431CF3D100228A2322601E
:108140002B6004B070BD00BF00000020400800207C
:1081500038B50C46084D8446114620461A46002381
:108160002B60644602F02CFA431C00D038BD2B680B
:10817000002BFBD0236038BD140A002070B50C46DC
:108180000646FFF73BFAE36A054633B1E16930463C
:1081900098470028B8BF4FF0FF35A3891B0619D4B4
:1081A000216B41B104F14003994202D03046FCF703
:1081B00049FC00232363616C21B13046FCF742FC8B
:1081C00000236364FFF7D8FB0023A381FFF7D6FBEE
:1081D000284670BD21693046FCF734FCE0E700BF5B
:1081E000B1B138B505460C4608B1836B4BB1B4F953
:1081F0000C300BB9002038BD21462846BDE8384078
:10820000BCE7FFF7B5FBB4F90C30002BF2D0F3E775
:1082100000207047C0B138B50C4B1D6804460DB145
:10822000AB6B4BB1B4F90C300BB9002038BD214613
:108230002846BDE83840A1E72846FFF799FBB4F986
:108240000C30002BF1D0F2E7002070470000002036
:1082500070B50C46084D03460026204611461C46C4
:108260002E6002F0BEF9431C00D070BD2B68002BBD
:10827000FBD0236070BD00BF140A002038B5074D45
:108280000022044608462A6002F0B0F9431C00D0E0
:1082900038BD2B68002BFBD0236038BD140A0020AA
:1082A00038B50C46084D8446114620461A46002330
:1082B0002B60644602F09CF9431C00D038BD2B684B
:1082C000002BFBD0236038BD140A002038B50C46C3
:1082D000084D8446114620461A4600232B6064460A
:1082E00002F060F9431C00D038BD2B68002BFBD096
:1082F000236038BD140A002081F0004102E000BF75
:1083000083F0004330B54FEA41044FEA430594EA55
:10831000050F08BF90EA020F1FBF54EA000C55EA90
:10832000020C7FEA645C7FEA655C00F0E2804FEA61
:108330005454D4EB5555B8BF6D420CDD2C4480EA43
:10834000020281EA030382EA000083EA010180EA73
:10835000020281EA0303362D88BF30BD11F0004FC1
:108360004FEA01314FF4801C4CEA113102D04042F7
:1083700061EB410113F0004F4FEA03334CEA133332
:1083800002D0524263EB430394EA050F00F0A7804A
:10839000A4F10104D5F1200E0DDB02FA0EFC22FA45
:1083A00005F2801841F1000103FA0EF2801843FA39
:1083B00005F359410EE0A5F120050EF1200E012A2A
:1083C00003FA0EFC28BF4CF0020C43FA05F3C01868
:1083D00051EBE37101F0004507D54FF0000EDCF1E1
:1083E000000C7EEB00006EEB0101B1F5801F1BD38A
:1083F000B1F5001F0CD349085FEA30004FEA3C0C8E
:1084000004F101044FEA445212F5800F80F09A8083
:10841000BCF1004F08BF5FEA500C50F1000041EB87
:10842000045141EA050130BD5FEA4C0C404141EB8B
:108430000101013C28BFB1F5801FE9D291F0000F86
:1084400004BF01460020B1FA81F308BF2033A3F135
:108450000B03B3F120020CDA0C3208DD02F1140C2C
:10846000C2F10C0201FA0CF021FA02F10CE002F167
:108470001402D8BFC2F1200C01FA02F120FA0CFC60
:10848000DCBF41EA0C019040E41AA2BF01EB0451A9
:10849000294330BD6FEA04041F3C1CDA0C340EDCA7
:1084A00004F11404C4F1200220FA04F001FA02F3EA
:1084B00040EA030021FA04F345EA030130BDC4F1A8
:1084C0000C04C4F1200220FA02F001FA04F340EA9D
:1084D0000300294630BD21FA04F0294630BD94F04E
:1084E000000F83F4801306BF81F480110134013D35
:1084F0004EE77FEA645C18BF7FEA655C29D094EAA6
:10850000050F08BF90EA020F05D054EA000C04BF23
:108510001946104630BD91EA030F1EBF002100200E
:1085200030BD5FEA545C05D14000494128BF41F0AD
:10853000004130BD14F580043CBF01F5801130BD11
:1085400001F0004545F0FE4141F470014FF000009C
:1085500030BD7FEA645C1ABF194610467FEA655C4D
:108560001CBF0B46024650EA013406BF52EA0335EF
:1085700091EA030F41F4002130BD00BF90F0000FDD
:1085800004BF0021704730B54FF4806404F1320419
:108590004FF000054FF0000150E700BF90F0000FD2
:1085A00004BF0021704730B54FF4806404F13204F9
:1085B00010F0004548BF40424FF000013EE700BFC9
:1085C00042004FEAE2014FEA31014FEA02701FBF59
:1085D00012F07F4393F07F4F81F06051704732F08B
:1085E0007F4208BF704793F07F4F04BF41F40021E2
:1085F000704730B54FF4607401F0004521F0004140
:108600001CE700BF50EA010208BF704730B54FF0C9
:1086100000050AE050EA010208BF704730B511F0CA
:10862000004502D5404261EB41014FF4806404F102
:1086300032045FEA915C3FF4D8AE4FF003025FEA88
:10864000DC0C18BF03325FEADC0C18BF033202EB0C
:10865000DC02C2F1200300FA03FC20FA02F001FA66
:1086600003FE40EA0E0021FA02F11444BDE600BF09
:1086700070B54FF0FF0C4CF4E06C1CEA11541DBFB8
:108680001CEA135594EA0C0F95EA0C0F00F0DEF883
:108690002C4481EA030621EA4C5123EA4C5350EA68
:1086A000013518BF52EA033541F4801143F48013B9
:1086B00038D0A0FB02CE4FF00005E1FB02E506F04A
:1086C0000042E0FB03E54FF00006E1FB03569CF09F
:1086D000000F18BF4EF0010EA4F1FF04B6F5007FA5
:1086E00064F5407404D25FEA4E0E6D4146EB060617
:1086F00042EAC62141EA55514FEAC52040EA5E50A0
:108700004FEACE2EB4F1FD0C88BFBCF5E06F1ED849
:10871000BEF1004F08BF5FEA500E50F1000041EB80
:10872000045170BD06F0004646EA010140EA02002D
:1087300081EA0301B4EB5C04C2BFD4EB0C0541EA4F
:10874000045170BD41F480114FF0000E013C00F364
:10875000AB8014F1360FDEBF002001F0004170BD88
:10876000C4F10004203C35DA0C341BDC04F11404A1
:10877000C4F1200500FA05F320FA04F001FA05F22D
:1087800040EA020001F0004221F0004110EBD370FA
:1087900021FA04F642EB06015EEA430E08BF20EA26
:1087A000D37070BDC4F10C04C4F1200500FA04F3C9
:1087B00020FA05F001FA04F240EA020001F000415B
:1087C00010EBD37041F100015EEA430E08BF20EACE
:1087D000D37070BDC4F1200500FA05F24EEA020E16
:1087E00020FA04F301FA05F243EA020321FA04F045
:1087F00001F0004121FA04F220EA020000EBD370FC
:108800005EEA430E08BF20EAD37070BD94F0000FFB
:108810000FD101F00046400041EB010111F4801F2F
:1088200008BF013CF7D041EA060195F0000F18BFE0
:10883000704703F00046520043EB030313F4801F1C
:1088400008BF013DF7D043EA0603704794EA0C0FD6
:108850000CEA135518BF95EA0C0F0CD050EA4106EC
:1088600018BF52EA4306D1D181EA030101F0004169
:108870004FF0000070BD50EA410606BF1046194691
:1088800052EA430619D094EA0C0F02D150EA01369D
:1088900013D195EA0C0F05D152EA03361CBF1046DE
:1088A00019460AD181EA030101F0004141F0FE417D
:1088B00041F470014FF0000070BD41F0FE4141F401
:1088C000780170BD70B54FF0FF0C4CF4E06C1CEA01
:1088D00011541DBF1CEA135594EA0C0F95EA0C0FB6
:1088E00000F0A7F8A4EB050481EA030E52EA033571
:1088F0004FEA013100F088804FEA03334FF0805592
:1089000045EA131343EA12634FEA022245EA1115BE
:1089100045EA10654FEA00260EF000419D4208BF6F
:10892000964244F1FD0404F5407402D25B084FEA1C
:108930003202B61A65EB03055B084FEA32024FF4C8
:1089400080104FF4002CB6EB020E75EB030E22BF25
:10895000B61A754640EA0C005B084FEA3202B6EBE5
:10896000020E75EB030E22BFB61A754640EA5C0094
:108970005B084FEA3202B6EB020E75EB030E22BF24
:10898000B61A754640EA9C005B084FEA3202B6EB25
:10899000020E75EB030E22BFB61A754640EADC00E4
:1089A00055EA060E18D04FEA051545EA16754FEA46
:1089B00006164FEAC30343EA52734FEAC2025FEA64
:1089C0001C1CC0D111F4801F0BD141EA00014FF0F3
:1089D00000004FF0004CB6E711F4801F04BF0143C4
:1089E0000020B4F1FD0C88BFBCF5E06F3FF6AFAEE0
:1089F000B5EB030C04BFB6EB020C5FEA500C50F170
:108A0000000041EB045170BD0EF0004E4EEA1131F2
:108A100014EB5C04C2BFD4EB0C0541EA045170BDF9
:108A200041F480114FF0000E013C90E645EA060E3D
:108A30008DE60CEA135594EA0C0F08BF95EA0C0F6B
:108A40003FF43BAF94EA0C0F0AD150EA01347FF4B3
:108A500034AF95EA0C0F7FF425AF104619462CE78A
:108A600095EA0C0F06D152EA03353FF4FDAE1046ED
:108A7000194622E750EA410618BF52EA43067FF43E
:108A8000C5AE50EA41047FF40DAF52EA43057FF4CE
:108A9000EBAE12E74FF0FF3C06E000BF4FF0010CD9
:108AA00002E000BF4FF0010C4DF804CD4FEA410C3D
:108AB0007FEA6C5C4FEA430C18BF7FEA6C5C1BD00A
:108AC00001B050EA410C0CBF52EA430C91EA030F8B
:108AD00002BF90EA020F0020704710F1000F91EAE8
:108AE000030F58BF994208BF90422CBFD8176FEAB6
:108AF000E37040F0010070474FEA410C7FEA6C5C84
:108B000002D150EA013C07D14FEA430C7FEA6C5C8A
:108B1000D6D152EA033CD3D05DF8040B704700BFB6
:108B20008446104662468C461946634600E000BF04
:108B300001B5FFF7B7FF002848BF10F1000F01BDD6
:108B40004DF808EDFFF7F4FF0CBF012000205DF8A1
:108B500008FB00BF4DF808EDFFF7EAFF34BF012026
:108B600000205DF808FB00BF4DF808EDFFF7E0FFBF
:108B700094BF012000205DF808FB00BF4DF808ED10
:108B8000FFF7CEFF94BF012000205DF808FB00BF77
:108B90004DF808EDFFF7C4FF34BF012000205DF859
:108BA00008FB00BF4FEA410C7FEA6C5C02D150EA3F
:108BB000013C0AD14FEA430C7FEA6C5C02D152EAD5
:108BC000033C02D14FF0000070474FF001007047A6
:108BD0004FEA410212F5001215D211D56FF47873E5
:108BE000B3EB625212D94FEAC12343F0004343EA88
:108BF000505311F0004F23FA02F018BF4042704763
:108C00004FF00000704750EA013005D111F00040EC
:108C100008BF6FF0004070474FF00000704700BF82
:108C2000F8B5214B984236D1204D21482C88214F50
:108C3000214E202102F014FA640024B2012808BF5A
:108C400044F001043C432C8019483488102102F080
:108C500007FA64002B8824B2012808BF44F00104FD
:108C60003C43B3F5704F34800DD1002310482B8066
:108C7000082102F0F5F9114B1A8801280CBF0132C6
:108C800002F1FF321A803388B3F5704F02D10C4BDA
:108C900001221A70F8BD0B4B984201BF0A4A138893
:108CA00001331380F6E700BF580B0020200A002094
:108CB0000000024000E0FFFF180A00201E0A00200A
:108CC0001C0A0020A00B00201A0A00202DE9F04108
:108CD00014228AB00DEB02000021F9F70FF80024EE
:108CE000424B01941A6BDFF80881424F424D42F02B
:108CF00004021A631A6B02F004020192019A0294B0
:108D00001A6B42F080021A631A6B02F08002029220
:108D1000029A03941A6B42F001021A631A6B02F072
:108D200001020392039A04941A6B42F002021A633E
:108D30001B6B03F002030493224640464FF400519C
:108D4000049B02F093F92246384648F2070102F0EC
:108D50008DF9384601224FF4B86102F087F92846B0
:108D60000122182102F082F9224628464FF4505180
:108D700002F07CF901264FF4005305A94046CDE9E5
:108D80000536CDE9074402F0A3F848F2C75305A918
:108D90003846CDE90536CDE9074402F099F8382385
:108DA00005A93846CDE90534079602F091F8042369
:108DB00005A92846CDE90534079402F089F843F265
:108DC000184305A92846CDE90536CDE9074402F048
:108DD0007FF84CF22003CDE9053405A9022328468B
:108DE000079302F075F80AB0BDE8F0810038024040
:108DF00000080240000002400004024000F10803A5
:108E000073B5044603600D46D9B10846F9F7F8FA80
:108E10000F2805EB0006019007D9002201A9204682
:108E200006F028FE019B2060A36032462946206898
:108E300006F07EFE019B226863600021D15402B0DF
:108E400070BD014806F00AFD3807010800F108036B
:108E500073B50360D1E900530446EE181DB916B18D
:108E60000C4806F0FBFC0F2B019307D9002201A947
:108E7000204606F0FFFD019B2060A3603246294694
:108E8000206806F04BFE019B226863600021D154EC
:108E900002B070BD3807010810B50E4C2378BFF33F
:108EA0005B8FDB0713D4204606F0BCFB78B10A4B7E
:108EB0000A4A0B4940F21450C3E900124FF4807281
:108EC000C3E902023C221A82204606F0CBFB02488C
:108ED00010BD00BF240A0020280A00200000FFFF68
:108EE0000000060870B58CB083880093C388019396
:108EF000037A0293437A0393837A0493C37A0593A4
:108F0000037B0693437B0793837B0893C37B09937F
:108F1000038A0A934FF2F00304680B9301F022FFD7
:108F20000021072001F0AEFF6D4604F1300655F830
:108F3000042B00232146022001F05EFF38B90434DF
:108F4000B442F4D10CB0BDE8704001F01DBF0CB0CC
:108F5000BDE8704001F022BF10B503688CB06A46CE
:108F600003F1300153F8044B42F8044B9942F9D114
:108F70000B9A4FF2F0039A4223D1009B8380019B0E
:108F8000C380029B0372039B4372049B003B18BF88
:108F900001238372059B003B18BF0123C372069B0C
:108FA000003B18BF01230373079B003B18BF01233D
:108FB0004373089B8373099BC3730A9B03820CB0A2
:108FC00010BD0023838042F21073C38040F2195316
:108FD0000381012343814FF48073838140F2235343
:108FE000C38105230382FFF77DFFE8E730B587B033
:108FF00004460D4668461146FFF728FF20460C4BF5
:1090000040F8083B6946FFF721FF04E0684606F098
:1090100055FD05F09FFD002384F82030684665600B
:1090200006F04CFD034B2360204607B030BD00BF67
:10903000B40A01086C0D010830B587B004460D462E
:1090400068461146FFF702FF20460C4B40F8083BEC
:109050006946FFF7FBFE04E0684606F02FFD05F0C9
:1090600079FD002384F820306846656006F026FD0F
:10907000034B2360204607B030BD00BFB40A01088F
:10908000000D010830B587B004460D46684611460C
:10909000FFF7DCFE20460C4B40F8083B6946FFF723
:1090A000D5FE04E0684606F009FD05F053FD0023F7
:1090B00084F820306846656006F000FD034B2360AD
:1090C000204607B030BD00BFD80A0108240D0108B2
:1090D00030B587B004460D4668461146FFF7B6FE28
:1090E00020460C4B40F8083B6946FFF7AFFE04E012
:1090F000684606F0E3FC05F02DFD002384F82030DF
:109100006846656006F0DAFC034B2360204607B032
:1091100030BD00BFFC0A0108480D010870B50446C7
:109120000E46817A1046154605F0D4FB304605F010
:109130007AFB237A984207DA0121284605F09AFB48
:10914000094B01221A7070BD304605F06CFB237A82
:10915000627A13449842F6DD0021284605F08AFB26
:10916000014B0022EEE700BFAD0900202DE9F047DA
:1091700004461E46237B884610468BB304F047FB0B
:1091800080F00105EDB2E37A002B6BD0384FDFF8A9
:10919000E49001F0C5FA228A3B684EF6602A0AFB89
:1091A0000233834248D24FF0000A4046C9F800A07B
:1091B00005F039FBA37B984229DA2F4CDFF8BC90ED
:1091C000DFF8BC8085B90021304605F053FB012350
:1091D000237089F80030002388F80030BDE8F0875C
:1091E00004F015FB0546CEE70121304605F042FBB1
:1091F000002389F80030012388F80030237813B168
:1092000001F08EFA38601C4B00221A70E6E74046E7
:1092100005F009FBA37BE27B13449842DEDD0121CC
:10922000304605F027FB154B83F800A0144B83F85C
:1092300000A0114B1B78E2E71248802101F01BFFD0
:109240000121304605F016FB238A3C680AFB0344E3
:1092500001F066FA241A4FF47A70B4FBF0F4C9F8FE
:109260000040BBE730460121BDE8F04705F002BBF6
:10927000500A0020400A00204C0A0020440A002026
:10928000AC0900200000024037B5044608460D46F0
:10929000F9F7B6F8294682B24FF4FA73204603F084
:1092A000F9FA0A238DF804300122642301A920462B
:1092B00003F0F0FA03B030BD08B572B6FFF706FD53
:1092C00002480022082101F0D1FEFEE7000402401E
:1092D00010B594B01422002109A8F8F70FFD14224C
:1092E000002103A8F8F70AFD00231C4A0193116C22
:1092F00041F080511164126C02F080520192019A87
:10930000174A0293116841F4404111601268022427
:1093100002F44042CDE90E430292C0200823CDE979
:1093200011030121029A08941022042308A8CDE910
:109330000B121092139302F051FD014608B1FFF792
:10934000BBFFCDE905000F23079003A8CDE9033447
:1093500002F022FF0028F2D114B010BD0038024004
:10936000007000402DE9F84FD0E9008992466FF077
:109370006043A9EB0802B3EBA20F06460F464FEA83
:10938000A20402D1224806F081FA012C224638BFFD
:109390000122A418A1EB080B1FD204B39C4228BFE2
:1093A0001C46A00006F080F90546DAF8003045F8C2
:1093B0000B300023CAF800302A464346BB4210D186
:1093C0003B1DA3EB08032B4439461A4649450DD0F3
:1093D00051F8040B42F8040BF8E71C46E1E7254678
:1093E000E3E753F8041B42F8041BE7E7CF1B1F44D5
:1093F000B8F1000F05D0B1684046A1EB080105F0B7
:10940000A7FB05EB8404C6E90057B460BDE8F88FFC
:109410006207010810B50446006810B103685B6874
:109420009847204610BD10B50446006810B1036887
:109430005B689847204610BD70B5D0E900560446D9
:10944000AE4204D02846FFF7EEFF0435F8E7206867
:1094500018B1A168091A05F07BFB204670BD10B554
:1094600004461C3006F02AFB04F10C0000F012F850
:109470002046FFF7E1FF204610BD38B505680446D9
:1094800035B12846FFF7EBFF3421284605F060FB95
:10949000204638BD70B5D0E900560446AE4204D02F
:1094A0002846FFF7EAFF0435F8E7206818B1A168FD
:1094B000091A05F04DFB204670BDF7B5054634206E
:1094C0000C4606F0F1F82368E268036063684360C5
:1094D000C260A3682269E169836002610023626956
:1094E0002360C4E90133C4E904334261E36004F159
:1094F0002402A3698361914200F12403C36121D155
:10950000114604F1340651F8047B43F8047BB14260
:10951000F9D1236A0362002384F82430E261D5E99B
:10952000041291422362019010D041F8040B019380
:1095300029612B6953F8043C01A89D61FFF79DFF49
:1095400003B0F0BD636AC1614362E2E701AA05F1BD
:109550000C00FFF707FFECE701A8FFF78EFF05F00F
:10956000F9FA002310B5C0E90033C0E90233C0E9BD
:109570000433044683611C30FFF768FC08E004F103
:109580000C00FFF787FF2046FFF756FF05F0E2FAD1
:10959000204610BD10B50446006810B103685B6832
:1095A0009847204610BD10B50446006810B1036806
:1095B0005B689847204610BD10B50446006810B19E
:1095C00003685B689847204610BD00002DE9F84FFE
:1095D000D0E9008992466FF06043A9EB0802B3EB33
:1095E000A20F06460F464FEAA20402D1224806F017
:1095F0004DF9012C224638BF0122A418A1EB080B1B
:109600001FD204B39C4228BF1C46A00006F04CF8B1
:109610000546DAF8003045F80B300023CAF8003070
:109620002A464346BB4210D13B1DA3EB08032B4403
:1096300039461A4649450DD051F8040B42F8040B3F
:10964000F8E71C46E1E72546E3E753F8041B42F838
:10965000041BE7E7CF1B1F44B8F1000F05D0B1682A
:109660004046A1EB080105F073FA05EB8404C6E956
:109670000057B460BDE8F88F6207010810B50A46CC
:10968000D0E90114A142034606D0106841F8040B4A
:1096900000201060596010BDFFF798FFFBE770B520
:1096A00088B005460E4602A81146FFF7A7FB242006
:1096B00005F0FAFF02AA31460446FFF797FC02A81C
:1096C000019406F0FBF9019B002202A92846CDE98E
:1096D0000123FFF7D3FF09E02421204605F038FAE3
:1096E00002A806F0EBF905F035FAF9E702A8FFF752
:1096F0009AFE01A8FFF760FF08B070BD02A8FFF74F
:1097000092FE01A8FFF758FFEDE770B588B0054657
:109710000E4602A81146FFF771FB242005F0C4FF96
:1097200002AA31460446FFF7D3FC02A8019406F0D2
:10973000C5F9019B002202A92846CDE90123FFF7C4
:109740009DFF09E02421204605F002FA02A806F058
:10975000B5F905F0FFF9F9E702A8FFF764FE01A8E3
:10976000FFF721FF08B070BD02A8FFF75CFE01A85B
:10977000FFF719FFEDE700002DE9F04FADF5497D4A
:1097800000F0A8FFB94CFFF7A3FDFFF79FFA1022E6
:10979000002164A8F8F7B2FA17234FF0804EC4E90D
:1097A00000E36322002380272046C4E902322361BC
:1097B000A76102F0D9FE08B1FFF77EFD4FF4805695
:1097C00064A92046649602F005FF05460028F3D1FF
:1097D000204602F0A3FD1022294649A8F8F78EFA88
:1097E000A34CDFF890C2A56045F6C053C4E900C39E
:1097F00020464EF27863C4E90335A76102F0B4FE57
:109800000028D9D149A92046499602F0E3FE054631
:109810000028D1D1204602F081FD102229463CA823
:10982000F8F76CFA944C954BA5600126C4E9003515
:109830002046934B2561257684F82050E562A3628B
:10984000E560E66184F83050666100F083FF00282F
:10985000B2D108233CA92046CDE93C363E9601F022
:10986000EBF80028A8D1874C874B884D2062C4E9CB
:1098700000534FF48043C4E90430C4E90200C4E952
:109880000600204601F0D4FC0346002894D180480D
:10989000804903614FF41652C0E900120C22C0E95E
:1098A0000233C0E90523C36102F0C6FF002883D15B
:1098B0001C2001F0AFF94E21204604F02FF9044698
:1098C0001C2001F099F9FFF7E7FAFFF745FB4CADD3
:1098D000714B4A937149499441F288332846ADF857
:1098E0002C31FFF78BFA0DE00324C4F10304182098
:1098F00000FB0454AC4200F00285183C204606F000
:10990000DDF8F7E7664952A8FFF778FA01E002248C
:10991000EBE7644958A8FFF771FA63495EA8FFF7BF
:109920006DFA01E00024E0E70022114649A803F0A7
:10993000C9FF01E00124D8E75C4964A8FFF75EFA9B
:1099400064A922A8FFF70DFE64A806F0B7F800236B
:1099500057498DF8193064A8FFF750FA242005F014
:10996000A3FE64AA06A90546FFF766FB64A83C951A
:1099700006F0A4F83C9B6493002264A922A83C92C0
:10998000FFF77CFE08E02421284605F0E1F8FFE718
:1099900064A806F093F810E064A8FFF744FD3CA823
:1099A000FFF738FD434964A8FFF728FA0AE064A8E6
:1099B000FFF739FD3CA8FFF72DFD22A8FFF74FFD6B
:1099C00000F094BC242005F06FFE64AA0DF119018B
:1099D0000546FFF731FB64A83C9506F06FF83C9B09
:1099E0006493002264A922A83C92FFF747FE01E09D
:1099F000C9E7CDE764A8FFF716FD3CA8FFF70AFD0D
:109A0000FFF74AFA2C49061D64A8FFF7F7F900E0B2
:109A1000CDE7242005F048FE64AA31460546FFF74D
:109A200031FB64A83C9506F049F83C9B6493002206
:109A300064A922A83C92FFF721FE01E0A3E7A7E773
:109A400064A8FFF7F0FC3CA8FFF7A4FDFFF724FA99
:109A50001A49861D64A8FFF7D1F931E064A8FFF721
:109A6000E2FC3CA8FFF796FDA7E700BF580B0020DB
:109A7000A00B002000040040BC0A00200020014090
:109A80000100000F040B0020A086010000540040DC
:109A9000E80B002000100140640032008408010837
:109AA0008707010898070108AD070108C1070108E9
:109AB000C6070108D6070108E5070108ED070108F8
:109AC000242005F0F1FD64AA31460546FFF7DAFAD5
:109AD00064A83C9505F0F2FF3C9B6493002264A9C6
:109AE00022A83C92FFF7CAFD01E04CE750E764A8CA
:109AF000FFF799FC3CA8FFF74DFDFFF7CDF9B14901
:109B000000F1080664A8FFF779F900E0A6E7242031
:109B100005F0CAFD64AA31460546FFF7D9FA64A8E4
:109B20003C9505F0CBFF3C9B6493002264A922A8DE
:109B30003C92FFF7A3FD01E025E729E764A8FFF7C2
:109B400072FC3CA8FFF72FFDFFF7A6F99E4A00F133
:109B5000090122A8FFF7D9FD06E064A8FFF763FC1E
:109B60003CA8FFF720FD28E7FFF796F9974900F199
:109B70000A0664A8FFF742F9242005F095FD64AABF
:109B800031460546FFF732FA64A83C9505F096FF8A
:109B90003C9B6493002264A922A83C92FFF76EFDCF
:109BA00001E0F0E6F4E664A8FFF73DFC3CA8FFF70F
:109BB00003FD874964A8FFF721F906E064A8FFF7D1
:109BC00032FC3CA8FFF7F8FCF7E664A92FA8FFF7E2
:109BD000C8FC64A805F072FFFFF75EF97D4A00F14A
:109BE0000B012FA8FFF75BFDFFF756F97A4A00F14A
:109BF0000D012FA8FFF753FDFFF74EF9774A00F14B
:109C00000C012FA8FFF74BFDFFF746F9744A00F14E
:109C10000E012FA8FFF779FDFFF73EF96A4A00F120
:109C20000F012FA8FFF771FDFFF736F96D4900F11D
:109C3000100664A8FFF7E2F8242005F035FD64AAB9
:109C400031460546FFF71EFA64A83C9505F036FF3D
:109C50003C9B6493002264A92FA83C92FFF70EFD61
:109C600008E02421284604F073FF64A805F026FFCD
:109C700011E0FAE764A8FFF7D6FB3CA8FFF78AFCDF
:109C8000594964A8FFF7BAF809E064A8FFF7CBFBCD
:109C90003CA8FFF77FFC2FA8FFF7E1FB8DE664A946
:109CA0003CA8FFF75EFC64A805F008FF22A93CA8C9
:109CB000FFF703FC2FA93CA8FFF7FFFB322300931B
:109CC0004A4A4B494FF480631AA804F085FDFFF718
:109CD000E3F80546FFF7E0F8291D821D1AA804F0F5
:109CE000B5FD42490023202207A803F07CFD012591
:109CF000404900952B462A460CA804F0D9FD3D4961
:109D000000950023022210A804F0D2FD0CA804F054
:109D1000E3FD10A804F0E0FD002337498DF81A3068
:109D200064A88DF81B30FFF769F8242005F0BCFC0F
:109D300064AA0DF11A010546FFF77EF964A83CAE4E
:109D4000149505F0BBFE149B6493002264A9304671
:109D50001492FFF793FC08E02421284604F0F8FE53
:109D6000FFE764A805F0AAFE10E064A8FFF75BFB1C
:109D700014A8FFF74FFB214964A8FFF73FF809E05B
:109D800064A8FFF750FB14A8FFF744FB3CA8FFF7BB
:109D900066FB80E7242005F087FC64AA0DF11B0117
:109DA0000546FFF749F964A8149505F087FE149B52
:109DB0006493002264A930461492FFF75FFC1FE011
:109DC000CAE7CEE7F4070108020801080C080108F9
:109DD0001708010824080108310801083E08010895
:109DE0004B080108550801085F08010800040240FB
:109DF000BC0A00200000024069080108730801083D
:109E000064A8FFF710FB14A8FFF704FB0023CDE9BB
:109E10000A36B64D09942B78BFF35B8FDB070AD463
:109E2000284605F0FFFB30B1B14B1A88B14B2846EC
:109E30001A8005F017FCB049B048FFF725FA00E09A
:109E40009EE7AF49AD48FFF71FFAAE4FDFF8B88283
:109E5000002600F065FC3B6803F57A73834280F0CE
:109E6000A08000F05DFC386098F80010204603F0F8
:109E700014FE00221146204603F034FE1AA804F016
:109E8000D2FCA249024614A8F8F718F914A92046F2
:109E900003F0EDFD01220021204603F023FE9C4B40
:109EA0001B78B3B19B4964A8FEF7A8FF64992046CC
:109EB00003F0DDFD64A805F001FE012296484FF491
:109EC000806101F0D3F802220021204603F00AFE4F
:109ED0000CE0924964A8FEF791FF6499204603F0D4
:109EE000C6FD64A805F0EAFD0022E7E78C4B1B786D
:109EF000B3B18C4964A8FEF781FF6499204603F052
:109F0000B6FD64A805F0DAFD002283484FF48071A5
:109F100001F0ACF803220021204603F0E3FD0CE041
:109F2000814964A8FEF76AFF6499204603F09FFD0B
:109F300064A805F0C3FD0122E7E77C4B1A687AB1FB
:109F40003B2A8ABF7A497B493C2314A888BFB2FBCD
:109F5000F3F2F8F7B3F814A9204603F088FD20E0E7
:109F6000754B1B7883B1754964A8FEF747FF649968
:109F7000204603F07CFD64A805F0A0FD00226648A1
:109F8000802101F073F80CE06D4964A8FEF736FFFC
:109F90006499204603F06BFD64A805F08FFD012253
:109FA000EDE7DFF8A091DFF8A0A1B9F80020DAF81A
:109FB00000309A4204DD002109A804F016FB02E0FB
:109FC00008DA0121F8E7B9F80030CAF8003000F0EB
:109FD000A7FB064600F0A4FB06F56A436033834204
:109FE000DFF868B134BF0023012388F800309BF804
:109FF000003073B900F094FB554D2B6803F59C536A
:10A0000008338342C0F0C9804FF47A7000F08EFBB1
:10A010002EE10121204603F040FD00238BF80030A3
:10A0200000F07EFB054601210CA804F023FC012171
:10A0300010A804F01FFC0CA804F04EFC10A804F0BB
:10A040004BFC09A804F090FB9BF800304BB10023B7
:10A05000022109A88BF8003004F0C7FA00F060FB79
:10A060000546B9F80020DAF800309A4204DD0021F4
:10A0700009A804F0BAFA02E008DA0121F8E7B9F811
:10A080000030CAF8003000F04BFB05460A2000F013
:10A090004DFB9DF8183083B109A804F065FB1AA8A0
:10A0A00004F0C4FB00238DF818309DF81A30002B03
:10A0B00050D009A804F058FB0DE09DF81930002B92
:10A0C000F3D009A804F050FB1AA804F0B7FB002352
:10A0D0008DF81930E9E7FEF7DFFEFEF703FF0023F6
:10A0E0008DF81A3000F01CFB47E000BF480A002042
:10A0F0001A0A00205A0A002079080108E80B0020FB
:10A1000099080108600A00203C0A0020AB080108F9
:10A11000AD090020C008010800000240D508010870
:10A12000440A0020EA080108FF080108400A00204C
:10A130001409010829090108AC0900203E09010899
:10A14000530901081E0A00205C0A00201C0A002096
:10A15000540A00209DF81B30002BC3D009A804F03E
:10A1600003FBFEF799FEFEF7F7FE4FF4967000F042
:10A17000DDFA00238DF81B30B4E705F51C531033CE
:10A180008342BFF450AF204603F07EFC0CA804F0DD
:10A19000A3FB10A804F0A0FB2CE700F0C1FA286094
:10A1A00000225F48402100F061FF1AA804F0DFFAA6
:10A1B00007A803F01FFBFEF76FFE0CAA1AA9FEF713
:10A1C000ADFFFEF769FE10AB07AA1AA9FEF7CEFF96
:10A1D000DFF85091544AB9F800301188994241D2C1
:10A1E0003C2513801AA8B3FBF5F205FB12339DB290
:10A1F00004F019FBDFF834A10AF805001AA8B9F831
:10A2000000503C23B5FBF3F504F00DFB4849B9F8C9
:10A21000003048553C205D1CB3FBF0F200FB123CC3
:10A22000B5FBF0FE1FFA8CFC00FB1E551AF80CC0A3
:10A230001AF80550ACEB0505DFF8F8C08CF80050B3
:10A240001825B2FBF5FC05FB1C22034492B2B3FBBC
:10A25000F0F3B3FBF5F005FB10338A5CCB5CD31A4B
:10A26000354A13702E480122402100F0FFFECBE654
:10A2700000F056FA314D2B6803F56A436033834290
:10A28000BFF4E7AD00F04CFA28601AA804F0CBFA4E
:10A290002B4B2C491D782C4B02462C48007800286B
:10A2A00014BF8C469C462A480078002814BF8E466E
:10A2B0009E46214890F9000004901E4890F9000045
:10A2C000039024480068CDF800C0CDE901E0002DDE
:10A2D00008BF0B4664A82049F7F7F0FE1F4864A9A1
:10A2E000FEF7D2FFB5E564A805F0E8FB00245EABFD
:10A2F0001819183C05F0E2FB14F1600FF7D104F0D7
:10A3000029FCFFF745BBB0E42BE52AE529E528E564
:10A3100027E526E53AE5BEE4FFF74FBBE6E700BFD9
:10A32000000002401A0A00205A0A00207F0A00207A
:10A33000680A0020590A0020580A0020640A0020F8
:10A34000AD090020820701087C070108440A0020AB
:10A35000AC090020400A002068090108E80B002031
:10A3600082B00C4B002100915A6C42F480425A6436
:10A370005A6C02F480420092009A01911A6C42F0E9
:10A3800080521A641B6C03F080530193019B02B04E
:10A39000704700BF0038024010B5044688B0142250
:10A3A000002103A8F7F7AAFC2268114B9A421DD19D
:10A3B00003F58C33002101915A6C0E4842F48072EF
:10A3C0005A645A6C02F480720192019A02911A6BDB
:10A3D00042F002021A631B6B03F002030293029B1A
:10A3E00003A90323CDE9033300F072FD08B010BDCB
:10A3F000002001400004024030B5044689B0142218
:10A40000002103A8F7F77AFC2268144B9A4222D164
:10A41000134C144800250195236B43F0020323637A
:10A42000236B03F002030193019B4FF4407212234C
:10A43000CDE9032303210423CDE9061303A900F08A
:10A4400047FD0295236C43F400132364236C03F44B
:10A4500000130293029B09B030BD00BF00540040BE
:10A4600000380240000402400368B3F1804F13B586
:10A4700029D1002403F50E3300941A6C42F0010236
:10A480001A641A6C02F001020092009A01941A6C8C
:10A4900042F002021A641B6C03F0020322462146BA
:10A4A00001931C20019B00F075FB1C2000F0A4FB15
:10A4B000224621461D2000F06DFB1D2002B0BDE8A4
:10A4C000104000F099BB02B010BD000010B504466A
:10A4D00088B01422002103A8F7F710FC2268144B5F
:10A4E0009A4222D103F59433002101915A6C11480C
:10A4F00042F010025A645A6C02F010020192019A62
:10A5000002911A6B42F002021A631B6B03F0020302
:10A510000293029BC02202230321CDE903230723D8
:10A52000CDE9061303A900F0D3FC08B010BD00BFAD
:10A530000010014000040240FEE7000008B5034C93
:10A5400000228021204600F091FDF9E70000024042
:10A55000FEE7FEE7FEE770477047704700F0D4B8AB
:10A56000014801F011BF00BF580B0020014801F065
:10A570000BBF00BFA00B0020014801F0E7B800BFEF
:10A58000BC0C00200120704708B5F6F757FF1623D2
:10A5900003604FF0FF3008BD08B5F6F74FFF1623F4
:10A5A0000360FEE770B50D4614460E46731B9C42D1
:10A5B00001DC204670BDAFF3008006F8010BF5E723
:10A5C00070B50D4614460E46731B9C4201DC2046B6
:10A5D00070BD16F8010BAFF30080F5E74FF0FF30C8
:10A5E00070474FF400534B600020704701207047C4
:10A5F000002070470B4A116810B5034609B90A4993
:10A600001160106809490A4C0344091B8B4206D9A2
:10A61000F6F714FF0C2303604FF0FF3010BD1360FA
:10A62000FCE700BF2C0C0020F811002000000220E5
:10A630000004000070470000DFF834D00D480E49D8
:10A640000E4A002302E0D458C4500433C4188C428C
:10A65000F9D30B4A0B4C002301E013600432A242F1
:10A66000FBD3FFF7E7FFF6F705FFFFF785F8704725
:10A670000000022000000020C4090020981C0108EE
:10A68000C4090020F8110020FEE7000038B50E4A8A
:10A690000E4B054618784FF47A73B3FBF0F310684D
:10A6A000B0FBF3F000F0CAFA044658B90F2D09D8F0
:10A6B000024629464FF0FF3000F06CFA044B20466A
:10A6C0001D6038BD0120FCE7B0090020B40900205E
:10A6D000B809002008B50B4B1A6842F400721A60E2
:10A6E0001A6842F480621A601A6842F480721A6032
:10A6F000032000F03DFA0F20FFF7C8FFFFF730FE00
:10A70000002008BD003C0240034A044B11681B783E
:10A710000B441360704700BF300C0020B4090020C8
:10A72000014B1868704700BF300C002038B5044654
:10A73000FFF7F6FF631C1CBF054B1B78054618BFCF
:10A74000E418FFF7EDFF431BA342FAD338BD00BF67
:10A75000B409002038B50446002800F09B80056C41
:10A7600025B9FFF719FE656484F83C50236CDB06BD
:10A7700000F18E80236C23F4885323F0020343F00E
:10A7800002032364444B5A6822F440325A605A68E8
:10A7900061680A435A60236821695A6822F480720A
:10A7A0005A605A6842EA01225A605A68A16822F047
:10A7B00040725A605A680A435A609A68E16822F403
:10A7C00000629A609A680A439A603449A26A8A428F
:10A7D00052D0996821F07061996099680A439A6033
:10A7E0009A68E16A22F040529A609A680A439A6035
:10A7F0009A6822F002029A609A68217E42EA410237
:10A800009A6094F82020002A3ED05A68616A42F487
:10A8100000625A605A6822F460425A605A680139EC
:10A8200042EA41325A60DA6AE16922F47002DA627D
:10A83000DA6A013942EA0152DA629A6822F4007255
:10A840009A609A6894F8301042EA41229A609A68B5
:10A85000616922F480629A609A68002042EA81224B
:10A860009A606064236C23F0030343F001032364C4
:10A87000002384F83C3038BD9A6822F070629A60F8
:10A880009A6822F04052B2E75A6822F40062C9E79F
:10A890000120EDE70120EEE7002301400100000F59
:10A8A00082B00023019390F83C30012B024660D027
:10A8B0000168012380F83C308B68D8070CD5886884
:10A8C00010F001001AD1136C43F010031364536CA1
:10A8D00043F0010353643DE08B68284843F00103D3
:10A8E0008B60274B1B68B3FBF0F303EB430301932F
:10A8F000019B002BE3D0019B013BF8E7136C23F491
:10A90000E06323F0010343F4807313644B685B0539
:10A9100041BF136C23F4405343F480531364136C0E
:10A9200013F480531CBF536C23F0060353640020C0
:10A930006FF0220382F83C000B60124B5A6812F051
:10A940001F0209D1886810F0405014D18B6843F081
:10A9500080438B6002B070470B4B9942FAD18B68F1
:10A9600013F04053F6D18A6842F080428A6018465C
:10A97000F0E70220EEE71046ECE700BF40420F0090
:10A98000B0090020002301400020014003689A68BC
:10A99000520570B504460D460BD59B68DE0508D5FB
:10A9A000036C43F020030364002380F83C30012053
:10A9B00070BDFFF7B5FE064623681A6891070CD5EF
:10A9C0006FF012021A60226C42F4007222649A68DC
:10A9D00012F0405F17D00020EAE7681CEDD065B99F
:10A9E00023681B6813F00203E6D1226C84F83C3024
:10A9F00042F0040222640320DAE7FFF791FE801B95
:10AA0000A842EDD8D8E7207E0028E4D1DA6A12F413
:10AA1000700F02D09B685A05DDD4236C23F4807339
:10AA20002364236CDB04D6D4236C43F0010323643A
:10AA3000BEE70368D86C7047F7B50023019390F820
:10AA40003C30012B69D0012380F83C300D6803684D
:10AA50008E68092DACB234D904EB4402DF681E3A8B
:10AA60004FF0070C0CFA02FC27EA0C07DF60DF68E6
:10AA700006FA02F23A43DA604968062901EB8102DC
:10AA80002FD8596B053A1F26964021EA06015963D3
:10AA9000596B04FA02F20A435A63304A93420AD1CC
:10AAA000122D3CD12E4B5A6822F400025A605A688B
:10AAB00042F480025A60002380F83C30184603B00C
:10AAC000F0BD1F6905EB45024FF0070C0CFA02FCC4
:10AAD00027EA0C071F611F6906FA02F23A431A615E
:10AAE000CAE70C294FF01F010BD81E6B233A914087
:10AAF00026EA01011963196B04FA02F20A431A6388
:10AB0000CBE7DE6A413A914026EA0101D962D96A6F
:10AB100004FA02F20A43DA62BFE70220CFE7114BE0
:10AB20009D4201D0112DC6D10D4B5A6822F48002EE
:10AB30005A605A6842F400025A600A4B9D42BAD1E8
:10AB4000094B0A4A1B68B3FBF2F30A2253430193F1
:10AB5000019B002BAFD0019B013BF8E70020014097
:10AB60000023014012000010B009002040420F00F5
:10AB70000749CA6822F4E0620302120403F4E063A6
:10AB8000120C134343F0BF6343F40033CB607047B0
:10AB900000ED00E0164B30B5DC68C4F30224C4F1CC
:10ABA0000703251D042B28BF0423062D4FF0FF3576
:10ABB00005FA03F38CBF033C002421EA0303A340FE
:10ABC00005FA04F422EA0402002843EA0203ACBFB7
:10ABD00000F16040074A4FEA0313B8BF00F00F00CE
:10ABE000DBB2AABF00F56140135480F8003330BDDA
:10ABF00000ED00E014ED00E0002808DB420901232D
:10AC000000F01F0003FA00F0014B43F822007047E8
:10AC100000E100E000280DDB4309012200F01F00E5
:10AC200002FA00F02033044A42F82300BFF34F8FAA
:10AC3000BFF36F8F704700BF00E100E00138B0F153
:10AC4000807F0BD24FF0E023054A5861F02182F853
:10AC500023100020072298611A6170470120704775
:10AC600000ED00E0094910B50C6924F440740C6152
:10AC70000C6944F440740C610C6944F001040C61EB
:10AC80000260BFF36F8F436010BD00BF003C024005
:10AC9000074B1A6922F440721A611A6942F4007271
:10ACA0001A611A6942F001021A610160704700BF1F
:10ACB000003C0240074B1A6922F440721A611A697B
:10ACC00042F480721A611A6942F001021A6101802D
:10ACD000704700BF003C0240204BDA68D00606D522
:10ACE0001F49CA6942F01002CA611022DA60DA68AC
:10ACF000910606D51A49CA6942F00802CA612022A3
:10AD0000DA60164BDA68520606D51549CA6942F070
:10AD10000402CA614022DA60DA68100606D51049DA
:10AD2000CA6942F00202CA618022DA600B4BDA681B
:10AD3000D10507D50A49CA6942F00102CA614FF438
:10AD40008072DA60DA68920706D50549CA6942F06E
:10AD50002002CA610222DA60704700BF003C024054
:10AD6000340C0020064B1A69002ABFBF054A5A60FE
:10AD700002F188325A60BABF1869C00F00207047CC
:10AD8000003C024023016745034A136943F0004336
:10AD900013610020704700BF003C0240014BD8699E
:10ADA000704700BF340C0020114B70B500220446E0
:10ADB000DA61FFF7B5FC0F4D0646EB68DA030CD4F9
:10ADC000EB68DB0744BF0123EB60E86810F4F9701F
:10ADD00007D0FFF781FF012003E0611CEDD00CB923
:10ADE000032070BDFFF79CFC801BA042E5D9F7E76C
:10ADF000340C0020003C02402DE9F0411F4E9846E3
:10AE0000337E012B07460D46144635D001234CF204
:10AE100050303376FFF7C8FFB0B9CFB9184B1A6975
:10AE200022F440721A611A691A611A69E4B242F096
:10AE300001021A612C704CF25030FFF7B5FF104A36
:10AE4000136923F00103136100233376BDE8F08119
:10AE5000012F04D1A1B22846FFF72CFFEBE7022F08
:10AE600004D121462846FFF713FFE4E72246434674
:10AE70002846FFF7F7FEDEE70220E7E7340C002064
:10AE8000003C024039B101291CD002290CBF4FF40B
:10AE900000714FF440710D4B1A6922F440721A612F
:10AEA0001A69114319611A6922F0F8021A611A69C4
:10AEB00042EAC00040F0020018611A6942F4803290
:10AEC0001A6170474FF48071E5E700BF003C024013
:10AED0002DE9F74FDFF87C915F4A00230D680124CC
:10AEE0009C4004EA050CAC4340F0A6804D6805F098
:10AEF00003044FEA43080326671E06FA08F6012FEB
:10AF00006FEA060634D8876807EA060ECF6807FAA4
:10AF100008F747EA0E078760476827EA0C0EC5F373
:10AF200000179F4047EA0E074760C76807EA060E0A
:10AF30008F6807FA08F747EA0E07022CC76019D195
:10AF40004FEAD30A00EB8A0A03F0070BDAF8207005
:10AF50004FEA8B0B4FF00F0E0EFA0BFE27EA0E0E88
:10AF60000F6907FA0BF747EA0E07CAF8207001E0ED
:10AF7000032CDAD1076804FA08F43E40264315F49E
:10AF8000403F066058D000240194D9F8446046F44C
:10AF90008046C9F84460D9F8446006F480460196BA
:10AFA000019E23F0030606F1804606F59C3603F069
:10AFB000030ED6F808804FEA8E0E0F2707FA0EF719
:10AFC00028EA0707DFF89480404513D004F1804455
:10AFD00004F50134A04236D004F58064A04234D098
:10AFE00004F58064A04232D004F58064A0420CBF16
:10AFF0000424072404FA0EF43C43B46094686FEA16
:10B000000C06EF0254BF34404CEA04049460D46848
:10B01000AF0254BF34404CEA0404D4605468AF0318
:10B0200054BF34404CEA040454601468ED0354BF28
:10B0300034404CEA040414600133102B7FF44EAF0B
:10B0400003B0BDE8F08F0124D4E70224D2E7032443
:10B05000D0E700BF00380240003C01400000024041
:10B060000369194214BF0120002070470AB18161B1
:10B0700070470904FBE7436901EA030221EA03017F
:10B0800041EA02418161704701684B6913F48063B2
:10B090004FF0000210D06FF480634B6120230263F5
:10B0A00080F83D3080F83E20036C80F83C2043F06F
:10B0B0000403036401207047184670472DE9F846E1
:10B0C00006460F4691461D464FEA114A3368BAF1CB
:10B0D000010F0CBF5C699C6927EA0404A4B2B4FAAE
:10B0E00084F46409A14501D0002017E06A1CEED069
:10B0F000FFF716FB089BC01AA84201D8002DE5D126
:10B1000000232022336386F83D2086F83E30326CDF
:10B1100086F83C3042F0200232640120BDE8F88617
:10B120002DE9F04104460F461646984625686869A1
:10B1300027EA000080B2B8B16B695A0516D52B68B2
:10B1400043F400732B606FF480636B612022002353
:10B15000236384F83D2084F83E30226C42F00402E0
:10B16000226484F83C300120BDE8F081731CDED0FD
:10B17000FFF7D6FAA0EB0800B04201D8002ED5D1D7
:10B1800000232022236384F83D2084F83E30226C83
:10B1900042F02002E4E770B504460D4616462368E7
:10B1A0005B695B0701D5002070BD2046FFF76CFF8F
:10B1B000A8B96A1CF3D0FFF7B3FA801BA84201D8E4
:10B1C000002DECD100232022236384F83D2084F855
:10B1D0003E30226C84F83C3042F020022264012090
:10B1E000E2E770B504460D46164623685B691B0608
:10B1F00001D5002070BD2046FFF746FFA8B96A1CA4
:10B20000F3D0FFF78DFA801BA84201D8002DECD1B6
:10B2100000232022236384F83D2084F83E30226CF2
:10B2200084F83C3042F0200222640120E2E7000072
:10B2300070B5044608B9012070BD90F83D3003F0A8
:10B24000FF021BB980F83C20FFF7D6F8242384F8CE
:10B250003D3023681A6822F001021A601A6842F42D
:10B2600000421A601A6822F400421A6001F036F8AF
:10B270003F4A6368934294BF3E4A3F4A90428CBF24
:10B2800000220122002AD6D12268394E55683B4956
:10B29000B0FBF1F125F03F050D43B342556088BF87
:10B2A0004FF49676156A88BF714325F03F0584BF39
:10B2B0004FF47A76B1FBF6F1013129431162D1697D
:10B2C0002B4D21F44F41AB4221F0FF0100F1FF3043
:10B2D00032D85B00B0FBF3F0431C40F6FC70034235
:10B2E00042D0C3F30B030B43D361D4E90730116899
:10B2F000034321F0C0010B4313609168D4E90303B9
:10B3000021F40341034321F0FF010B439360D4E98F
:10B310000530D168034321F0FF010B43D36013686C
:10B3200043F00103136000202023206484F83D30A3
:10B33000206384F83E007FE7A56855B903EB43031B
:10B34000B0FBF3F30133C3F30B037BB143F40043CE
:10B35000C9E719256B43B0FBF3F30133C3F30B03C8
:10B3600023B143F44043BEE70423BCE70123BAE71B
:10B37000A08601007F841E00FF083D0040420F00B0
:10B380002DE9F043044685B098460C9F0D46914642
:10B39000FFF7C6F994F83D30202B064604D002256D
:10B3A000284605B0BDE8F08300905D4919230122CD
:10B3B0002046FFF783FE0028F1D194F83C30012BA2
:10B3C000EDD02168012384F83C300B68DA075EBFBA
:10B3D0000B6843F001030B600B6823F400630B6000
:10B3E000212384F83D30102384F83E300023236469
:10B3F000A4F82A80638D23854A4BE362E36AC4F88C
:10B400002490082B04D0012B02D013F5803F04D1E7
:10B410000B6843F480730B6002E0236B122BF7D0B0
:10B42000002200963B464FF001112046FFF746FEF2
:10B43000226838B11368DB0544BF4FF400732364FE
:10B440000125ADE72369B3F5804F21D105F0FE0555
:10B450001561354933463A462046FFF761FE0546F9
:10B460000028EDD1236803905A6903929B690393E6
:10B47000039B238DF3B921680A6842F400720A60C5
:10B48000202284F83D2084F83C3084F83E3087E761
:10B49000EB1103F0060343F0F00313612349334635
:10B4A0003A462046FFF73CFE0028C9D12368EDB29A
:10B4B0001D61CEE7324639462046FFF792FE40B185
:10B4C000236C042BBCD12268136843F4007313600F
:10B4D000B6E7636A20681A4612F8011B01616262CE
:10B4E000628D013A92B26285228DD0F814C0511E4D
:10B4F00089B21CF0040F21850AD049B15978016145
:10B5000002336362638D013B9BB2023A63852285FD
:10B51000324639462046FFF73EFE0028A9D0CFE745
:10B52000020010000000FFFF0200010008000100FF
:10B5300010B590F8BC24012A04460BD0012280F8F3
:10B54000BC2480F83810006801F00CFD002084F85D
:10B55000BC0410BD0220FCE770B501F00F0606EB3D
:10B56000C60411F0800F05464FEA84044FF0240012
:10B570001FD000FB065004F13C010124294480F84F
:10B580003D40CA604A780E700B7102B10E81022BE9
:10B5900004BF00234B7195F8BC34012B12D001235A
:10B5A000286885F8BC3401F06CFA002085F8BC04EA
:10B5B00070BD00FB065004F51F710024294480F87B
:10B5C0007D42DEE70220F3E738B501F00F052424C1
:10B5D00004FB050104FB050401F51F71C4F8943256
:10B5E0000023C4F88C22C4F89C3284F87D3284F89D
:10B5F0007C5203690068012B08BFC4F89022DAB2BC
:10B600001DB901F07DFA002038BD01F04BFBFAE7CF
:10B6100038B501F00F05242404FB050104FB0504E3
:10B620003C3163650023E3650123E26484F83D3027
:10B6300084F83C5003690068012B08BF2265DAB228
:10B640001DB901F05DFA002038BD01F02BFBFAE7CF
:10B6500038B5436801F00F059D4204462CD811F01F
:10B66000800F4FF024001ED000FB054200FB054177
:10B6700001233C3182F83D3001238B700D7094F82A
:10B68000BC249A421AD0206884F8BC3401F016FC1D
:10B690002DB9217C206804F2C44201F0B7FC0020DF
:10B6A00084F8BC0438BD00FB01431A4603F51F7142
:10B6B000002382F87D32DFE70120F3E70220F1E783
:10B6C00038B5436801F00F029A4204462AD802EBCB
:10B6D000C20311F0800F4FEA83034FF0240018D00B
:10B6E00000FB024003F13C010123214480F83D307E
:10B6F00000258D700A7094F8BC34012B14D00123FE
:10B70000206884F8BC3401F004FC84F8BC5428465A
:10B7100038BD00FB024003F51F710023214480F86F
:10B720007D32E5E70120F3E70220F1E701F00F03A6
:10B7300003EBC3030A064FEA83034CBF03F13C014A
:10B7400003F51F710144006801F056BA2DE9F04F6E
:10B75000066889B00446304601F043FC0390002897
:10B7600040F05681206801F00DFC002800F0508167
:10B77000D6F808382068C3F30D23C4F8FC3401F070
:10B7800001FC810748BF2268206842BF536903F06B
:10B790000203536101F0F6FBC20606F500652CD5E5
:10B7A0002268936923F010039361D6F82080C8F3D0
:10B7B0004343022B08F00F0740F02D8147F6F0734A
:10B7C00018EA030F14D0242303FB0747C8F30A1910
:10B7D000D7F88C124A46304601F050FBD7F88C322D
:10B7E0004B44C7F88C32D7F89C324B44C7F89C3294
:10B7F0002268936943F010039361206801F0C2FB53
:10B80000030300F11A81206801F0BCFB47030CD54B
:10B81000206801F0C3FB2746049006F5106A4FF03C
:10B820000009049B002B40F0D081206801F0AAFBA6
:10B83000002813DA6B6823F001036B6094F8F4348A
:10B84000012B40F06A82002184F8F414204600F0B5
:10B85000C3FA2268536903F000435361206801F082
:10B8600091FB01050AD5AB68DA0702D5204603F043
:10B870006FF82268536903F400635361206801F094
:10B8800081FBC30433D56B68206823F001036B6030
:10B89000102101F0C5F806F510634FF67F3162689C
:10B8A0000398824200F24282EB6943F00113EB619C
:10B8B000236B002B00F05282D5F8843043F00B0349
:10B8C000C5F884306B6C43F00B036B64D6F800381A
:10B8D000217C206823F4FE63C6F8003804F2C442D9
:10B8E00001F094FB2268536903F48053536120688C
:10B8F00001F048FB870416D5206801F076FB20682C
:10B9000001F0B4F8E060276800F0E2FC227B014619
:10B91000384601F015F8204603F007F8226853690D
:10B9200003F400535361206801F02CFB000707D596
:10B93000204602F0F6FF2268536903F008035361C2
:10B94000206801F01FFB010600F11382206801F05E
:10B9500019FBC2020CD5A04606F5126901276368DF
:10B96000BB4200F21F822268536903F480135361C3
:10B97000206801F007FB83022DD5D4F804E02346AC
:10B9800006F5326001218E4520D993F8A4C20268E1
:10B99000BCF1010F40F01C82002A80F21982D4F819
:10B9A000FC7402F4803207F00107BA4240F01082C2
:10B9B00083F8A3C2B26942F08002B26172691706CD
:10B9C00000F106826B6843F400736B602268536970
:10B9D00003F400135361206801F0D4FA410007D545
:10B9E000204602F0D9FF2268536903F08043536177
:10B9F000206801F0C7FA42070AD523685D686B0723
:10BA000002D5204602F0CCFF226853682B435360D6
:10BA100009B0BDE8F08F062B7FF4EAAE082204F2ED
:10BA2000C441304601F02AFA242303FB0747C8F338
:10BA30000A18D7F89C324344D8E6206801F0A6FAE9
:10BA400006F530680490A2460027049B002B3FF4C3
:10BA5000DAAE049BD80776D55FFA87FB2068594693
:10BA600001F0A4FA10F0010F81461CD02068216972
:10BA70000123C8F8083000F5306303EB47130129B0
:10BA8000D0F840C09A6840F08B80110707D5A549CF
:10BA90008C4508D9100406D54FF4004202E0910607
:10BAA0005AD520229A6019F0080F21D00823C8F82F
:10BAB000083023689B481A6C03F5306303EB471387
:10BAC0008242996804D9090444BF4FF40041996047
:10BAD0002046059202F00EFF924B059A9A4207D932
:10BAE0002169012904D1206804F2C44201F08EFAD0
:10BAF00019F0100F1CBF1023C8F8083019F0020FFE
:10BB000014D073691B0642BF6B6843F480636B609B
:10BB10009AF87F32012B06D100238AF87F325946EA
:10BB2000204602F031FF0223C8F8083019F0200F38
:10BB30001CBF2023C8F8083019F4005F1CBF4FF465
:10BB40000053C8F80830049B5B080137049308F1E0
:10BB500020080AF1240A78E712F0280FA3D17149CE
:10BB60008C4501D9120497D41A69DAF89832C2F3D5
:10BB700012029B1ACAF89C326FB9D4F894222AB9DF
:10BB800004F2C442012101F041FA04E0D4F88C220D
:10BB90001344C4F88C325946204602F0B1FE82E7C5
:10BBA00061498C4507D111043FF576AF9006F2D577
:10BBB00020229A60EFE7002FEDD1D4F89432002BC9
:10BBC000E9D104F2C4423946DDE7049BD80740F1CD
:10BBD0009B805FFA89FB2068594601F0F0F910F06C
:10BBE000010F80461FD06B6B012109F00F0201FA93
:10BBF00002F223EA02036B63CAF8081021690129E3
:10BC00000DD1D7E912231344FB64B9F1000F06D11B
:10BC1000636D23B9206804F2C44201F0F7F9594674
:10BC2000204602F076FE18F0080F1CBF0823CAF861
:10BC3000083018F0100F1CBF1023CAF8083018F095
:10BC4000400F1CBF4023CAF8083018F0020F12D072
:10BC50004946304600F0E4FE97F83F30012B07D10B
:10BC60004FF0000387F83F305946204602F090FE1F
:10BC70000223CAF8083018F0800F45D0FA6D7B6DAA
:10BC80009A4241D89B1ABA6C21680591934228BF09
:10BC9000134603339B08069301F5106303EB491326
:10BCA0000793079B06989969FA6D7B6D89B281426B
:10BCB00028D39A420CD3059B09F00F01D3F83428FE
:10BCC000012000FA01F122EA0102C3F834281BE046
:10BCD000A3EB0208BB6C0598984528BF984608F16D
:10BCE00003039B080693237C0093F96C1FFA88F3E7
:10BCF0005A4600F0C3FFFB6C4344FB64FB6D4344B6
:10BD0000FB65CEE79A42D6D2049B5B0809F1010994
:10BD1000049324370AF1200A83E5204602F030FE1E
:10BD200097E500BF0A30544F0A31544F99601A68A2
:10BD300022F400121A60C3F80812D3F8002222F489
:10BD40000012C3F80022D3F8002242F00062C3F8C8
:10BD50000022039A013203922033A0E56B6943F479
:10BD6000005343F02B036B612B6943F00B032B61F2
:10BD7000ACE5B36923F08003B361012704F27F28A7
:10BD80004FF024096368BB427FF6E0AD09FB07F37F
:10BD900018F80330012B03D1F9B22046FFF7C6FC97
:10BDA0000137EFE798F86430D9F80020012B09D16A
:10BDB000002A07DA67F07F0188F86330C9B22046AD
:10BDC000FFF7B4FC013708F1240809F12009C6E5A2
:10BDD000013124332030D6E5704700002DE9F341CE
:10BDE000044640B30368DD0710D4236898075ED487
:10BDF00023681A0700F1A08023685B0700F1C08068
:10BE0000A069002840F0288100202BE08F4B9A6821
:10BE100002F00C02042A07D09A6802F00C02082AE9
:10BE20000BD15A68510208D5884B1B689A03DCD5A0
:10BE30006368002BD9D1012014E06268B2F5803F1D
:10BE400013D11A6842F480321A60FEF769FC7F4E03
:10BE5000054633689B03C8D4FEF762FC401B642888
:10BE6000F7D9032002B0BDE8F081784DB2F5A02FDC
:10BE70002B6807D143F480232B602B6843F4803375
:10BE80002B60E2E723F480332B602B6823F48023BC
:10BE90002B60002AD9D1FEF743FC06462B689F038E
:10BEA000A3D5FEF73DFC801B6428F7D9D9E7674B83
:10BEB0009A6812F00C0F07D09A6802F00C02082A58
:10BEC00011D15B685E020ED4604A13689D0702D5EB
:10BED000E368012BAFD11368216923F0F80343EA2B
:10BEE000C103136084E7E268594BB2B101221A60C2
:10BEF000FEF716FC554D06462B68980707D52B68AC
:10BF0000226923F0F80343EAC2032B6070E7FEF7CF
:10BF100007FC801B0228EFD9A3E71A60FEF700FC9C
:10BF20004A4E0546336899077FF562AFFEF7F8FB86
:10BF3000401B0228F6D994E76269454B82B1012281
:10BF4000C3F8802EFEF7ECFB404E0546736F9F074B
:10BF50003FF552AFFEF7E4FB401B0228F6D980E71D
:10BF6000C3F8802EFEF7DCFB384E0546736F98074A
:10BF70007FF542AFFEF7D4FB401B0228F6D970E7ED
:10BF8000324B1A6C12F0805228D101921A6C42F096
:10BF900080521A641B6C03F080530193019B0127AC
:10BFA0002C4D2B68D9051BD5A368284D012B27D113
:10BFB0002B6F43F001032B67FEF7B2FB234E0546C0
:10BFC00041F28838336F9B0739D5002F3FF418AF03
:10BFD0001E4A136C23F08053136411E70027DFE738
:10BFE0002B6843F480732B60FEF79AFB06462B68A0
:10BFF000DA05D9D4FEF794FB801B0228F7D930E785
:10C00000052B04D12B6F43F004032B67D0E72A6F75
:10C0100022F001022A672A6F22F004022A67002B0D
:10C02000CAD1FEF77DFB41F2883806462B6F980790
:10C03000CBD5FEF775FB801B4045F7D911E7FEF71E
:10C040006FFB401B4045BDD90BE700BF00380240E5
:10C050000000474200700040364DAB6803F00C030F
:10C06000082B3DD0344B002202281A662BD1FEF754
:10C0700057FB06462B6899011FD4D4E907321343B6
:10C08000626A43EA8213E26A43EA0263A26A5208DE
:10C09000013A43EA02436B60274B264D01221A66A0
:10C0A000FEF73EFB04462B689A013FF5ADAEFEF766
:10C0B00037FB001B0228F6D9D3E6FEF731FB801BC5
:10C0C0000228D7D9CDE6FEF72BFB04462B689B014F
:10C0D0007FF59AAEFEF724FB001B0228F6D9C0E6D6
:10C0E00001283FF4BFAE6B68E26903F4800191421E
:10C0F0007FF4A1AE216A03F03F028A427FF49BAE37
:10C10000616A47F6C0721A40B2EB811F7FF493AEAA
:10C11000A26A520803F44031013AB1EB024F7FF4B6
:10C120008AAEE26A03F07063B3EB026F3FF46CAE69
:10C1300081E600BF0038024000004742134908B5BD
:10C140008B6803F00C03042B1CD0082B1CD14A680D
:10C150004B68496813F4800314BF0D480D48C1F3C0
:10C16000881118BF002302F03F02A1FB0001F4F781
:10C170006BF8064B5B68C3F3014301335B00B0FB14
:10C18000F3F008BD0248FCE70248FAE70038024035
:10C19000001BB7000024F4002DE9F0410D460446D1
:10C1A00010B90120BDE8F081444B1A6802F0070283
:10C1B0008A4228D3226897072DD4D00741D43F4B19
:10C1C0001A6802F00702AA4266D8226851076CD4A6
:10C1D000130707D53A4A2169936823F4604343EA79
:10C1E000C1039360FFF7AAFF354B364A9B68C3F340
:10C1F0000313D35CD840344B1860344B1868FEF7F7
:10C2000045FA0020CEE7CAB21A701B6803F0070394
:10C210008B42C6D1CEE72A4B12F0040F1EBF99689D
:10C2200041F4E0519960160742BF996841F46041BA
:10C2300099602349A0688B6823F0F00303438B6067
:10C24000BBE762681E4B012A1CD11B6813F4003F38
:10C25000A7D01B4EB36823F003031343B360FEF76C
:10C260005FFA41F288380746B368626803F00C034E
:10C27000B3EB820FA3D0FEF753FAC01B4045F3D9AE
:10C2800003208FE7911E01291B6802D813F0007F5D
:10C29000DEE713F0020FDBE7EAB21A701B6803F067
:10C2A0000703AB427FF47DAF8FE70549E0688B68F9
:10C2B00023F4E05303438B608AE700BF003C024055
:10C2C00000380240180B0108B0090020B80900200E
:10C2D000014B1868704700BFB0090020044B054AA5
:10C2E0009B68C3F38223D35C034A1068D84070472D
:10C2F00000380240280B0108B0090020044B054A11
:10C300009B68C3F34233D35C034A1068D84070473C
:10C3100000380240280B0108B009002090F83D3099
:10C32000012B28D1022380F83D300368DA6842F0FF
:10C330000102DA60114A934212D0B3F1804F0FD05C
:10C34000A2F57C4293420BD002F58062934207D063
:10C3500002F58062934203D002F59A32934204D1EF
:10C360009A6802F00702062A03D01A6842F0010216
:10C370001A60002070470120704700BF0000014094
:10C38000704770477047704703681A69910710B586
:10C3900004460ED5DA6892070BD56FF002021A61D7
:10C3A000012202779B699B0777D0FFF7EAFF002302
:10C3B000237723681A69500710D5DA6851070DD51D
:10C3C0006FF004021A61022222779B6913F4407F06
:10C3D000204668D0FFF7D5FF0023237723681A692A
:10C3E00012070FD5DA6810070CD56FF008021A6132
:10C3F00004222277DB69990720465AD0FFF7C1FF54
:10C400000023237723681A69D20610D5DA68D0068C
:10C410000DD56FF010021A6108222277DB6913F440
:10C42000407F20464BD0FFF7ACFF002323772368E3
:10C430001A69D10708D5DA68D20705D56FF001026D
:10C440001A612046FCF7ECFB23681A69100608D530
:10C45000DA68110605D56FF080021A61204600F0F7
:10C4600056F923681A69520608D5DA68500605D5C8
:10C470006FF040021A612046FFF785FF23681A69B2
:10C48000910622D5DA6892061FD56FF02002204669
:10C490001A61BDE8104000F039B9FFF771FF20467E
:10C4A000FFF770FF83E7FFF76BFF2046FFF76AFF98
:10C4B00092E7FFF765FF2046FFF764FFA0E7FFF76D
:10C4C0005FFF2046FFF75EFFAFE710BD244A036819
:10C4D00090420ED0B0F1804F0BD0A2F57C4290423A
:10C4E00007D002F58062904203D002F5806290424C
:10C4F00015D14A6823F070031343194A904219D0AA
:10C50000B0F1804F16D0A2F57C42904212D002F5D5
:10C51000806290420ED002F5806290420AD0114AA9
:10C52000904207D002F58062904203D002F580620B
:10C53000904203D1CA6823F4407313434A6923F03D
:10C540008003134303608B68C3620B688362044BF0
:10C55000984204BF0B69036301234361704700BF26
:10C56000000001400040014010B5044630B390F88F
:10C570003D3003F0FF021BB980F83C20FDF774FF4B
:10C580000223206884F83D30211DFFF79FFF01231F
:10C5900084F84630002084F83E3084F83F3084F838
:10C5A000403084F8413084F8423084F8433084F8D5
:10C5B000443084F8453084F83D3010BD0120FCE75C
:10C5C00010B584680A4324F47F4442EA03222243DC
:10C5D000826010BD70B590F83C30012B04464FF0DE
:10C5E000020300F09180012280F83D3080F83C2069
:10C5F0000068836823F47F4323F0770383600B682C
:10C60000602B52D033D8402B67D016D8202B0DD0BA
:10C610000AD833F0100109D0012384F83D300023FB
:10C6200084F83C30104670BD302BF5D1826822F082
:10C630007002134343F0070317E0502BECD14A6814
:10C64000CE68016A056A25F001050562836921F05B
:10C650000A0123F0F00343EA06130A4383610262EE
:10C66000836823F0700343F05703836011E0B3F550
:10C67000805F0ED0B3F5005F0DD0702BCCD1CB68AE
:10C68000D1E90121FFF79CFF2268936843F077030B
:10C6900093600022C0E7CB68D1E90121FFF790FF4A
:10C6A0002268936843F48043F2E74D68CE68016ADC
:10C6B00021F0100101628269036A22F4704223F0C2
:10C6C000A00343EA051342EA0632826103628368EB
:10C6D00023F0700343F06703C7E74A68CE68016A36
:10C6E000056A25F001050562836921F00A0123F03E
:10C6F000F00343EA06130A4383610262836823F06E
:10C70000700343F04703B0E71A468BE77047704762
:10C710000268C16838B5136923F440530B431361B1
:10C72000054683680069D168034368690343E86983
:10C7300021F4164121F00C0103430B43D3605369EC
:10C74000A96923F440730B4353611F4B9A4203D0F2
:10C7500003F580639A4224D1FFF7D0FDEA691921DD
:10C76000B2F5004FD5E90043A0FB01011CD1DA1856
:10C770004FF0000545EB0503F3F766FD6421B0FBC0
:10C78000F1F501FB1503DB003233B3FBF1F303F0EA
:10C7900007025B0002EB051203F4F8731344A36075
:10C7A00038BDFFF79BFDD9E79A009B0FF3F74CFDCF
:10C7B0006422B0FBF2F102FB11031B013233B3FB25
:10C7C000F2F303EB0113EAE700100140F8B5044669
:10C7D0000E4617461D462268136836EA030301D148
:10C7E000002028E06B1CF7D025B1FDF799FFC01B96
:10C7F0008542F0D2226802F10C0353E8003F23F493
:10C80000D0730C3242E8003021680028F2D101F1E7
:10C81000140353E8003F23F0010301F1140040E842
:10C820000032002AF3D1202384F83D3084F83C20E4
:10C8300084F83E300320F8BD10B5044640B390F8AC
:10C840003D3003F0FF021BB980F83C20FDF73EFEAF
:10C850002268242384F83D30D36823F40053D36046
:10C860002046FFF755FF23681A6922F490421A61A7
:10C870005A6922F02A025A61DA6842F40052DA60F8
:10C8800000202023206484F83D3084F83E3010BD21
:10C890000120FCE72DE9F843994690F83D30202B24
:10C8A00004460E46174648D1002944D0002A42D0FB
:10C8B00090F83C30012B40D0012380F83C3000251B
:10C8C0002123056480F83D30FDF72AFFA368A78483
:10C8D000B3F5805F8046E78403D123690BB9354601
:10C8E0001E46002384F83C30E38C9BB253B94B4680
:10C8F000424640212046FFF769FF50B9202384F8C3
:10C900003D3007E04B46424680212046FFF75EFF60
:10C9100010B10320BDE8F88322684EB935F8023B18
:10C92000C3F308035360E18C013989B2E184DBE78A
:10C9300016F8013BF6E70120ECE70220EAE70000E9
:10C94000022A4AD1274B284A0B44934239D9274B14
:10C95000274A0B44934236D9264AA1F57403A3F51E
:10C960001053934231D9244AA1F18373A3F5E743CD
:10C9700093422CD3214B224A0B44934229D9214B79
:10C98000214A0B44934226D3204B214A0B44934225
:10C9900023D3204AA1F1B773A3F5585393421ED372
:10C9A0001D4B1E4A0B44934234BF07230623C26823
:10C9B00022F47052C260C26842EA8323C36000203E
:10C9C00070470F23F3E70E23F1E70D23EFE70C2366
:10C9D000EDE70B23EBE70A23E9E70923E7E7082361
:10C9E000E5E700BF405327FFFF340C00401E1BFF4C
:10C9F0003F420F007F4F120020D6130060B6E5FEC5
:10CA00005FE3160000D3CEFE40771B00C05BB3FE91
:10CA1000C091210020753800E05459FEE09C41008F
:10CA200082B00246002310480193019B0133019319
:10CA3000019B834215D81369002BF6DA890141F076
:10CA400020010023019311610749019B01330193E8
:10CA5000019B8B4205D8106910F02000F5D102B07F
:10CA600070470320FBE700BF400D0300D0F80838F3
:10CA700013F0060004D013F0020F14BF02200F20A1
:10CA8000704730B50D78012405F00F039C404B78BA
:10CA900000F50062012B00EB4510D36918D11C434F
:10CAA000D461D0F800391A0410D4CA68D0F800490B
:10CAB000C2F30A030A79234343EA824343EA8553D4
:10CAC00043F0805343F40043C0F80039002030BDE8
:10CAD00043EA0444D461D0F8003B1B04F6D4CB688D
:10CAE000D0F8002BC3F30A0313430A7943EA8243C5
:10CAF00043F0805343F40043C0F8003BE6E70000F6
:10CB00004B78DFF8ECC0F0B50E788D69394F012B0A
:10CB100000EB461446D104F51063BDB91D692F40E2
:10CB20001F611D6945F400251D611D6905EA0C059D
:10CB3000012A1D6123D14A6902B15A61D4F8003932
:10CB400043F00443C4F800390020F0BDD3F810E0EE
:10CB50000EEA0C0CC3F810C0D3F810C00CEA07079B
:10CB60001F61CF68AF421D6938BF8F6145F4002552
:10CB70001D618D691F69C5F312053D43D8E7D4F8DF
:10CB8000003943F00443C4F800398B69002BDBD033
:10CB9000D0F8342806F00F060123B3401343C0F841
:10CBA0003438D1E7D4F8100B00EA0C00C4F8100BAD
:10CBB000D4F8100B384004F530631861C86805B12B
:10CBC00088611D69C86145F400251D611D69C0F3B8
:10CBD00012002843012A186102D10A6902B15A6180
:10CBE000D4F8003B43F00443C4F8003BACE700BF7B
:10CBF0000000F8FFFFFF07E082B000234A780193AE
:10CC00000B78012A4FEA43131ED100F51060C118BA
:10CC1000C258002A02DB002002B07047C25842F01E
:10CC20000062C250C25842F08042C25042F21072BA
:10CC3000019B01330193019B934201D90120EBE752
:10CC40000B68002BF4DBE6E700F53060C118C25832
:10CC5000002AE0DAC25842F00062C250C25842F0E4
:10CC60008042C25042F21072019B01330193019B3A
:10CC70009342E3D80B68002BF6DBCCE710B59DF8A8
:10CC8000084044B9033301329B0800EB023001EB4A
:10CC900083038B4201D1002010BD51F8042B0260A8
:10CCA000F7E700002DE9F3414D788B690F79DFF844
:10CCB000C0C1DFF8C0E116460A78012D00EB42142E
:10CCC00040F08D8004F51065D5F810806BBB08EA44
:10CCD0000C0CC5F810C0D5F810C04CF4002CC5F8E9
:10CCE00010C0D5F810C00CEA0E0EC5F810E0012EE9
:10CCF0004ED14B6903B16B61012F0CD1D0F80838CC
:10CD000013F4807FD4F800390CBF43F0005343F094
:10CD10008053C4F80039D4F8003943F00443C4F810
:10CD20000039002002B0BDE8F08108EA0E0EC5F817
:10CD300010E0D5F810E00EEA0C0CD1F80CE0C5F8C4
:10CD400010C00EEB030C0CF1FF3CBCFBFEFEDFF849
:10CD500028C1D5F810800CEACE4C4CEA080CC5F876
:10CD600010C0D5F810E0C3F3120C4CEA0E0C012FE2
:10CD7000C5F810C0BBD1D5F810C02CF0C04CC5F818
:10CD800010C0D5F810C04CF0005CC5F810C0AEE77C
:10CD9000D4F80059012F45F00445C4F800590BD0D0
:10CDA000002BBED0D0F8343802F00F0101228A40A7
:10CDB0001A43C0F83428B4E7D0F8085815F4807F37
:10CDC000D4F800590CBF45F0005545F08055C4F823
:10CDD0000059009609699BB2FFF750FFA1E7D4F80C
:10CDE000105B05EA0E05C4F8105BD4F8105B05EA89
:10CDF0000C0504F530621561CD681BBB1369C5F3E2
:10CE000012051D431561136943F400231361012EBC
:10CE100002D10B6903B15361012F0CD1D0F808384E
:10CE200013F4807FD4F8003B0CBF43F0005343F071
:10CE30008053C4F8003BD4F8003B43F00443C4F8EB
:10CE4000003B6EE72B44DFF830C0D2F810E0013B26
:10CE5000B3FBF5F39BB25D430CEAC34343EA0E0315
:10CE6000CD6113611369C5F312051D431561CEE74A
:10CE7000FFFF07E00000F8FF0000F81F034670B551
:10CE80009008002402F0030203F58055844210D379
:10CE900001EB800062B103F580531C680023D900C8
:10CEA00024FA01F1C154013399B28A42F7D11044F6
:10CEB00070BD2E6841F824600134E7E74A780B78AA
:10CEC000012A00EB431012D1D0F80029002A06DB1A
:10CED0002BB1D0F8003923F08043C0F80039D0F8E6
:10CEE000003943F40013C0F8003900207047D0F82F
:10CEF000002B002A06DB2BB1D0F8003B23F0804347
:10CF0000C0F8003BD0F8003B43F40013C0F8003BEE
:10CF1000EBE70B784A7800EB43100B79012AA3F179
:10CF20000203DBB20FD1D0F80029012B22F400124A
:10CF3000C0F8002905D8D0F8003943F08053C0F874
:10CF4000003900207047D0F8002B22F40012012B8A
:10CF5000C0F8002B9EBFD0F8003B43F08053C0F8D0
:10CF6000003BEEE7D0F8003823F4FE63C0F8003849
:10CF7000D0F80038090101F4FE611943C0F8001827
:10CF8000002070474269806910407047D0F8183817
:10CF900000F50060C0691840000C7047D0F81838E0
:10CFA00000F50060C069184080B2704700EB411185
:10CFB00000F50060D1F8082B40691040704710B5AB
:10CFC000D0F81048D0F8343800EB411001F00F01D0
:10CFD000CB4000F51060DB018068DBB223431840D2
:10CFE00010BD406900F001007047D0F8003923F40B
:10CFF000FF6323F00703C0F80039D0F8043843F486
:10D000008073C0F8043800207047000030B5056C0C
:10D01000104CA54200F5306303D9D0F8004B002C2A
:10D0200016DB00241C611C6944F400241C611C698B
:10D0300044F018041C611C69012944F0C0441C61BF
:10D0400001BF5A61D0F8003B43F08023C0F8003B99
:10D05000002030BD0A30544FD0F8B8320BB11B68F5
:10D0600018471846704708B5D0F8B8325B6898473B
:10D07000002818BF032008BD38B5044600F2AA25D1
:10D08000284600F072FB012394F8AA12C4F89432E7
:10D09000B4F8B032C4F8983201F01F03012B08D065
:10D0A000022B0CD08BB929462046BDE8384000F051
:10D0B00039B929462046BDE8384000F089BA2946EA
:10D0C0002046BDE8384000F0B2BA204601F08001A9
:10D0D000BDE8384001F090BC70B50446164609BB67
:10D0E000D0F89432032B0CD1D0E9573293420AD9AD
:10D0F0009B1A9A42C0F85C3128BF1A46314600F0AC
:10D1000054FB002070BD90F89C32032B06D1D0F860
:10D11000B8321B6913B1C0F8D4129847204600F00A
:10D120004CFBEEE790F89C32032BEAD1D0F8B832F2
:10D130009B69002BE5D00022BDE87040C0F8D422E6
:10D14000184770B5044616460D4600293DD1D0F863
:10D150009432022B0ED1D0E90732934212D99A1A97
:10D16000C261314600F019FB2B462A46294620466B
:10D1700001F066FC94F8A03213B1002384F8A032C9
:10D18000002070BD0CD18269934209D8D0F8983242
:10D190009A4205D20A4600F000FBC4F89852E3E731
:10D1A00094F89C32032B08D1D4F8B832DB6823B151
:10D1B0000022C4F8D422204698478021204601F05E
:10D1C0001BFC204600F004FBD4E790F89C32032BB4
:10D1D000D6D1D0F8B8325B69002BD1D00022BDE89F
:10D1E0007040C0F8D4221847F8B5012380F89C326B
:10D1F000D0F8B83200210446C0F894124160C0F85B
:10D20000A41280F8A012B3B90026002240251146CE
:10D2100001274023204601F0E3FBA4F86471C4F821
:10D2200060512B4600228021204601F0D9FBA784C3
:10D2300025623046F8BD5B68002BE5D09847002892
:10D24000E2D00326E1E701740020704790F89C3299
:10D25000DBB280F89D32042380F89C3200207047B6
:10D2600090F89C32042B02BF90F89D32DBB280F81C
:10D270009C320020704708B590F89C22032A05D103
:10D28000D0F8B83213B1DB6903B19847002008BD6C
:10D29000D0F8D422AE3208B550F8222042B190F82E
:10D2A0009C32032B02D1136A23B19847002000E07F
:10D2B000032008BD1846FCE7D0F8D422AE3208B5EA
:10D2C00050F8222042B190F89C32032B02D1536ACD
:10D2D00023B19847002000E0032008BD1846FCE772
:10D2E00000207047012208B580F89C22D0F8B822AF
:10D2F0000AB9002008BD5268017990470028F8D08B
:10D300000320F7E7002070470020704710B5802108
:10D31000044601F071FB20460021BDE8104001F0F9
:10D320006BBB00002DE9F3410D7805F06005202D61
:10D3300004460E4614D0402D12D0002D40F00A8134
:10D340004F78092F00F20681DFE817F00B01340156
:10D35000040123010401860016000401F300A20069
:10D36000D4F8D432AE33314654F823309B6820468B
:10D3700002B0BDE8F04118470023ADF806304B88F5
:10D380001A0A013A062A37D8DFE802F0041C2936C7
:10D3900036515B00D0F8B4321B68207C0DF10601D9
:10D3A0009847F288002A00F00181BDF806301BB3CF
:10D3B0009A4228BF1A46ADF806200146204600F0E2
:10D3C000DFF91CE0027CD0F8B83232B99B6A0DF16B
:10D3D0000600984702234370E3E7DB6AF7E7DBB216
:10D3E000052B09D8DFE803F0030F13171B1FD0F834
:10D3F000B4325B68002BD0D12046FFF787FF284668
:10D4000002B0BDE8F081D0F8B4329B68F2E7D0F802
:10D41000B432DB68EEE7D0F8B4321B69EAE7D0F843
:10D42000B4325B69E6E7D0F8B4329B69E2E7037C8B
:10D43000002BE1D1D0F8B8320DF106005B6B9847B4
:10D44000AFE7037C002BD7D1D0F8B8320DF106003E
:10D450001B6B98470723BEE78B88002BCCD1CB886A
:10D46000002BC9D14E887F2EC6D890F89C32032B52
:10D47000C2D0F1B280F89E1201F0D0FA204600F03E
:10D480009CF91EB1022384F89C32B8E70123FAE725
:10D490008E784E4F012E3E7003D9FFF737FF0325DC
:10D4A000ADE790F89C32022B5FFA83F809D0B8F10F
:10D4B000030F18D0FFF72AFF39782046FFF7D3FD76
:10D4C000EDE7002E72D001214160FFF7C5FD054652
:10D4D000204625B1FFF71AFF84F89C828FE700F001
:10D4E0006CF90323CFE75EB9022380F89C324660D3
:10D4F0003146FFF7B8FD204600F05FF935467EE77C
:10D500004168012952D0C9B2FFF7ADFD3978616099
:10D510002046FFF7A1FD0646002847D02046FFF72A
:10D52000F5FE21792046FFF79EFD022384F89C3208
:10D53000E4E7CA88012A7FF45FAF90F89C120229C1
:10D54000CBB205D833B10146002341F8083F35E797
:10D55000032B04D02046FFF7D9FE00254FE7011D1D
:10D560002CE790F89C32013B022BF3D8CB88022B9E
:10D570007FF442AF0123C360D0F8A4320BB1032380
:10D58000C360022204F10C01204600F0F9F83D4688
:10D5900035E74B88012B02D1C4F8A43206E0022BF8
:10D5A0007FF42AAF8B881B0A80F8A032204600F057
:10D5B00004F924E790F89C32013B022BCAD84B882F
:10D5C000012B7FF41CAF0023E6E700BF540C0020C2
:10D5D00070B50B7803F06002402A04460E4601D075
:10D5E0005B061FD494F89C32013B022B1AD8317988
:10D5F0000129204617D8FFF785FE88B9D4F8B8323C
:10D600009B686BB1C4F8D402314620469847054662
:10D61000F3881BB915B9204600F0CFF8284670BD35
:10D620000325F5E72046FFF771FE0025F6E770B504
:10D630000B788A880E7903F06003202B04460D4690
:10D6400053D0402B51D063BB4B78012B3BD0032BE5
:10D6500020D033BB90F89C32022BD9B261D0032981
:10D660001FD106F00F0312F0800F4FF0140202FBDF
:10D67000030365D09B8CA3B106F07F05013505EB54
:10D68000850500EB850516F07F0365D12B6002222E
:10D69000294651E090F89C32022BDAB237D0032AA7
:10D6A00003D02046FFF732FE0BE04B8833B97106FA
:10D6B00004D0EB8813B9314601F09EF9204600F002
:10D6C0007CF8002070BD90F89C32022BDAB21ED09C
:10D6D000032AE6D14B88002BF3D1730602D03146E2
:10D6E00001F093F9204600F068F831462046FFF734
:10D6F0000BFE0028E5D1D4F8B832C4F8D4029B68F8
:10D70000002BDED029462046BDE87040184772063F
:10D71000C7D0314601F070F98021204601F06CF944
:10D72000CFE77106BDD113064CBF00F1140100F51F
:10D73000AA7100230B600222204600F021F8C0E706
:10D74000B3F86431002BACD006F07F05142303FB43
:10D75000050505F5AA7596E73146204601F024F93E
:10D7600008B1012392E7286091E70B7803704B78AA
:10D7700043704B8843808B888380CB88C3807047FD
:10D7800010B513460222C0E90633C0F894220A46B7
:10D79000002101F04CF9002010BD08B513460A46DF
:10D7A000002101F044F9002008BD08B513460A46DF
:10D7B000002101F045F9002008BD08B5042200232E
:10D7C000C0F8942219461A4601F031F9002008BD2C
:10D7D00008B505220023C0F8942219461A4601F024
:10D7E0002FF9002008BD10B58371012301608280EC
:10D7F000C37110BD10B5818804460068FDF730FC88
:10D80000A379012818BF83F00103E37110BDC0792B
:10D81000B0FA80F04009704770B50C4615460646D0
:10D82000294600222046FDF721FCB088FCF77EFF48
:10D83000294620460122BDE87040FDF717BCF8B527
:10D8400004460D4600680121264600F037F920689D
:10D8500000F01AF9294656F80C0B00F01EF90025C5
:10D860001827EAB22068002100F03CF907FB05F315
:10D870002068F158013500F0FAF8042DF1D10022AA
:10D880002068114600F02EF92089FCF74FFF206830
:10D89000BDE8F84000F0F8B838B5094D044601225B
:10D8A0004FF400412846FDF7E1FBE088FCF73EFF1E
:10D8B00028460022BDE838404FF40041FDF7D6BBB2
:10D8C0000000024038B50446154DFFF7E5FF20463D
:10D8D0000121FFF7B4FF294620460822FFF79CFFED
:10D8E00029462046A5F580651022FFF795FF2946B9
:10D8F00020464022FFF790FF294620468022FFF76E
:10D900008BFF294620464FF48072FFF785FF29469A
:10D9100020464FF48062BDE83840FFF77DBF00BF6E
:10D920000004024030B590F85630DB00DBB221F045
:10D930000F0243EA011185B0C9B21A4341F0040352
:10D940008DF80E306423009342F004058DF80D200D
:10D950008DF80F100423B0F854108DF80C5003AA62
:10D96000FDF70EFD05B030BD30B590F85630DB0048
:10D97000DBB221F00F0243EA011185B0C9B21A43AC
:10D9800041F005038DF80E306423009342F0050545
:10D9900041F0010142F001028DF80D208DF80F10C9
:10D9A0000423B0F854108DF80C5003AAFDF7E8FCDE
:10D9B00005B030BD38B5044615465422F4F788F852
:10D9C000A4F854500025A4F85650A4F8585084F8F0
:10D9D0005A503220FCF7AAFE30212046FFF7A2FF62
:10D9E0000520FCF7A3FE30212046FFF79BFF012016
:10D9F000FCF79CFE30212046FFF794FF0A20FCF73D
:10DA000095FE20212046FFF78DFF0A20FCF78EFEB1
:10DA100028212046FFF786FF0120FCF787FE08211A
:10DA20002046FFF77FFF0120FCF780FE0121204602
:10DA3000FFF778FF0120FCF779FE0120FCF776FE66
:10DA400006212046FFF76EFF0120FCF76FFE0C2138
:10DA50002046FFF767FF0120FCF768FE4FF0012327
:10DA600084F85750A365A4F85C50204638BD38B5FB
:10DA700005464C1E14F8011F19B12846FFF774FF24
:10DA8000F8E738BDFFF770BF08B50121FFF74AFF7F
:10DA9000BDE808400120FCF749BE1FB5642380F8AB
:10DAA00056100093C9008DF80F100123B0F85410E0
:10DAB0000DF10F02FDF764FC04B010BD38B590F80D
:10DAC00058300D4643EA810390F8571043EA41036A
:10DAD000044643F00803D9B2FFF724FF84F85B50F3
:10DAE00038BD0000531EDBB2022B70B515469ABF3D
:10DAF000094AD35C00230B4463F07F0304460E46BF
:10DB0000D9B2FFF70FFF0120FCF710FE84F85C602C
:10DB100084F85D5070BD00BF300B010838B5044675
:10DB20000C480378BFF35B8FDB070D460AD401F086
:10DB300079FD38B108482A462146FFF73BFF0548E2
:10DB400001F090FD044838BD024801F087FD01F066
:10DB500001F800BF580C00205C0C00207047704793
:10DB60000020704770477047002070474268137864
:10DB700083F0010313707047436801221A707047E5
:10DB800090F8203083F0010380F82030704742681D
:10DB9000138801331380704742681388013B138058
:10DBA000704790F82000704790F8203083F0010310
:10DBB00080F82030704742681378632B9CBF013394
:10DBC00013707047426813780BB1013B13707047B4
:10DBD00090F820007047000008B5034650B1064A8F
:10DBE000904201D901F02AFE18205843BDE80840B0
:10DBF00001F05ABD08BD00BF5555550518B1182391
:10DC0000594300F0A5BF704700F1080373B50360E6
:10DC1000D1E900530446EE181DB916B10C4801F0C5
:10DC20001DFE0F2B019307D9002201A9204601F008
:10DC300021FF019B2060A36032462946206801F045
:10DC40006DFF019B226863600021D15402B070BD5A
:10DC50003807010810B5044B044640F8083B01F0B2
:10DC60002DFF204610BD00BFFC0A010810B5044678
:10DC7000FFF7F0FF2046242100F06AFF204610BD88
:10DC800010B5044B044640F8083B01F017FF20464E
:10DC900010BD00BFD80A010810B50446FFF7F0FF19
:10DCA0002046242100F054FF204610BD0B4600F111
:10DCB0000802026070B553F8084B9C420FD11C4615
:10DCC00001F1180554F8046B42F8046BAC42F9D129
:10DCD0004A680B60002342604B600B7270BD8A681B
:10DCE00004608260F4E770B504460E461546B442FF
:10DCF00009D021462846FFF7D9FF204601F0DEFE75
:10DD000018341835F3E7284670BD000010B5044BF1
:10DD1000044640F8083B01F0D1FE204610BD00BF8C
:10DD2000B40A010810B50446FFF7F0FF204624218D
:10DD300000F00EFF204610BD10B5044B044640F81D
:10DD4000083B01F0BBFE204610BD00BFB40A01082D
:10DD500010B50446FFF7F0FF2046242100F0F8FE3E
:10DD6000204610BDF8B581EAE174A4EBE174CF0F51
:10DD700006462346012542F20F7142F21072092B2A
:10DD800002D9632B20D8013506F1080379193360D5
:10DD90002D22304601F09AFE3368194AD9190D44F4
:10DDA0004FF0640E632C1CD9B4FBFEFC0EFB1C4030
:10DDB000644602EB400C12F810009CF801C005F814
:10DDC00001CC05F8020DEDE7B3F57A7F01D20235FB
:10DDD000DAE78B4201D80335D6E70435B3FBF2F31B
:10DDE000CDE7092C85BF064A02EB44003034407869
:10DDF00085BF12F814204870DC55DA553046F8BD5E
:10DE00006B0B0108002908DBD0E903239B1AB1EB57
:10DE1000A30F02D252F82100704700207047D0E9CA
:10DE200003239B1AB1EBA30F10B54FEAA3040AD347
:10DE3000D0E900239B1A04EBA303994203D2091BE8
:10DE400052F8210010BD0020FCE7000000F108039B
:10DE500073B5044603600D46E1B10846F4F7D0FA05
:10DE60000F2805EB0006019007D9002201A92046E2
:10DE700001F000FE019B2060A36020683246294625
:10DE800001F056FE019B2268636000212046D154B8
:10DE900002B070BD014801F0E1FC00BF3807010885
:10DEA00070B553681546CA688EB0C3F113039B1A48
:10DEB00004AA02920022934204460E4603928DF871
:10DEC000102006DD2021009102A8114601F090FEED
:10DED00005E004D0144908AAFFF7B8FF1CE006F1DA
:10DEE000080108A8FFF790FE02A908A801F0E6FFC4
:10DEF00007E008A801F0E2FD02A801F0DFFD00F054
:10DF000029FE294608A801F0D9FF01462046FFF75F
:10DF1000CDFE08A801F0D2FD02A801F0CFFD2046F9
:10DF20000EB070BDE5E7E7E7330B010830B54B688D
:10DF300004460D4618780D490D4B89B0002808BFDE
:10DF4000194601AA02A8FFF781FF02AA2946204626
:10DF5000FFF7A6FF04E002A801F0B0FD00F0FAFD13
:10DF600002A801F0ABFD204609B030BD390B010815
:10DF70003D0B010830B54B6804460D4618780D4935
:10DF80000D4B89B0002808BF194601AA02A8FFF767
:10DF90005DFF02AA29462046FFF782FF04E002A89F
:10DFA00001F08CFD00F0D6FD02A801F087FD2046AF
:10DFB00009B030BD410B0108450B010870B553682D
:10DFC0001546CA688EB0C3F113039B1A04AA0292C5
:10DFD0000022934204460E4603928DF8102006DD7F
:10DFE0002021009102A8114601F002FE05E004D0B4
:10DFF000144908AAFFF72AFF1CE006F1080108A847
:10E00000FFF702FE02A908A801F058FF07E008A8E0
:10E0100001F054FD02A801F051FD00F09BFD2946DE
:10E0200008A801F04BFF01462046FFF73FFE08A875
:10E0300001F044FD02A801F041FD20460EB070BD84
:10E04000E5E7E7E7330B010870B50C464B6894F839
:10E05000206019888CB00546684686B1FFF782FEBD
:10E06000194A0021684601F0E1FE014606A8FFF7C3
:10E070001DFE024621462846FFF7A0FF0FE0FFF7EE
:10E0800071FE124A3146684601F0D0FE014606A8EC
:10E09000FFF70CFE024621462846FFF78FFF06A831
:10E0A00001F00CFD684601F009FD28460CB070BD7A
:10E0B00006A801F003FDFFE7684601F0FFFC00F051
:10E0C00049FDF5E7F8E700BF490B0108A30D01087A
:10E0D00070B553681546CA688EB0C3F113039B1A16
:10E0E00004AA02920022934204460E4603928DF83F
:10E0F000102006DD2021009102A8114601F078FDD4
:10E1000005E004D0144908AAFFF7A0FE1CE006F1C0
:10E11000080108A8FFF778FD02A908A801F0CEFEC3
:10E1200007E008A801F0CAFC02A801F0C7FC00F053
:10E1300011FD294608A801F0C1FE01462046FFF75F
:10E14000B5FD08A801F0BAFC02A801F0B7FC204612
:10E150000EB070BDE5E7E7E7330B010870B50C467C
:10E160004B6894F8206019788CB00546684686B1F3
:10E17000FFF7F8FD194A0021684601F057FE0146F5
:10E1800006A8FFF793FD024621462846FFF7A0FFA9
:10E190000FE0FFF7E7FD124A3146684601F046FE00
:10E1A000014606A8FFF782FD024621462846FFF7F2
:10E1B0008FFF06A801F082FC684601F07FFC28462C
:10E1C0000CB070BD06A801F079FCFFE7684601F0CD
:10E1D00075FC00F0BFFCF5E7F8E700BF4C0B010849
:10E1E0004D0B010810B504461046D4E900239B1AD4
:10E1F0000A4A0B4CDB105343E21A8A4201D201F067
:10E2000045FB994238BF19465B1804D2A34228BF88
:10E210002346184610BD2046FCE700BFABAAAAAAB9
:10E22000555555052DE9F84F0E46934601211F4AD5
:10E230000546FFF7D7FFD5E9008A0746FFF7CCFC74
:10E24000A6EB08098144044659464846FFF7DCFC22
:10E25000224631464046FFF746FD514600F118027E
:10E260003046FFF740FDAB681149A3EB0803DB1014
:10E27000064659434046FFF7C1FC1820C5E9004651
:10E2800000FB0744AC60BDE8F88F00F02DFD14B929
:10E29000484601F013FC39462046FFF7AFFC01F079
:10E2A00089F900F05FFD00F055FC00BF620701082E
:10E2B000ABAAAAAA2DE9F74F0E4693460121204AA0
:10E2C0000546FFF78FFFD5E9008A0746FFF784FC74
:10E2D000A6EB08098144044601AA59464846FFF7BF
:10E2E000B5FD224631464046FFF7FDFC514600F1A0
:10E2F00018023046FFF7F7FCAB681249A3EB08039E
:10E30000DB10064659434046FFF778FC1820C5E964
:10E31000004600FB0744AC6003B0BDE8F08F00F09E
:10E32000E3FC14B9484601F0C9FB39462046FFF723
:10E3300065FC01F03FF900F015FD00F00BFC00BF9B
:10E3400062070108ABAAAAAA2DE9F04FD1E900267D
:10E350000023B21AC0E900338360D1E903639E1B36
:10E36000B6105E4B06EBA2069E428BB004460D46ED
:10E3700003D95B4801F08AFA9CE0B6B13046FFF75A
:10E380002BFC02460746D4E90001FFF7ACFC2068ED
:10E39000A168544B091AC9105943FFF72FFC1822E2
:10E3A000C4E9007702FB0676A660D5E90367B742A9
:10E3B000334619D0196804A81C310436FFF724FC31
:10E3C000D4E90103984209D004A9FFF71DFC636852
:10E3D0001833636004A801F071FBE8E7014604AA62
:10E3E0002046FFF71FFFF5E76B68D5F80080DFF8E0
:10E3F000F8900193019B434542D058F8041B0B68E9
:10E4000004A89B699847D4E901639E420AD004A9F5
:10E410003046FFF74BFC63681833636004A801F0D3
:10E420004DFBE7E74A4601212046FFF7DBFED4E932
:10E43000007AF31B02900393FFF7CEFB8346F01B99
:10E4400004A95844FFF732FC31465A463846FFF7D4
:10E450004AFC514600F118023046FFF744FCA1681F
:10E46000204AC91BC910064651433846FFF7C6FB70
:10E47000029B182000FB03B3C4E900B6A360CDE7FC
:10E48000AB6953B1D4E9010398420AD0174904AAF1
:10E49000FFF7DCFC63681833636020460BB0BDE80F
:10E4A000F08F0146114A2046FFF704FFF5E704A864
:10E4B00001F004FBD4E90056AE4205D0284601F035
:10E4C000FDFA1835F8E7F2E72068A36805491B1A3A
:10E4D000DB105943FFF792FB00F03CFB5555550507
:10E4E000500B0108ABAAAAAA62070108600B010839
:10E4F0000246D0E90330C01AD2E900135B1A9B1020
:10E5000003EBA0009369002B18BF0130704770B572
:10E510000D46044641682846FFF774FC616830B137
:10E520002846FFF76FFC0023A060636070BD28469B
:10E53000FFF775FC40B161682846FFF770FC03687F
:10E54000BDE870409B681847A3689B69002BEDD01D
:10E55000C4E90103EAE770B54668044608460D467B
:10E56000FFF7C6FF86421AD231462846FFF757FC0E
:10E5700088B161682846FFF752FC03685B699847D9
:10E5800048B161682846FFF74AFC0368BDE870405F
:10E59000DB680121184728466668FFF7A9FF0138A4
:10E5A00086423CBF0136666070BD70B50D4641685D
:10E5B0000029044618DD2846FFF731FC88B1616860
:10E5C0002846FFF72CFC03685B69984748B16168EF
:10E5D0002846FFF724FC0368BDE870401B69012151
:10E5E00018476368013B636070BD012905D00229AB
:10E5F00006D041B98168FFF7AEBF8168FFF7D5BF8C
:10E600008168FFF784BF704770B5D0E900560446B3
:10E61000AE4204D0284601F051FA1835F8E72068D8
:10E6200018B1A168091A00F093FA204670BD0000E5
:10E630002DE9F04F4468DFF820B1634203F0030393
:10E6400004F0030858BFC3F10008002CB8BF03341E
:10E650008DB005460F4624F0030400265FFA86F9C4
:10E6600028684A460021FFF73DFAB04526D12868C0
:10E670007E21FFF707FA4A4628680121FFF732FAA0
:10E68000394603A8FFF760FE3846FFF731FFA04286
:10E6900055D9039A18236343D11808A8069052F855
:10E6A00003904B6809EB030AB9F1000F0BD1BAF1E3
:10E6B000000F08D0294801F0D1F848E0284928681F
:10E6C000FFF7D5F9D7E70F2B029307D9002202A94C
:10E6D00006A801F0CFF9029B0690089306985246CF
:10E6E000494601F01BFA029B069A07930020D0547A
:10E6F000079913290CD9092300930A465B46014662
:10E7000006A801F0CDFA06992868FFF7B0F908E0ED
:10E71000202300930246C1F1130306A801F068FA12
:10E72000F1E706A801F0CAF903A80136FFF76CFF6C
:10E73000042E04F1010491D10DB0BDE8F08F094918
:10E740002868FFF794F9EFE706A801F0B7F903A8E6
:10E75000FFF75AFF00F0FEF9880D0108380701089D
:10E76000A40D0108920D01088168FFF761BF70B523
:10E770000446818B80690122FCF778FCA088FBF7B6
:10E78000D5FF002635462388B3420FDD6088FBF7AE
:10E79000CDFF6069FCF784F861886069FCF7F6F8E2
:10E7A0006069FCF746F901360544ECE70022A18BCD
:10E7B000A069FCF75BFC2388B5FBF3F5A368258211
:10E7C0001A88ADB26423AD1A5D43E3681B889B1AB7
:10E7D00095FBF3F5A57470BD2DE9F0411D46BDF81C
:10E7E000183003800A2343804FF4FA730446838071
:10E7F00002200F46164600F057FF4FF00008A0F821
:10E800000080A060022000F04FFF4FF6FF730380EE
:10E81000E060C4E90576A4F8108084F81280A5832E
:10E820002046BDE8F08190F91200704710B504460B
:10E83000FFF79DFFA368228A1A8010BD10B5044619
:10E84000FFF795FFE368228A1A8010BDC0E9021223
:10E85000704770B50546FBF763FFAE68EC88801B18
:10E86000844205D3FBF75CFF3444241AA0B270BD88
:10E870000020FCE738B504460D4679B9437B012BEF
:10E880000BD1FFF7E6FF054638B9227B82F0010283
:10E89000A1882068FCF7EAFB657338BD0129FCD12B
:10E8A000437B002BF9D1FBF73BFF227BA060EFE716
:10E8B00038B50D469DF810108280037300220123A5
:10E8C00004460560C2808260437309B9FFF7D2FF36
:10E8D000204638BD01737047437B33B9027B82F019
:10E8E000010281880068FCF7C1BB012B01D1027BCA
:10E8F000F7E7704700F2C441D0F80805FEF7BCBB4B
:10E90000242303FB0103D0F80805D3F88C22FEF77B
:10E91000E3BB242303FB0103D0F80805DA6CFEF700
:10E9200010BCD0F80805FEF7A6BCC368022B10B5D2
:10E93000044601D0FAF7C0FCD4F808050121FEF71F
:10E9400082FCD4F80805BDE81040FEF74DBC00007D
:10E9500010B50446D0F80805FEF778FC2268D2F816
:10E96000003E43F00103C2F8003E236A23B1034A8C
:10E97000136943F00603136110BD00BF00ED00E012
:10E98000D0F80805FEF76CBCD0F80805FEF794BC7B
:10E99000D0F80805FEF77CBCD0F80805FEF7A0BC4F
:10E9A000D0F80805FEF79EBC11F0800FD0F8C832F1
:10E9B0004FF024021BBF01F07F0102FB013102FB7B
:10E9C000013191F83E0008BF91F87E0270470000C7
:10E9D00003289ABF014B185C03207047A60D01085D
:10E9E00010B51446D0F8C8021A462346FCF7B4FD09
:10E9F000BDE81040FFF7ECBF08B5D0F8C802FCF73F
:10EA000027FEBDE80840FFF7E3BF08B5D0F8C8020D
:10EA1000FCF756FEBDE80840FFF7DABF08B5D0F8AE
:10EA2000C802FCF785FDBDE80840FFF7D1BF08B577
:10EA3000D0F8C802FCF7ECFDBDE80840FFF7C8BFFE
:10EA400008B5D0F8C802FCF7BFFDBDE80840FFF7E5
:10EA5000BFBF000070B5036884B000249E690394B2
:10EA6000102315460293CDE900446B461268B04767
:10EA70009DF8043003F00603062B03BF009B2B60B8
:10EA80000120204604B070BD0098904214BF0120C0
:10EA90000620704710B5034B0360044600F0B4FE37
:10EAA000204610BDE40D010810B5054B0360044677
:10EAB00000F0AAFE2046082100F04AF8204610BDCA
:10EAC000E40D01082DE9F041069F0899099E8F4247
:10EAD000044690461D460CD02946204600F098FE7C
:10EAE00020B10123376086F80480B3710020BDE8AF
:10EAF000F081079900F08CFE0028EDD086F80580A3
:10EB00000020BDE8F08100BF38B515461C4600F076
:10EB10007FFE00B938BD082206232560E26023711C
:10EB200038BD00BF2DE9F041064617461D460C468C
:10EB300000F06EFE48B9032D07D823683A463146E7
:10EB400020465B69BDE8F0411847BDE8F08100BF91
:10EB500001F0D6B91EB400F08FF81EBCF2F76EFAC1
:10EB6000F0B50278472A83B00C461D4619D0002321
:10EB7000264E0193336830469B68984778B1019BD5
:10EB80001B68019302272368314620461E6901AAAB
:10EB90000123B04718BB0746384603B0F0BD012734
:10EBA000F1E743784E2BE2D18378552BDFD1C37840
:10EBB000432BDCD10379462B1BD00379432BD6D1D1
:10EBC00043792B2BD3D183792B2BD0D1C379012B34
:10EBD000CDD809D050F8206C58300190CAE7019B7D
:10EBE0002B60384603B0F0BD50F8200C50F8786C1C
:10EBF000F3E743794F2BE0D18379522BDDD1C379F1
:10EC0000002BDAD1024E0193B4E700BF340E0108A5
:10EC10002C0E010810B5044600F002F9224612F845
:10EC20002039472B04D0836823BB8260012010BDAC
:10EC300063784E2BF7D1A378552BF4D1E378432B8F
:10EC4000F1D12379432BEED163792B2BEBD1A3792F
:10EC50002B2BE8D1E379012BE5D854F8043C0133A0
:10EC6000012B44F8043CE1D1836844F8083C8260FD
:10EC7000012010BD00F00EFC08B500F0D1F883684B
:10EC800083B393F82020472A04D00022826003F146
:10EC9000200008BD93F821204E2AF6D193F82220B7
:10ECA000552AF2D193F82320432AEED193F8242059
:10ECB000432AEAD193F825202B2AE6D193F826207F
:10ECC0002B2AE2D193F82720012ADED8DA69013A0B
:10ECD000DA61002ADBD19969816000229A6103F12F
:10ECE000200008BD00F0D6FB38B5044600F098F8C7
:10ECF0002246056812F82039472B03D085BB0260F5
:10ED0000284638BD63784E2BF8D1A378552BF5D122
:10ED1000E378432BF2D12379432BEFD163792B2B6B
:10ED2000ECD1A3792B2BE9D1E379012BE6D854F868
:10ED30000C3C002B11DB013344F80C3C4368013BD5
:10ED40004360954218BF44F8105C656A18BF0260C2
:10ED50002046F1F7B5FD284638BDC3F10103EBE7C6
:10ED600000F098FB08B500F057F803687BB393F800
:10ED70002020472A07D00022026003F12000BDE8CE
:10ED80000840F1F79FBD93F821204E2AF3D193F864
:10ED90002220552AEFD193F82320432AEBD193F870
:10EDA0002420432AE7D193F825202B2AE3D193F896
:10EDB00026202B2ADFD193F82720012ADBD85A6995
:10EDC000002A05DB013A08D0511C0ED05A6108BD5B
:10EDD0000132FBD119690160F8E71A69026003F199
:10EDE0002000BDE80840F1F76DBD00F053FB00BF07
:10EDF000704700BF704700BF00487047080E010809
:10EE000000487047180E010810B504210446FFF7AA
:10EE10009FFE204610BD00BF00487047C81100206B
:10EE200000487047C8110020502870B51DD0844696
:10EE300000F00F000C2855D8DFE800F00744260743
:10EE40001E545454542A22071E00104650F8046BD6
:10EE50004EB10CF07004102C08BF11460E441CF08B
:10EE6000800F18BF36681E6070BD033222F00300A9
:10EE700050F8046B1E6070BD104650F8086BE7E751
:10EE8000104630F9026BE3E7104630F8026BDFE71B
:10EE900000261046344610F8015B05F07F0E0EFA8E
:10EEA00004FE15F0800F46EA0E0604F10704F2D1C5
:10EEB0001F2CCDD86D06CBD54FF0FF3505FA04F4E5
:10EEC0002643C6E700261046344610F8015B05F0DD
:10EED0007F0E0EFA04FE2D0646EA0E0604F1070424
:10EEE000F3D4B5E7F2F79CFAFF2808B5034619D02A
:10EEF00003F07002302A084616D005D8202A09D11E
:10EF0000BDE8084001F0B7BA402A09D1BDE8084081
:10EF1000F2F774BA02D813F0600F03D0F2F780FA58
:10EF2000502AFBD1002008BDBDE8084001F0A0BA7E
:10EF3000F8B50C461546064608B1F2F75FFA2860A8
:10EF400014F8017BFF2F29D16860204610F8013B9F
:10EF50002B75FF2B33D0102300242B75224610F87D
:10EF6000011B01F07F039340090644EA030402F108
:10EF70000702F4D40444EC6010F8013B6B750024E4
:10EF8000224610F8011B01F07F0393401C430B063F
:10EF900002F10702F5D404442C61F8BD314638462D
:10EFA000FFF7A2FF224601462B1D3846FFF73CFF24
:10EFB0000446204610F8013B2B75FF2BCBD10023D4
:10EFC000EB60D9E72DE9F04F00F0030493B0002384
:10EFD000012C08938846174613D0022C08D13946D5
:10EFE0004046F2F7F5F940B9082013B0BDE8F08FBC
:10EFF000002C00F09480F2F713FA092013B0BDE85A
:10F00000F08F0DF1300A10F00804CDF800A000F0E8
:10F010009D8044F0020202920C910C22194638465F
:10F02000F1F77CFC3846F2F7EFF983460028D6D09A
:10F03000524601463846FFF77BFF394605469DF8A4
:10F040004400FFF751FF0DF12C0900230E901946E3
:10F05000CDF800900F223846F1F73AFC0B9B23F0D5
:10F0600001035E1E109B9D4237D29DF84540002152
:10F070002046FFF739FF2A46014609AB2046FFF735
:10F08000D3FE9DF84550044600212846FFF72CFF8B
:10F09000224601460AAB2846FFF7C6FE9DF84550BA
:10F0A000044600212846FFF71FFF224601464B4633
:10F0B0002846FFF7B9FE00240546224615F8011B35
:10F0C00001F07F0393401C430B0602F10702F5D4C5
:10F0D0000C9B099A1344B34219D9029BD80730D527
:10F0E0000024039400231946CDF8009038460D22E1
:10F0F000089DF1F7EDFB039BC8F830300B9BC8F877
:10F100002CB0C8E909540620C8F820306DE70A9AE7
:10F110001344B3426ED8109BAB42A6D8DDE702077A
:10F120003FF55DAF012302930DF1300A0023CDF8C6
:10F1300000A00C2219463846CDF83080F1F7EEFBDE
:10F1400070E7029B1A0752D500F0A4F90D6A234616
:10F150000D2221463846F1F7BBFB0C9B9D4202D0A5
:10F1600002230293E2E72346CDF800A021460C22B9
:10F170003846CDF83080F1F7D1FBD8F83030039322
:10F18000ABB3D8E90A4B0DF12C09002C4EDB03255B
:10F1900000231A461946CDF800903846CDF82C8049
:10F1A000F1F7BCFB002319460122CDF80090384648
:10F1B0000B94F1F7B3FB002319460F22CDF8009012
:10F1C0003846F1F785FB0B9A0399CDF8009002F0D1
:10F1D00001020A4300230B9238460F221946F1F729
:10F1E0009DFB022D1DD0072013B0BDE8F08F4046D7
:10F1F00000F054FF0B9B002B3FF4F1AE0D9A13442B
:10F200000393002C38D1002B3FF4E9AE029BDD07BD
:10F210003FF5E5AE029B1B0740F123810024022548
:10F22000B6E74046FFF7F6FC0720DEE66FF0404306
:10F230001B1B1E46524659463846FFF779FE9DF87D
:10F2400044003946FFF750FE0E9005460F9850F8DF
:10F25000263000EB860033B10246002352F8041F2B
:10F2600001330029FAD1C8E90A350423C8F834006B
:10F27000C8F8303003258BE7109E039B013C2644E1
:10F28000002B3FF4ACAE029B002E00F0E28013F0A6
:10F290000803049300F0C980472388F800304E2308
:10F2A00088F80130552388F80230432388F803306A
:10F2B000462388F804304F2388F80530522388F815
:10F2C0000630002388F807300023CDF818B00597E2
:10F2D0009B46CDF81CA00024224616F8011B01F025
:10F2E0007F039340080644EA030402F10702F4D4C2
:10F2F0001F2A05D84B0603D5012393405B421C43CC
:10F30000002530462A4610F8011B01F07F03934088
:10F310000F0645EA030502F10702F4D41F2A05D8B7
:10F32000490603D5012393405B421D43002C37D08F
:10F3300039DCB8F1000F02D0049B002B50D06FF0E5
:10F34000404A0F9BAAEB040A53F82A30BBB1002DA8
:10F3500075D02E44BFE7A3005B420F9A0E991A4462
:10F360004B46FFF761FD0B9949B1B8F1000FEED0A4
:10F3700008AB00224046FFF7F3FB0028E7D0029BD2
:10F38000DDF81CA0D907DDE9057B3FF5ABAE049B9A
:10F39000002B3FF4FAAE002CBFF6F9AE00F088F86F
:10F3A0004FF0010BD3E79DF84400FF2831D000F067
:10F3B0000703042B3FF61FAE01A252F823F000BF53
:10F3C00057F30008F7EF0008DBF3000857F30008D5
:10F3D000D5F30008E3005B42BFE763005B42BCE794
:10F3E0006FF0404A0F9F089B0B93AAEB040A57F853
:10F3F0002A1007EB8A0719B90DE057F8041F51B11D
:10F4000039444B4600224046FFF7AAFB0028F4D0BF
:10F410009DE70023A1E7029BDA075646DDE9057B5D
:10F42000DDF81CA03FF55EAE04E798F80730012B2D
:10F430000CBF58F8203C08F15803089344E75B469A
:10F44000059F002B3FF4CBAD029BDB073FF5C7AD1B
:10F45000E4E6DE073FF5C3AD029B13F008047FF43A
:10F46000DDAE022594E6FFF73FFC6DE608B5804768
:10F47000F1F7D6FFFFF738FCF1F7D2FF0C4605464F
:10F48000FFF770FC013402D1284600F017FEFFF7A9
:10F4900061FB00BF08B5034B1868BFF35B8FFFF734
:10F4A000E5FF00BFC009002008B58047FFF7F2FF65
:10F4B00008B5034B1868BFF35B8FFFF7F5FF00BF7C
:10F4C000BC090020024B1868BFF35B8F704700BF78
:10F4D000C0090020024B1868BFF35B8F704700BF64
:10F4E000BC090020012810B51AD8BFF35B8FA1F129
:10F4F000280353E8002F013A43E800200028F8D100
:10F50000BFF35B8F5AB951F81C3C01F158040BB1A1
:10F51000204698472046BDE8104000F07DBD10BD54
:10F5200051F8140CFFF7A2FF38B5002540E91E1270
:10F5300040F8805C0446FFF7CDFF44F8700CFFF7FD
:10F54000C1FF43222B23472104F8552C04F8542CE7
:10F5500004F8533C04F8523C4E22552304F8581C3E
:10F5600004F8515C054904F8572C04F8563C44F85B
:10F570006C0C44F8501CA4F1800038BDE5F4000880
:10F5800070B504460D461646FFF74AFC4368013342
:10F590003246294643602046FFF7C6FF0446012352
:10F5A00044F8283B2046F1F737FD2046FFF79CFB47
:10F5B000FFF770FF10B5FFF733FCD0E900420132CE
:10F5C000426064B194F82020472A0AD000220260E9
:10F5D00020342046F1F744FD2046FFF785FBFFF776
:10F5E00059FF94F821204E2AF0D194F82220552A70
:10F5F000ECD194F82320432AE8D194F82420432A1C
:10F60000E4D194F825202B2AE0D194F826202B2A47
:10F61000DCD194F82720012AD8D86269524262616D
:10F62000D6E700BF0368DB0705D443782BB9012375
:10F630004370184670470020704710B5042000F052
:10F64000D3FC044600F02AF8024A03492046FFF79B
:10F6500097FF00BF6DF60008CC0E01080023437031
:10F66000704700BF01230360704700BF10B5034B14
:10F6700003600446FFF7BCFB204610BD040F0108E1
:10F6800010B5054B03600446FFF7B2FB204604218A
:10F69000FFF75EFA204610BD040F0108014B03601E
:10F6A000704700BF040F0108012838BF012010B5C2
:10F6B00004462046F1F702FF00B110BD00F070FDD6
:10F6C00008B18047F5E7042000F08EFC024B034AA6
:10F6D00003490360FFF754FFD8100108D1FE00086A
:10F6E000B410010808B5FFF7D5FE00BF10B5034BF5
:10F6F00003600446FFF7CEF9204610BD4C0F010809
:10F7000010B5054B03600446FFF7C4F920460C21F1
:10F71000FFF71EFA204610BD4C0F010870B582B0ED
:10F720000446069E96420D4609D0A06804680696D7
:10F73000246A2946A44602B0BDE8704060471946D5
:10F740000192009300F064F8DDE900320028ECD06B
:10F75000062002B070BD00BF2DE9F04F0D4681B00C
:10F760001946DDE90A7ADDE90C981C4606469346FF
:10F7700000F04EF880B94F4527D0B06823460468A2
:10F78000CDE90C98CDE90A7AE4695A462946A4469F
:10F7900001B0BDE8F04F6047002DC8F8007088F850
:10F7A00004B00CDB3D44A9450CBF4FF006094FF0F7
:10F7B000010988F80690002001B0BDE8F08F0235FD
:10F7C000F9D1012388F80630F5E75146304600F0BC
:10F7D0001FF80028D1D088F805B0ECE72DE9F041FA
:10F7E00006460F4614461D46FFF78EF948B9B06825
:10F7F000016822468C692B463946A446BDE8F04193
:10F800006047BDE8F08100BF704700BF002070472F
:10F81000814211D008B5406803782A2B0AD0496884
:10F820000B782A2B08BF0131F2F76EFCB0FA80F09A
:10F83000400908BD002008BD0120704708B504201C
:10F8400000F0D2FB024B034A03490360FFF798FE26
:10F85000D8100108D1FE0008B410010810B5044604
:10F86000082000F0C1FB2146044600F06FFD054A68
:10F8700005492046FFF784FE204600F0CDFBFFF748
:10F8800069F900BFB5010108E410010810B504468C
:10F89000082000F0A9FB2146044600F097FD054A28
:10F8A00005492046FFF76CFE204600F0B5FBFFF748
:10F8B00051F900BFF5010108F01001080FB4F0B5CF
:10F8C00083B000AF07F1200454F8046B3046F2F720
:10F8D00097FD00F2072323F00703ADEB030D6D4600
:10F8E00000F500712346324628467C6000F06CF833
:10F8F000082000F079FB2946044600F071FD054A16
:10F9000005492046FFF73CFE204600F085FBFFF747
:10F9100021F900BF35020108FC100108F0B59DB0C7
:10F9200000AF0C1A06460F496922381DF2F7D0F8CD
:10F9300004F1700323F00703ADEB030D6D4668225D
:10F94000391D2846F2F7C4F82246314605F1680011
:10F950002C44F2F7BDF80023284684F86830FFF7FE
:10F960007DFF00BF880F01082DE9F84300AF84B088
:10F970006E4606F10C08DFF84890124DC646A5FB0E
:10F980000243DB0803EB830CA2EB4C0C1446092C5E
:10F9900019F80C200EF8012D1A46F0D8A8EB0E0825
:10F9A000884509D8C8F10C0142463144F2F790F875
:10F9B0004046BD46BDE8F8834FF0FF38F8E700BF8A
:10F9C000F40F0108CDCCCCCC2DE9F04115461278CE
:10F9D0004E1E07460644002A44D0B04245D219467E
:10F9E000044607E02A7804F8012B01352A78F2B1A1
:10F9F000B4423BD2252AF5D16A78732A1CD07A2AE0
:10FA000003D0252AEED10135EDE7AB78752BE9D18E
:10FA10008846204658F8042B311BFFF7A5FF002825
:10FA200024DDEA78033504444146002AE0D1E01B96
:10FA300000232370BDE8F08151F8042B137853B1F3
:10FA4000A64202D809E0A64208D004F8013B12F809
:10FA5000013F002BF7D10235C8E72646314638462C
:10FA6000FFF75CFF04461046E2E7044621463846AD
:10FA7000FFF754FF0868B0F1804F08B519D29042E3
:10FA800012D9B0EB420F4FEA42030DD2B3F1804FCF
:10FA900008D36FF040430B604FF08040BDE8084052
:10FAA000FFF702BE0B601846BDE808400130FFF7C3
:10FAB000FBBD0148FFF7EAFE00100108034653F8BA
:10FAC000080B984201D000F01BBA704730B583B0E4
:10FAD0000F290191044615460FD800680B463BB12B
:10FAE000012B12D01A462946F2F708F9019B20682B
:10FAF00063600022C25403B030BD002201A9FFF7A9
:10FB0000B9FF019B2060A360E9E70570019B2068B5
:10FB100063600022C25403B030BD00BF521A012AF4
:10FB200003D002B97047F1F7D3BF0B780370704769
:10FB3000521A012A03D002B97047F1F7C9BF0B78F6
:10FB4000037070472DE9F04F83B04768DDF830B09F
:10FB500081469A46ABEB02033B44019359F8083BBC
:10FB6000994501EB02060D4614BF82680F2201A9D8
:10FB70000446FFF77FFFBF1B80462DB1012D216892
:10FB800029D02A46F1F7A4FFBAF1000F0BD0BBF140
:10FB9000000F08D0BBF1010F08EB050022D0514641
:10FBA0005A46F1F795FF57B123685D44012F08EBE2
:10FBB000050003EB060111D03A46F1F789FF2068F2
:10FBC000814501D000F09CF9019BC4F80080A3603E
:10FBD00003B0BDE8F08F0B780370D5E79B5D08F8A4
:10FBE0000530ECE79AF8003008F80530DBE700BF95
:10FBF0002DE9F0411D460F4602F180434168013B6B
:10FC000082B05B1A9D429DF8208044D8044650F88B
:10FC1000083B834218BFA068A5EB02060E4408BF4C
:10FC20000F20B04223D302EB070CB1EB0C0C0DD02C
:10FC3000AA420BD03B44BCF1010F03EB050003EBE0
:10FC400002011ED06246F1F7DDFF236845B1012DA8
:10FC500003EB07001BD02A464146F2F74FF8236812
:10FC60006660002220469A5502B0BDE8F08100236C
:10FC7000009539462046FFF765FF2368002DEFD039
:10FC8000E5E79A5C5A552368002DE9D0DFE703F8D1
:10FC900007802368E4E70148FFF7F8FD50100108EA
:10FCA0002DE9F04F154685B042680E9E1F4605F1BE
:10FCB0008043013B9B1A9E4200F2B2800346A6EBB2
:10FCC000050B53F808AB9A4518BF836802EB0B0984
:10FCD00008BF0F234B45044688463DD36B18BA45F1
:10FCE0005144A2EB030302911FD963B1B5420AD07C
:10FCF0000AEB0802012B02EB060002EB050151D0D2
:10FD00001A46F1F77FFF36B1012E2BD0029832460A
:10FD10003946F1F7DDFE2368C4F80490002220463E
:10FD200003F8092005B0BDE8F08F52449742DCD8B3
:10FD300036B3B5421AD23BBB0AEB08031D44BB19CC
:10FD40009D4237D3012E0DD0002EE4D002983246CA
:10FD50003946F1F757FFDEE700963B462A46FFF7A4
:10FD6000F1FED8E73B780AF80830D4E7012E44D0FA
:10FD7000324639460AEB08000393F1F743FF039B31
:10FD8000002BC8D0B542C6D00AEB0802012B02EB0B
:10FD9000060002EB05010AD01A46F1F733FFB5421F
:10FDA000CAD3B8E7535D9355002EB4D0ACE7535D8A
:10FDB0009355F4E7BD420AD8012E07EB0B0126D07C
:10FDC000002EA8D002983246F1F782FEA3E7ED1B81
:10FDD000012D18D025B1029839462A46F1F712FFB5
:10FDE000029B721B012A03EB050003EB060113D0F3
:10FDF000002A90D0F1F76CFE8DE73A780AF80820D7
:10FE0000002BCCD0BEE73B780AF80830E8E717F8BB
:10FE10000B300AF808307EE71A469B5D53557AE7A7
:10FE20000148FFF733FD00BF8810010870B5054693
:10FE300082B010460C461646F2F7E2FA6B689C4216
:10FE400008D800903346002221462846FFF728FFB5
:10FE500002B070BD024903482246FFF72FFD00BFE4
:10FE60007010010818100108F0B54768044650F8F2
:10FE7000085B854218BFA36807EB020608BF0F2383
:10FE80009E4283B00DD832B1012A05EB070011D094
:10FE9000F1F71EFE2568666000232046AB5503B0CF
:10FEA000F0BD00920B46002239462046FFF74AFE7D
:10FEB0002568F0E70B78EB552568ECE708B5D1E944
:10FEC0000012FFF7D1FF08BD00487047A4100108D9
:10FED00010B5034B03600446FEF78AFF204610BDB1
:10FEE000D810010810B5054B03600446FEF780FFEB
:10FEF00020460421FEF72CFE204610BDD810010834
:10FF0000F1F7E4BA20494B6830B5A0F108046BB3AF
:10FF100050F8085C04EB050E734527D821D05A68C9
:10FF200001F1040C32B90FE0516803F1040C21B364
:10FF300013460A469645F7D304BFDEE9002159600F
:10FF4000DCF8003008BFAD181A6899188C4211D03F
:10FF50005B6840F8043CDCF8003040F8085C5C600A
:10FF600030BD1A685B682A4440F8082C40F8043C0D
:10FF70004C6030BD2A441A6030BD5B681A6899181D
:10FF80008C42E5D1F6E700BFD4110020154900F1FD
:10FF900008034868082B38BF0823A0B1073323F0B3
:10FFA0000703043102E0011D4068C8B102689342B2
:10FFB000F9D810B4D41A072C06D84368026010BCD4
:10FFC0000B60083070477047C218D0F804C0C2F800
:10FFD00004C0C450086810BC036008300A60704751
:10FFE000704700BFD411002010B500F180042046F6
:10FFF000F1F764FA034630B1802200211846F1F788
:020000040801F1
:100000007DFE803010BD2046FFF7C0FF034600286C
:10001000F2D1FFF73FFA00BF064A93688038984252
:1000200005D9D2681344984201D2FFF76BBFF1F7AC
:100030004DBA00BFD411002038B5084C4FF41E65EE
:100040002846E560F1F73AFAA06020B10023C0E944
:100050000053606038BDE060606038BDD41100209E
:100060000378472B01D00020704743784E2BFAD1FC
:100070008378552BF7D1C378432BF4D10379432BE5
:10008000F1D143792B2BEED183792B2BEBD1C07996
:1000900001288CBF00200120704700BF10B530B18F
:1000A0000446FEF721FE2046FFF7DAFF08B9FFF706
:1000B000F1F954F8140CFFF7D9F900BF2DE9F04F0E
:1000C00085B00246FFF7CCFF38B152E90674D2E999
:1000D0000C85D2F828A0002605E004460746012634
:1000E0000546804682461046FEF7FEFD0EB1FFF73C
:1000F000DFF93846FFF7D8F9FEF7F6FD0EB1FFF746
:10010000C9F9FEF789FE0768DFF888B097F827304D
:10011000012B0CBF3B6807F17803029328F003031F
:10012000019320374FF00009CA4520DDD5F8008043
:10013000B8F1000F00D0A84402AB00224146384677
:10014000FEF70EFD08B1FFF735FAD8F8003003903E
:1001500003AA40465946D3F810800123C047019BAB
:10016000002818BF064609F101091D44DCE746B125
:100170000420FFF739FF084B084A06490360FFF7E0
:10018000FFF92046FFF772F9FEF7ECFDFEF7EAFDF6
:10019000FEF7E0FC3C0E0108C00E0108F5ED00087A
:1001A000024B1868BFF35B8F704700BFE41100205B
:1001B0004068704710B543680C4A0D490446A3F1E6
:1001C0000C00904282B0216005D12046FEF710FE5F
:1001D000204602B010BD53F8042C511E002A43F8EB
:1001E000041CF2DC01A900F041F9EEE7E81100205F
:1001F0004811010810B543680C4A0D490446A3F1A3
:100200000C00904282B0216005D12046FEF7F0FD3F
:10021000204602B010BD53F8042C511E002A43F8AA
:10022000041CF2DC01A900F021F9EEE7E81100203E
:100230004811010810B543680C4A0D490446A3F162
:100240000C00904282B0216005D12046FEF7D0FD1F
:10025000204602B010BD53F8042C511E002A43F86A
:10026000041CF2DC01A900F001F9EEE7E81100201E
:100270004811010810B543680E4A0F490446A3F11E
:100280000C00904282B0216008D12046FEF7B0FDFC
:100290002046FFF735FE204602B010BD53F8042C6F
:1002A000511E002A43F8041CEFDC01A900F0DEF81F
:1002B000EBE700BFE81100204811010810B54368C2
:1002C0000E4A0F490446A3F10C00904282B021600F
:1002D00008D12046FEF78CFD2046FFF711FE204690
:1002E00002B010BD53F8042C511E002A43F8041C20
:1002F000EFDC01A900F0BAF8EBE700BFE81100203D
:100300004811010810B543680E4A0F490446A3F18D
:100310000C00904282B0216008D12046FEF768FDB3
:100320002046FFF7EDFD204602B010BD53F8042C27
:10033000511E002A43F8041CEFDC01A900F096F8D6
:10034000EBE700BFE811002048110108F0B51B4B96
:10035000036083B0044649B308460D46F2F750F8EF
:100360000746A8B101AA002100F044F8012F064673
:1003700000F10C0311D0184629463A46F1F7A8FBC4
:1003800003460F4A96420BD12046636003B0F0BD8E
:100390000C4B6360204603B0F0BD2A780273F0E78F
:1003A0000022B26037603E443273EDE70648FFF743
:1003B00055FA2046FEF71CFDFEF7CCFB481101085C
:1003C000E8110020F41100207C11010810B504464A
:1003D000FFF7BCFF014B2360204610BD5C110108F4
:1003E00010B50446FFF7B2FF014B2360204610BD55
:1003F000701101081B4B984210B530D88842044652
:100400001CD94A00904238BF144604F11D02B2F5CF
:10041000805F04F10D0018D98C4216D9C2F30B028B
:1004200004F58054A41A9C4228BF1C4604F10D0018
:10043000FFF73AF90022C0E9014210BD00F11D03A7
:10044000B3F5805F00F10D0001D9002805DBFFF74F
:100450002BF90022C0E9014210BDFFF7EFF9024875
:10046000FFF714FAFCFFFF3FA8110108FFF748BD92
:1004700008B5F0F7D5FF08B5FFF7FAFF024B13B147
:100480000248F0F7D5BF704700000000491400088B
:10049000F8B500BFF8BC08BC9E467047F8B500BF71
:0804A000F8BC08BC9E46704741
:1004A800080000202020202020202020202020209C
:1004B8002020202030303030303030303030303074
:1004C80030303030002020202020202020202828F4
:1004D80028282820202020202020202020202020FC
:1004E800202020202088101010101010101010103C
:1004F800101010101004040404040404040404106C
:1005080010101010101041414141414101010101F9
:1005180001010101010101010101010101010101C3
:1005280010101010101042424242424202020202CF
:100538000202020202020202020202020202020293
:100548001010101020000000000000000000000043
:100558000000000000000000000000000000000093
:100568000000000000000000000000000000000083
:100578000000000000000000000000000000000073
:100588000000000000000000000000000000000063
:100598000000000000000000000000000000000053
:1005A8000000000000000000000000000000000043
:1005B8000000000000000000000000000000000033
:1005C8000000000000000000050000001900000005
:1005D8007D00000000000000000000000000F03F67
:1005E8000000000000002440000000000000594006
:1005F8000000000000408F40000000000088C34059
:1006080000000000006AF8400000000080842E41CD
:1006180000000000D01263410000000084D7974119
:100628000000000065CDCD41000000205FA002421F
:10063800000000E876483742000000A2941A6D4294
:10064800000040E59C30A2420000901EC4BCD64287
:1006580000003426F56B0C430080E03779C3414332
:1006680000A0D8855734764300C84E676DC1AB43A8
:10067800003D9160E458E143408CB5781DAF1544C6
:1006880050EFE2D6E41A4B4492D54D06CFF08044A1
:10069800F64AE1C7022DB544B49DD9794378EA44B6
:1006A800BC89D897B2D29C3C33A7A8D523F6493940
:1006B8003DA7F444FD0FA5329D978CCF08BA5B2562
:1006C800436FAC642806C80A0080E03779C3414309
:1006D800176E05B5B5B89346F5F93FE9034F384DA0
:1006E800321D30F94877825A3CBF737FDD4F15754C
:1006F80020202020202020202020202020202020F2
:1007080030303030303030303030303030303030E1
:1007180020202020202020202020202020202020D1
:1007280030303030303030303030303030303030C1
:1007380062617369635F737472696E673A3A5F4D99
:100748005F636F6E737472756374206E756C6C2062
:100758006E6F742076616C696400766563746F727D
:100768003A3A5F4D5F7265616C6C6F635F696E7377
:100778006572740066616C7365007472756500203B
:1007880020202020526576203538323061386100CB
:1007980020202020202A2A2A2A2A2A2A2A2A2A20ED
:1007A80020202020002020207777772E726F627417
:1007B8006F722E64652020200054616E6B004B61BF
:1007C8006C2E20556E742E2050756E6B74004B6124
:1007D8006C2E204F622E2050756E6B74004B205586
:1007E8006E74656E004B204F62656E004D696E2E0B
:1007F800204675656C6C73742E0048797374657245
:1008080065736500496E762052656C616973004EA8
:100818006163687370656973756E67004E616368BC
:1008280073702E20616B742E004E6F746162736357
:1008380068616C742E004E6F744162732E20496E8D
:10084800762E00417566662E2062697300576172C4
:1008580074657A6569740048617570746D656E7544
:100868000053706569636865726E004C6164656EFB
:100878000048656C6C6F2066726F6D20466C6F6106
:100888007450554D5020436F6E74726F6C6C657266
:10089800005265766973696F6E3A20353832306177
:1008A8003861004675656C6C7374616E6420202035
:1008B800202533642025250054616E6B2057617311
:1008C8007365726D616E67656C2020200054616EDF
:1008D8006B204E6F726D616C20202020202020201C
:1008E80020004E6163687370656973756E67206C6C
:1008F800616575667420004E61636873706569731D
:10090800756E6720696E616B746976004E73702E20
:10091800207761727465743A20253364206D696E9E
:10092800004E73702E207761727465743A202533F7
:100938006420736563004E616368737065697375DD
:100948006E67206D616E67656C20004E6163687329
:1009580070656973756E67206F6B202020202000FA
:100968007B22537461747573223A20747275652CF6
:10097800202254616E6B4C6576656C223A2025689E
:1009880068642C202254616E6B50756D70223A2079
:1009980025732C2022526566696C6C50756D702227
:1009A8003A2025732C2022526566696C6C456D705F
:1009B8007479223A2025732C2022526566696C6C62
:1009C800436F6F6C646F776E223A20256868642CD9
:1009D8002022486F75726C7948697374223A202511
:1009E8006868642C20224461696C794869737422B0
:1009F8003A20256868642C207D004E39666C6F614A
:100A08007470756D70346D656E753130494D656EF5
:100A180075456E7472794500E40D0108020A0108F3
:100A28004E39666C6F617470756D70346D656E7576
:100A3800394D656E75456E74727949624545000099
:100A48004C0F0108280A0108200A01084E39666C73
:100A58006F617470756D70346D656E75394D656E46
:100A680075456E7472794974454500004C0F01084C
:100A7800540A0108200A01084E39666C6F617470C7
:100A8800756D70346D656E75394D656E75456E742E
:100A980072794968454500004C0F0108800A010831
:100AA800200A010800000000480A010800000000B0
:100AB80000000000E5F60008E5F60008E5F6000885
:100AC800E5F60008E5F6000800000000740A0108D1
:100AD8000000000000000000E5F60008E5F6000848
:100AE800E5F60008E5F60008E5F600080000000055
:100AF800A00A01080000000000000000E5F6000858
:100B0800E5F60008E5F60008E5F60008E5F6000851
:100B180000000000000000000102030406070809A5
:100B280000000000010203044014544552524F5281
:100B3800004F4E20004F4646005B2D5D005B585D20
:100B4800003E20003E202500766563746F723A3AB5
:100B580072657365727665003C2D205A75727565ED
:100B6800636B003030303130323033303430353030
:100B78003630373038303931303131313231333144
:100B8800343135313631373138313932303231322A
:100B98003232333234323532363237323832393310
:100BA8003033313332333333343335333633373309
:100BB80038333934303431343234333434343534EE
:100BC80036343734383439353035313532353335D4
:100BD80034353535363537353835393630363136BA
:100BE80032363336343635363636373638363937A0
:100BF8003037313732373337343735373637373799
:100C0800383739383038313832383338343835387D
:100C18003638373838383939303931393239333963
:100C28003439353936393739383939004C0F0108F4
:100C3800640C0108480A01084C0F0108880C0108D7
:100C4800740A01084C0F0108AC0C0108A00A01083D
:100C58004C0F0108D00C0108480A01084E39666C8F
:100C68006F617470756D70346D656E7531364D6574
:100C78006E75456E7472794578656375746545005F
:100C88004E39666C6F617470756D70346D656E7514
:100C980031364D656E75456E7472794E756D657237
:100CA800696345004E39666C6F617470756D703498
:100CB8006D656E7531364D656E75456E7472795019
:100CC800657263656E7445004E39666C6F61747049
:100CD800756D70346D656E7531384D656E75456E20
:100CE800747279436865636B61626C6545000000E6
:100CF80000000000340C010839DD000851DD00084F
:100D080079DB000865DB000867DB000869DB0008A1
:100D180075DF000800000000400C010881DC0008B5
:100D280099DC000881DB00088FDB000899DB0008EC
:100D3800A3DB000849E00008000000004C0C010893
:100D480055DC00086DDC0008A9DB0008B7DB0008EB
:100D5800C5DB0008D1DB00085DE1000800000000E9
:100D6800580C01080DDD000825DD00086DDB0008C2
:100D78005DDB00085FDB000861DB00082DDF000891
:100D88002D2D20455252202D2D00202020202020BE
:100D980020202020202020202020202020000003A8
:100DA800010300004C0F0108B80D0108700F01087D
:100DB8004E31305F5F637878616269763131375FD1
:100DC8005F636C6173735F747970655F696E666F7A
:100DD8004500000000000000AC0D010895EA00087D
:100DE800A9EA00080DF800080DF8000825EB00082E
:100DF80055EA000809EB0008C5EA000889EA000876
:100E08007374643A3A657863657074696F6E00004C
:100E18007374643A3A6261645F6578636570746993
:100E28006F6E0000E40D0108500E0108E40D010882
:100E3800700E01084C0F0108940E0108480E0108B5
:100E4800E40D0108A80E01084E31305F5F63787821
:100E5800616269763131355F5F666F726365645FC1
:100E6800756E77696E6445004E31305F5F637878E0
:100E7800616269763131395F5F666F726569676E85
:100E88005F657863657074696F6E450053743133BC
:100E98006261645F657863657074696F6E000000F5
:100EA800537439657863657074696F6E000000006B
:100EB800000000003C0E0108F5ED000809EE0008EE
:100EC80001EE00084C0F0108D80E0108480E010871
:100ED8004E395F5F676E755F63787832307265632D
:100EE8007572736976655F696E69745F6572726F32
:100EF8007245000000000000CC0E01086DF60008E5
:100F080081F60008F9ED00084C0F01081C0F0108D4
:100F1800AC0D01084E31305F5F63787861626976A5
:100F28003132305F5F73695F636C6173735F7479CB
:100F380070655F696E666F45000000000000000084
:100F4800100F0108EDF6000801F700080DF8000879
:100F58000DF8000825EB000855EA0008DDF7000841
:100F680059F700081DF70008E40D0108780F01087B
:100F7800537439747970655F696E666F000000009C
:100F88006E6F7420656E6F75676820737061636536
:100F980020666F7220666F726D617420657870616B
:100FA8006E73696F6E2028506C6561736520737568
:100FB800626D69742066756C6C2062756720726555
:100FC800706F72742061742068747470733A2F2F74
:100FD8006763632E676E752E6F72672F627567730E
:100FE8002F293A0A20202020000000003031323317
:100FF800343536373839000062617369635F73745A
:1010080072696E673A3A5F4D5F6372656174650035
:1010180025733A205F5F706F73202877686963686B
:1010280020697320257A7529203E20746869732DFC
:101038003E73697A6528292028776869636820697A
:101048007320257A7529000062617369635F737480
:1010580072696E673A3A5F4D5F7265706C6163657D
:101068005F6175780000000062617369635F737483
:1010780072696E673A3A7265706C61636500000068
:1010880062617369635F737472696E673A3A5F4D40
:101098005F7265706C616365000000007374643A88
:1010A8003A6261645F616C6C6F6300004C0F010809
:1010B800C0100108480E01085374396261645F6109
:1010C8006C6C6F630000000000000000B4100108A1
:1010D800D1FE0008E5FE0008C9FE00084C0F010813
:1010E80008110108480E01084C0F010818110108E1
:1010F800E41001084C0F01082C110108E410010844
:10110800537431316C6F6769635F6572726F720017
:10111800537431326C656E6774685F6572726F7292
:1011280000000000537431326F75745F6F665F7230
:10113800616E67650000000000000000E41001080F
:10114800B501010875020108B1010108000000009D
:10115800F0100108F501010805030108B1010108B3
:1011680000000000FC10010835020108BD0201085A
:10117800B101010862617369635F737472696E67B4
:101188003A3A5F535F636F6E737472756374206E5F
:10119800756C6C206E6F742076616C696400000059
:1011A80062617369635F737472696E673A3A5F5319
:1011B8005F63726561746500494E4600696E66003A
:1011C8004E414E006E616E00303132333435363761
:1011D800383961626364656600000000303132337B
:1011E800343536373839414243444546000000001B
:1011F800286E756C6C290000300000004E614E00AE
:10120800496E66696E6974790000000042616C6C11
:101218006F6320737563636565646564000000002F
:101228002E2E2F2E2E2F2E2E2F2E2E2F2E2E2F2ED1
:101238002E2F2E2E2F2E2E2F6E65776C69622F6C17
:101248006962632F7374646C69622F64746F612EB2
:10125800630000002E2E2F2E2E2F2E2E2F2E2E2FF7
:101268002E2E2F2E2E2F2E2E2F2E2E2F6E65776C94
:1012780069622F6C6962632F7374646C69622F6D85
:10128800707265632E6300002C2066756E63746946
:101298006F6E3A2000000000617373657274696FA5
:1012A8006E2022257322206661696C65643A206687
:1012B800696C6520222573222C206C696E652025B7
:1012C80064257325730A000043000000504F5349FA
:0812D800580000002E00000088
:1012E000E5DCFF7FB0A90600FFFF010C0C04000045
:1012F0001A04200026040000CDDCFF7FB0A9060000
:10130000FFFF010C0C0400001A042000260400005A
:10131000B5DCFF7FB0A90600FFFF010C0C04000044
:101320001A042000260400009DDCFF7FB0A90600FF
:10133000FFFF010C0C0400001A042000260400002A
:1013400008B10181B0B000840000000079DCFF7FAB
:10135000B0AB0200FFFF010F080400009801049EDB
:101360000100A401040000005DDCFF7FB0B0A80014
:10137000FFFF010816041C002A04000049DCFF7F5F
:10138000B0AA0700FFFF01140C04000012044C0077
:101390001C043A0034045E004804000029DCFF7F8E
:1013A000B0AA0700FFFF01140C04000012044C0057
:1013B0001C043A0034045E004804000009DCFF7F8E
:1013C000AF48B200FFFF01ED0208CE020000EA02C2
:1013D00004F002009003049603009E0304BC030083
:1013E000A60304AC0300B60312A41700CC0304EE5A
:1013F0001600E00304A01700E60304980400F003BD
:10140000048E0400880404B60400B00404A017008D
:10141000CE0404FA0400DA0404F80400F204049888
:101420000500920504A017009C0504C60500A6054A
:1014300004C40500BE0504E40500DE0504A0170091
:10144000CA0604F40600D40604F20600EC0604946E
:1014500007008E0704A01700980704C20700A20720
:1014600004C00700BA0704E20700DC0724A0170045
:10147000820804AC08008C0804AA0800A40804C46C
:101480000800BE0804A01700D608048A1700EC085C
:10149000549E1700C20904FA0900CC0904EA0900A5
:1014A000E40904920A008C0A049E1700AA0A048E1A
:1014B0001700B80A7A9C1700B40B04EA0B00C00BA3
:1014C00004E00B00DA0B04880C00820C049C17006B
:1014D0009E0C04CA0C00AA0C04C80C00C20C04C860
:1014E0000D00C20D729C1700B80E04901700CA0EB2
:1014F000189C1700E60E04921700FE0E049C1700BD
:10150000860F04941700980F189C1700B40F0496C8
:101510001700E20F149C1700FA0F049817008A10A6
:101520000E9C17009C10049A1700C210AA069C1764
:10153000008617040000000008B10181B0B00084EB
:101540000000000081DAFF7FA908B100FFFF010859
:101550001E042C003204000008B10181B0B00084E8
:101560000000000061DAFF7FB0AA0D00FFFF01124A
:101570002C1C8601004C0452005E040000660484AA
:101580000100000041DAFF7FB0A90800FFFF010C55
:101590001A04000024042A003004000029DAFF7F26
:1015A000B0A90800FFFF010C1A04000024042A005F
:1015B0003004000011DAFF7FB0AA0D00FFFF011216
:1015C0002C1C8601004C0452005E0400006604845A
:1015D00001000000F1D9FF7FB0AA0B00FFFF011C42
:1015E000140400001E04700030046800360400007B
:1015F00040047C0052047A0076040000C9D9FF7FC1
:10160000B0AA0D00FFFF01122C1C8601004C0452F1
:10161000005E04000066048401000000A9D9FF7F79
:10162000B0AA0B00FFFF011C140400001E04700090
:10163000300468003604000040047C0052047A0044
:101640007604000081D9FF7FAF08B100FF101901B7
:10165000110E0E0000280466017A047E0082010447
:1016600000000100000000005DD9FF7FB0AF020064
:10167000FF101D01120E0E00002A046A017E048272
:1016800001008601040000010000000000000000CD
:1016900035D9FF7FB0AF0A00FFFF011F2C4C30008F
:1016A00082011CE60200BC01023000E20112FE02CF
:1016B00000C8021C300090030400000009D9FF7F1D
:1016C000B0AF0C00FFFF0126362200008601048A1D
:1016D00001009001040000A201048A0100D2011E51
:1016E0009802009202048A0100A402040000000093
:1016F000D5D8FF7FA908B100FFFF010008B1018123
:10170000B0B0008400000000BDD8FF7FB0AF120071
:10171000FF101901101E98070000D80704A2090144
:10172000C4080400000100000000000099D8FF7FF9
:101730008408B101B0B0B000FF1019010C02060816
:10174000010C0410051E08000001007F00007D0050
:10175000000000000000000008B10181B0B000846A
:101760000000000008B10181B0B00084000000005A
:1017700008B10181B0B000840000000049D8FF7FAB
:10178000B0B0A800FFFF01080E041C00180E0000F6
:1017900035D8FF7FB0B0A800FFFF01080E041C0081
:1017A000180E000021D8FF7FAB029701B0B00FB137
:1017B000FFFF010C300400003E044C00480E000006
:1017C00008B10181B0B000840000000008B10181BF
:1017D000B0B0008400000000EDD7FF7FB0AF040080
:1017E000FF1019010F320A3C01840142CC0100D4E0
:1017F000010400000100000000000000C9D7FF7FC5
:10180000B0AB0200FFFF01081C4A66006C04000038
:1018100008B10181B0B000840000000008B101816E
:08182000B0B0008400000000DC
:1018280050EAFE7F01000000B0EDFE7FB0A9028003
:1018380044EEFE7FB0B0A88094EEFE7F0100000069
:10184800A0EEFE7FB0B0AA80D4EEFE7FAE71B2806B
:1018580098EFFE7F0100000094EFFE7FAB3F3880D9
:10186800F4EFFE7F01000000FCEFFE7FB0B0AA801D
:1018780038F0FE7F01000000E4F0FE7FAA0DB28080
:1018880060F1FE7FB0AF088000F4FE7F0100000029
:1018980004F4FE7FAD3F028080F6FE7F0100000069
:1018A8005CF8FE7F0084048070F8FE7F0100000071
:1018B8006CF8FE7FB0AD048010FBFE7FB0A80380FB
:1018C80034FBFE7F44FFFF7F38FBFE7F48FFFF7F2E
:1018D80044FBFE7F01000000EC73FF7FB0AC098081
:1018E8001475FF7FB0AA0180A875FF7F0100000072
:1018F800EC75FF7FB0AA0B805876FF7FB0A80B80ED
:10190800E476FF7FD4F9FF7F2877FF7FE4F9FF7F34
:101918006C77FF7FF4F9FF7FB077FF7F04FAFF7FD2
:10192800F477FF7FB0B0AA803C78FF7FB0B0AE807C
:101938005079FF7FB0A902807879FF7FFCF9FF7F9B
:101948008879FF7FB0A81380147AFF7FAF08B18031
:10195800BC7AFF7F010000005A7BFF7FE8F9FF7F18
:10196800FA7BFF7FFCF9FF7F247CFF7F01000000EA
:10197800547CFF7FAF08B180FC7CFF7FB0B0A880AB
:10198800167DFF7FF0F9FF7F7A7DFF7F08FAFF7FE2
:10199800E07DFF7F20FAFF7FC089FF7F0100000004
:1019A8004CBEFF7FB0B0A8805EBEFF7F0100000084
:1019B80060BEFF7FB0B0AA807EBEFF7FAB08B1805B
:1019C800D0BEFF7FA908B18054BFFF7FB0A90480B3
:1019D800DCBFFF7FA908B180A4C0FF7F0100000021
:1019E800A0C0FF7F4CFBFF7FAAC0FF7FB0A8038089
:1019F800C4C0FF7FA908B180E4C0FF7FB0B0AA804F
:101A080014C1FF7F38FBFF7F4CC1FF7F010000003E
:101A1800C0C1FF7F3CFBFF7FDCC1FF7F01000000EE
:101A2800E0C1FF7FB0AA018024C2FF7F010000004F
:101A38002CC3FF7FAB08B180C4C3FF7F0100000047
:101A480004C4FF7FB0AA018050C4FF7F10FBFF7F52
:101A5800D4C4FF7F28FBFF7F14C5FF7F38FBFF7FBF
:101A680054C5FF7F48FBFF7FD8C5FF7F60FBFF7F22
:101A780058C6FF7F80FBFF7FDCC6FF7F98FBFF7F98
:101A88005CC7FF7FB0B0A88094C7FF7FB0FBFF7F23
:101A98001CC8FF7FCCFBFF7FA8C8FF7FECFBFF7F44
:101AA80048CAFF7F010000005ECAFF7FB0B0AA806D
:101AB80032CBFF7F0100000070CBFF7FF8FBFF7F78
:101AC800A0CCFF7F010000009ECCFF7FB0B0AA80B1
:101AD80000CDFF7FB0B0AC8046CDFF7F0100000095
:101AE80044CDFF7FB0B0A8805CCDFF7F010000002F
:101AF8005ACDFF7FB0B0AA8074CDFF7FA908B1800E
:101B0800CCCDFF7F0100000044CFFF7FB0AA038047
:101B180070CFFF7F0100000040D0FF7FB0AB028094
:101B2800ECD0FF7F01000000B8D1FF7FBCFBFF7F36
:101B38002CD2FF7F01000000E8D2FF7FB0B0AA805E
:101B4800A0D3FF7FB0FBFF7FE0D3FF7FAB08B1805E
:101B58006CD4FF7FACFBFF7F0CD9FF7FC8FBFF7FF6
:101B68002CD9FF7F0100000038D9FF7FE4FBFF7FFD
:101B780038D9FF7FE8FBFF7F44D9FF7F01000000D1
:101B88005CD9FF7FB0B0A88098D9FF7F0100000022
:101B9800E8D9FF7FB0B0AA8014DAFF7FB0B0A88080
:101BA800B4DAFF7F01000000F8DAFF7FB0B0A88048
:101BB8002CDBFF7F010000001CDCFF7FB0B0AC8095
:101BC80040DCFF7F010000006CDCFF7F9CFBFF7F97
:101BD80084DCFF7FA0FBFF7FACDCFF7FACFBFF7FDB
:101BE800D4DCFF7FB8FBFF7F2CDDFF7FAB1C978029
:101BF80070DDFF7F01000000C8DDFF7FB0B0AC8062
:101C08006CDEFF7FB4FBFF7FACDEFF7F01000000CE
:101C1800B4DEFF7FB0A90280FCDEFF7F0100000078
